:100000000C9478030C9497030C9497030C94970327
:100010000C9497030C9497030C9497030C949703F8
:100020000C9497030C9497030C9459530C94904E92
:100030000C94A2610C9497030C9497030C9497036F
:100040000C9497030C9497030C9497030C949703C8
:100050000C9448170C9497030C9497030C949703F3
:100060000C9497030C9497030C9497030C949703A8
:100070000C9497030C9497030C9497030C94970398
:100080000C9497030C9497030C9497030C94970388
:100090000C9497030C9497036E616E00696E660072
:1000A000456E676C697368005452414E5356455211
:1000B00054455200506F77657220436F6E74726FB3
:1000C0006C00506F776572204D6F64756C650050E1
:1000D0007265737320746865004F464620627574BC
:1000E000746F6E005072657373204F4646006167EF
:1000F00061696E00456E74657220342044696769D9
:10010000742050494E00444320494E004143204949
:100110002F4F00504D20252D32640054253032647D
:1001200058004C4E20256400524C59202564005440
:10013000455354004D41494E0053455455500052CB
:1001400065626F6F74207468652055493F00286FA1
:100150006E6C79207468652055492900504D7320D4
:1001600077697468204572726F72733A004348452C
:100170004D495354525900543133580053657475E6
:100180007000436C6F636B005365742054696D6538
:10019000005465737473004175746F00544C6F772D
:1001A00000544C6F773A00544869676800506F7785
:1001B00065720044432050777200414320507772AB
:1001C00000205553422052455345542020202041C1
:1001D00055544F00414C41524D0052455345540037
:1001E00059454152004D4F00444159004852004D7D
:1001F000494E00555000444F574E00555020313065
:1002000000444F574E203130005550203100444FAC
:10021000574E2031005550202E3100444F574E206C
:100220002E310053415645005642413A0056424253
:100230003A004942413A004942423A005635303A82
:1002400000563530413A00563530423A0056313981
:10025000303A0056494E3A0049494E3A0050494E0C
:100260003A0049523A2000504D00414300487A007C
:10027000564100503A0050663A0043616E63656C27
:1002800000537769746368204F4646004F4E004F15
:1002900046460054696C6C00444320494E0041437B
:1002A00020492F4F004C4F434B004F4B00424154CD
:1002B000004241545445525900534F4C00534F4C47
:1002C00041520048594400485944524F00574E4447
:1002D0000057494E4400475249440053594E434841
:1002E0000047454E45524154004E4F4E450050493F
:1002F0004E005550444154450053455420555050EC
:10030000455200534554204C4F5745520043544CDE
:10031000204C494D4954004C494D495400535552C5
:10032000474500504F55540046414E005042410051
:100330005042420056353000426174746572792033
:1003400042616E6B733A00416D702D487273004DBF
:10035000696E732F42616E6B004C454144004E69DB
:100360004344004C495448004E694D4800434F4EA9
:10037000535452554354494F4E005745540041473A
:100380004D0047454C0041626F7274005265626FC8
:100390006F74004572726F727300414343004348AB
:1003A0004700566572004C494E45530052454C413A
:1003B0005953004B574800204F50454E00434C4F77
:1003C00053450053434845442000454E41424C4567
:1003D000440044495341424C4500494E20004F558A
:1003E00054004F4E20004F46460043484152474973
:1003F0004E47200044495343484152474500204658
:10040000554C4C00454D5054590020564241002057
:10041000564242004E4F4E4520202000534F4C4143
:1004200052202000485944524F20200057494E4442
:1004300020202000475249442020200053594E4399
:1004400048202000313256003234560033365600F0
:10045000464C4F4154494E47004348415247494E4C
:1004600047004F50454E202000434C4F5345440019
:10047000564F5554204241440056313930204241B4
:1004800044004E4F204552524F520006A0FF090132
:10049000A1010902A10006A1FF0903090415802595
:1004A0007F350045FF750895088102090509061585
:1004B00080257F350045FF750895089102C0C01260
:1004C000011001FFFFFF082509222200010102039C
:1004D0000109022900010100C0320904000002FFE5
:1004E000FFFF0009211101000122340007058203EA
:1004F000400001070501034000010403090424032F
:100500004800650061007200740020005400720011
:1005100061006E0073007600650072007400650073
:100520007200000026034800540032003000300002
:10053000300020005400720061006E0073007600ED
:100540006500720074006500720000001C03540016
:1005500052003000300030003100300030003300F5
:10056000310032003300340000008E008E0287001C
:100570008700840287028702840289008B008D0035
:1005800089028B028D0288008A008C0088028A0210
:100590008C020B000F000B020F020A000E000A0271
:1005A0000E0209000D0009020D0208000C000802ED
:1005B0000C0207008100830007028102830206000B
:1005C0008000820006028002820285028502850286
:1005D000850202000500020205020100040001027A
:1005E0000402CF08CF08CF08CF0ACF0ACF0A0000F5
:1005F00003000002030200407A10F35A00A0724E7A
:1006000018090010A5D4E80000E87648170000E4B7
:100610000B54020000CA9A3B000000E1F5050000FF
:1006200080969800000040420F000000A086010064
:100630000000102700000000E80300000000640034
:10064000000000000A00000000000100000000009F
:100650002C76D888DC674F0823DFC1DFAE59E1B1C3
:10066000B796E5E3E453C63AE651997696E8E6C2D2
:100670008426EB898C9B62ED407C6FFCEFBC9C9FD9
:1006800040F2BAA56FA5F490055A2AF75C936B6CFB
:10069000F9676DC11BFCE0E40D47FEF520E6B500EF
:1006A000D0ED902E0300943577050080841E08005D
:1006B00000204E0A000000C80C333333330F986E0D
:1006C00012831141EF8D2114893BE65516CFFEE6CA
:1006D000DB18D1844B381BF77C1D901DA4BBE42490
:1006E000203284725E228100C9F124ECA1E53D270D
:1006F00011241FBECFEFD0E2DEBFCDBF1BE0A0E0D4
:10070000B1E0E8E9F1E501E00BBF02C007900D920E
:10071000A03EB107D9F714E1A0EEBBE001C01D92E5
:10072000AB3FB107E1F70E9421610C94CAA80C9479
:1007300000008091E00B882311F4409A0895419ABB
:1007400008958091E00B882311F440980895419812
:1007500008958093E00B08950E94990300C00E94C1
:10076000A10308951F93662311F0429A01C0429895
:1007700043983C9A3D9A3E9A3F9A479846984598A6
:10078000449887FD479A182F86FD469A15FD459A8D
:1007900014FD449A0E94AC034798469845984498A3
:1007A00013FD479A12FD469A11FD459A10FD449A91
:1007B0000E94AC03449A459A469A479A1F9108951D
:1007C0001F93882311F0429A01C04298439A3C98A3
:1007D0003D983E983F980E94990300C0349B02C008
:1007E00010E101C010E03599106236991064379914
:1007F00010680E94A10300C00E94990300C03499B0
:1008000011603599126036991460379918600E940A
:10081000A103812F1F910895CF93DF93C8EED3E0FA
:1008200004C0219739F00E94196180E00E94E00322
:1008300087FDF7CF84E090E00197F1F780E00E9418
:10084000E00390E0DF91CF9108950E940C0481E0D5
:100850000E94E00308951F93182F0E940C04812F1B
:1008600061E00E94B2031F9108951F93182F0E9408
:100870000C04812F60E00E94B2031F910895DF9263
:10088000EF92FF920F931F93CF93DF93D82E109286
:10089000E00B3A9A3B9A389A399A3C9A3D9A3E9A9A
:1008A0003F9A80E09DE70197F1F7C0E0D0E0E12CAE
:1008B00087E2F82E00E810E0C093E00B459A449AD6
:1008C0000E94AC03C7010197F1F70E94AC03C80175
:1008D0000197F1F70E94AC03C8010197F1F7449822
:1008E0000E94AC03C8010197F1F788E20E94350429
:1008F00088E00E94350481E00E94350486E00E9471
:1009000035048D2D0E9435042196C230D105A1F603
:10091000DF91CF911F910F91FF90EF90DF9008959D
:100920001092E00B662319F091E09093E00B877032
:10093000880F880F880F805C0E943504089564300A
:1009400008F063E070E0FB01E050FF4F908190936E
:10095000E00B80586C5F7E4FFB019081890F0E94F5
:10096000350408951F93182F0E940C041A3049F47F
:10097000803410F080E001C080E480580E9435048B
:1009800004C0812F61E00E94B2031F9108950F936C
:100990001F93DF93CF930F92CDB7DEB78C0106C0C4
:1009A0000F5F1F4F69830E94B2046981662329F09B
:1009B000F80180816150882399F70F90CF91DF91E2
:1009C0001F910F910895CF93DF93EC0102C00E9415
:1009D000B20489918823D9F7DF91CF9108959EBD04
:1009E0000DB407FEFDCF3EB58EBD0DB407FEFDCFA5
:1009F0002EB5932F80E030E0282B392BC9010895C4
:100A0000E4E6F0E080818B7F808384B1866084B9E6
:100A100089E58CBD8DB58EB508958EBD0DB407FEEC
:100A2000FDCF8EB50895FC01862F972F2FEF07C0BD
:100A30002EBD0DB407FEFDCF3EB5319301971816BC
:100A40001906B4F30895262F372F0AC0FC01408100
:100A50004EBD0DB407FEFDCF01964EB5215030407E
:100A6000121613069CF308950E94EF0408950F9345
:100A70001F93CF93DF93EC01062F172F08C080E060
:100A800090E00E94EF048993999301501040101652
:100A90001106ACF3DF91CF911F910F9108950F9341
:100AA0001F93CF93DF93EC01062F172F06C0899178
:100AB00099910E94EF040150104010161106BCF3EA
:100AC000DF91CF911F910F910895E091FF14F09164
:100AD0000015E550FB4E808108958091FF149091A0
:100AE0000015019797FF02C083E090E085509B4E70
:100AF000FC01808108952BEF34E1E091FF14F09127
:100B00000015E20FF31F9081290F311DF901808339
:100B1000089509966AE070E00E9442A67093EF0B78
:100B20006093EE0B08958AE090E09093EF0B809332
:100B3000EE0B0E941A128091CF1181508093CF1139
:100B40008CE00E943504E091FF14F0910015E5500F
:100B5000FB4EE081F0E0EE0FFF1FE85FFE4F0190DB
:100B6000F081E02D0190F081E02D09958091CF1169
:100B70008F5F8093CF1108958091FF14909100159D
:100B8000FC01E550FB4E22E02083019797FF02C055
:100B900083E090E0909300158093FF14FC01E550F2
:100BA000FB4E8081882311F482E080830E949305AC
:100BB0000895E091FF14F0910015E550FB4E8083FD
:100BC0000E94930508952091FF14309100152F5F26
:100BD0003F4F2430310514F020E030E03093001511
:100BE0002093FF1425503B4EF90180830E9493050A
:100BF00008958DE00E94E305089588E10E94E305D1
:100C0000089583E00E94E30508958CE00E94E305C7
:100C1000089582E00E94E3050895CF92DF92EF925B
:100C2000FF920F931F93DF93CF930F92CDB7DEB751
:100C3000982F6B0180E0692F49830E949F0400E098
:100C400010E04981E42EFF2407C00E942504F6012C
:100C500081936F010F5F1F4F0E151F05B4F30F90A7
:100C6000CF91DF911F910F91FF90EF90DF90CF9088
:100C70000895CF93DF93682F80E00E949F04CAE716
:100C8000D1E189910E94B20481E1CE38D807C9F739
:100C9000DF91CF9108950E94E30408950F931F936D
:100CA000DF93CF93CDB7DEB766970FB6F894DEBF6C
:100CB0000FBECDBF2DB73EB7285030400FB6F894C9
:100CC0003EBF0FBE2DBFEDB7FEB731968E010F5F51
:100CD0001F4FADB7BEB712961C930E93119725E127
:100CE00030E03383228375836483978386834E8BBE
:100CF0000E94CEA72DB73EB7285F3F4F0FB6F8949E
:100D00003EBF0FBE2DBFC8014E89642F0E94C7048D
:100D100066960FB6F894DEBF0FBECDBFCF91DF91C0
:100D20001F910F9108950F931F93DF93CF93CDB72A
:100D3000DEB766970FB6F894DEBF0FBECDBFADB776
:100D4000BEB71A970FB6F894BEBF0FBEADBFEDB7D2
:100D5000FEB731968E010F5F1F4F12961C930E93B4
:100D60001197A5E1B0E0B383A283558344836683E2
:100D70007783808791872E8B0E94CEA7EDB7FEB731
:100D80003A960FB6F894FEBF0FBEEDBFC8012E898C
:100D9000622F0E94C70466960FB6F894DEBF0FBE9E
:100DA000CDBFCF91DF911F910F910895EF92FF92E8
:100DB0000F931F937A018B010E9417688091FB0D9E
:100DC0009091FC0DA091FD0DB091FE0D8093E50B6F
:100DD0009093E60BA093E70BB093E80BC801B70123
:100DE000675F7F4F8F4F9F4F2AE030E040E050E039
:100DF0000E9456A62093E90B3093EA0B4093EB0B2D
:100E00005093EC0B1F910F91FF90EF9008958091FC
:100E1000ED0B882329F090911B12933009F084E0A8
:100E200040E050E0BA010E94D6060895823060F496
:100E3000E091FF14F0910015E550FB4E808169E0D0
:100E400070E00E94EC270895843071F0833071F4D3
:100E50008091E90B9091EA0BA091EB0BB091EC0B18
:100E60000097A105B10511F40E9407070895CF92DC
:100E7000DF92EF92FF920F931F93809117138823B5
:100E800061F08091CF1181508093CF110E94E8359D
:100E90008091CF118F5F8093CF110E945C098823CE
:100EA00009F437C18091CF1181508093CF1180E137
:100EB00090E00E946709882399F0E091FF14F09177
:100EC0000015E550FB4EE081F0E0EE0FFF1FE85FFC
:100ED000FE4F0190F081E02D0684F785E02D18C0CB
:100EE00088E090E00E9467098823A9F0E091FF1450
:100EF000F0910015E550FB4EE081F0E0EE0FFF1F92
:100F0000E85FFE4F0190F081E02D0088F189E02D2F
:100F1000309709F0099582E090E00E9467098823E4
:100F200099F0E091FF14F0910015E550FB4EE0813F
:100F3000F0E0EE0FFF1FE85FFE4F0190F081E02D23
:100F40000488F589E02D18C084E090E00E946709CC
:100F50008823A9F0E091FF14F0910015E550FB4EB5
:100F6000E081F0E0EE0FFF1FE85FFE4F0190F0819F
:100F7000E02D0288F389E02D309709F0099580E093
:100F800091E00E946709882399F0E091FF14F091A5
:100F90000015E550FB4EE081F0E0EE0FFF1FE85F2B
:100FA000FE4F0190F081E02D0680F781E02D4AC0D0
:100FB00080E890E00E946709882399F0E091FF148F
:100FC000F0910015E550FB4EE081F0E0EE0FFF1FC1
:100FD000E85FFE4F0190F081E02D0084F185E02D67
:100FE00031C080E490E00E946709882399F0E09185
:100FF000FF14F0910015E550FB4EE081F0E0EE0F9C
:10100000FF1FE85FFE4F0190F081E02D0284F38521
:10101000E02D18C080E290E00E9467098823A9F0C3
:10102000E091FF14F0910015E550FB4EE081F0E0F7
:10103000EE0FFF1FE85FFE4F0190F081E02D04846A
:10104000F585E02D309709F0099580E092E00E9447
:1010500067098823A9F0E091FF14F0910015E5508D
:10106000FB4EE081F0E0EE0FFF1FE85FFE4F0190C6
:10107000F081E02D0480F581E02D309709F009958D
:1010800080911B12833011F084E001C08CE048E8AD
:1010900053E160E070E00E94D60681E090E00E949B
:1010A0006709882381F1E091FF14F0910015E55064
:1010B000FB4EE081F0E0EE0FFF1FE85FFE4F019076
:1010C000F081E02D0688F789E02D309711F0099521
:1010D0001AC080911B128823B1F08091ED0B8C30E7
:1010E00010F48C5F01C084E08093ED0B8091ED0BD8
:1010F00068E070E00E94EC278091ED0B40E050E04A
:10110000BA010E94D6068091CF118F5F8093CF11D4
:1011100028C02091E90B3091EA0B4091EB0B5091E4
:10112000EC0B2115310541055105D9F08091FB0DDE
:101130009091FC0DA091FD0DB091FE0DE090E50B9E
:10114000F090E60B0091E70B1091E80B8E199F09C8
:10115000A00BB10B82179307A407B50710F00E94EC
:1011600007072091E10B3091E20B4091E30B509186
:10117000E40B8091FB0D9091FC0DA091FD0DB091C1
:10118000FE0D281739074A075B07D1F16C017D0175
:10119000C21AD30AE40AF50A4091EE0B5091EF0B04
:1011A00060E070E0C416D506E606F70648F18093C5
:1011B000E10B9093E20BA093E30BB093E40BE0916F
:1011C000FF14F0910015E550FB4EE081F0E0EE0FCA
:1011D000FF1FE85FFE4F0190F081E02D8281938137
:1011E000009771F08091CF1181508093CF110280D0
:1011F000F381E02D09958091CF118F5F8093CF11FE
:101200001F910F91FF90EF90DF90CF90089588E0AD
:1012100090E064E04CE024E00E94F9278093ED0B1D
:101220008091E21280FD07C08091FF14909100151B
:1012300084309105B0F080E04AEF50E060E070E06B
:101240000E94D6061092FB141092FC141092FD140A
:101250001092FE14109200151092FF140E94311F7C
:1012600002C00E9407071092CF1180E00E94E305A0
:1012700008952091F40B3091F50B282B392B3093E6
:10128000F50B2093F40B089580E02091F00B309142
:10129000F10B33702115310509F081E0089540E02C
:1012A0002091F00B3091F10B2823392321153105C2
:1012B00009F041E0842F089580E02091F20B3091F5
:1012C000F30B33702115310509F081E0089540E0FA
:1012D0002091F20B3091F30B28233923211531058E
:1012E00009F041E0842F08950E9468646091F00B3A
:1012F0007091F10B9093F10B8093F00B2FB7F89452
:101300004091F40B5091F50B1092F50B1092F40BE9
:1013100027FF01C078942091F00B3091F10B8627C4
:10132000972782239323842B952B9093F30B809301
:10133000F20B242B352B3093F10B2093F00B0895F7
:1013400080E092E09093F10B8093F00B0E9474097F
:10135000089580918F11882321F481E080938F116B
:10136000089510928F110895AF92BF92CF92DF929D
:10137000EF92FF920F931F93DF93CF93CDB7DEB71A
:1013800029970FB6F894DEBF0FBECDBF80911B1218
:10139000882309F481C18091C1128F3F09F485C16E
:1013A0008091C3128F3708F080C190918F11809186
:1013B0001712992351F50E940F6660939411709350
:1013C000951180939611909397118091171290E048
:1013D0000E941B65609398117093991180939A11E4
:1013E00090939B118091171290E00E9495656093F5
:1013F0009C1170939D1180939E1190939F118091E9
:10140000171290E00E94D9642AC090E00E944C66B6
:101410006093941170939511809396119093971106
:101420008091171290E00E94586560939811709314
:10143000991180939A1190939B118091171290E0CB
:101440000E94D26560939C1170939D1180939E11B0
:1014500090939F118091171290E00E94D564609341
:10146000A8117093A9118093AA119093AB11809148
:10147000171290E00E94DD646093AC117093AD117F
:101480008093AE119093AF1160919411709195116A
:101490008091961190919711209198113091991106
:1014A00040919A1150919B110E9404A5D62EC72EEF
:1014B000B82EA92EA6019501652F742F832F922F88
:1014C00020E030E040EA50E40E9400A518165CF0ED
:1014D0000F2EF0E0EF2EF0E0FF2EF0E00F2FF0E007
:1014E0001F2FF02D33C060919C1170919D11809140
:1014F0009E1190919F11D601F5012B2F3A2F4F2F5E
:101500005E2F0E94B5A3E62EF72E082F192F20E09C
:1015100030E0A9010E94B1A3882324F417FB1095A1
:1015200017F91095C801B70120E030E040E85FE30B
:101530000E9400A5181654F40F2EF0E0EF2EF0E0F4
:10154000FF2EF0E80F2FFFE31F2FF02D83E060E068
:101550000E949F04E0918F11F0E0EE0FFF1FE15712
:10156000FE4E818192810E94E3048DE060E00E9442
:101570009F046091AC117091AD118091AE1190916A
:10158000AF114AE551E026E00E94930680E061E059
:101590000E949F0460919411709195118091961111
:1015A000909197114AE551E026E00E9493068BE066
:1015B00061E00E949F048091171290E0019660E61E
:1015C00071E042E00E944E068DE061E00E949F04BF
:1015D000609198117091991180919A1190919B113D
:1015E0004AE551E026E00E94930683E062E00E9413
:1015F0009F0460919C1170919D1180919E1190911A
:101600009F1145E651E027E00E9493068BE062E0DF
:101610000E949F04A6019501652F7C2D832F9A2D92
:1016200045E651E027E00E94930683E063E00E94D4
:101630009F04C801B7014BE651E027E00E949306E2
:101640008BE063E00E949F0460919411709195116A
:10165000809196119091971120E030E0A9010E94AD
:10166000B1A3882359F480E090E0DC018093A811B5
:101670009093A911A093AA11B093AB116091A811F6
:101680007091A9118091AA119091AB114BE651E094
:1016900028E00E94930668C0CE01019666E372E0DE
:1016A0000E9481A706E312E008C0CE0101966EE316
:1016B00072E00E9481A70EE312E083E062E00E94E4
:1016C0009F047E010894E11CF11CC7010E944B0697
:1016D0008BE062E00E949F04C7010E944B0683E0FA
:1016E00063E00E949F04C7010E944B068BE063E009
:1016F0000E949F04C7010E944B06B8016F5F7F4F95
:10170000C7010E9481A783E060E00E949F04E091EE
:101710008F11F0E0EE0FFF1FE157FE4E81819281A5
:101720000E94E3048DE060E00E949F04C7010E94D4
:101730004B0680E061E00E949F04C7010E944B06B7
:101740008BE061E00E949F048091171290E0019667
:1017500060E671E042E00E944E068DE061E00E948A
:101760009F04C7010E944B0629960FB6F894DEBF6E
:101770000FBECDBFCF91DF911F910F91FF90EF90E2
:10178000DF90CF90BF90AF900895EF92FF920F93AC
:101790001F93CF93DF9381E080938F118FE70E9497
:1017A0005E12909391118093901180E80E945E12D6
:1017B000909393118093921184EF91E00E94890598
:1017C000CAE7D1E1CE0160E270E044E150E00E945E
:1017D00071A780E40E945E12BC01FC010190002010
:1017E000E9F73197E81BF90BCE01AF010E9468A71A
:1017F0008AE30E945E12BC01FC0101900020E9F71F
:101800003197E81BF90B9E01295F3F4FC901AF01DA
:101810000E9468A786E580938D1180E090E00E9489
:101820003906CE0160E270E044E150E00E9471A709
:101830008FE30E945E12BC01FC0101900020E9F7D9
:101840003197E81BF90B9E01285F3F4FC901AF019B
:101850000E9468A781E480938D1181E090E00E944E
:101860003906CE0160E270E044E150E00E9471A7C9
:1018700083E40E945E12BC01FC0101900020E9F7A4
:101880003197E81BF90BCE01AF010E9468A787E5ED
:101890008093831182E40E945E12BC01FC010190DE
:1018A0000020E9F73197E81BF90B8E010E5E1F4F00
:1018B000C801AF010E9468A782E090E00E9439064B
:1018C000CE0160E270E044E150E00E9471A784E440
:1018D0000E945E12BC01FC0101900020E9F73197E3
:1018E000E81BF90BCE01AF010E9468A781E40E94BA
:1018F0005E12BC01FC0101900020E9F73197E81B62
:10190000F90BC801AF010E9468A783E090E00E9434
:1019100039060E94B409DF91CF911F910F91FF907A
:10192000EF900895EF92FF920F931F93DF93CF9361
:10193000CDB7DEB729970FB6F894DEBF0FBECDBF87
:101940008091171290E00E94876760938F117093C7
:10195000901180939111909392118091171290E0C1
:101960000E948167609393117093941180939511F5
:10197000909396118091171290E00E94D367609324
:101980009711709398118093991190939A11809167
:10199000171290E00E94CD6760939B1170939C1189
:1019A00080939D1190939E118091171290E00E9458
:1019B0007B6760939F117093A0118093A111909306
:1019C000A2118091171290E00E9495676093A31175
:1019D0007093A4118093A5119093A6118091171272
:1019E00090E00E94DD646093A7117093A81180932A
:1019F000A9119093AA1180911B12882309F488C021
:101A00008091C1128F3F09F48EC084E060E00E9493
:101A10009F0460918F11709190118091911190911C
:101A2000921149E851E027E00E9493068CE060E0C3
:101A30000E949F0460919711709198118091991163
:101A400090919A1149E851E027E00E94930684E0C2
:101A500061E00E949F0460919311709194118091B4
:101A600095119091961149E851E027E00E94930664
:101A70008CE061E00E949F0460919B1170919C1129
:101A800080919D1190919E1149E851E027E00E94BC
:101A9000930684E062E00E949F0460919F11709120
:101AA000A0118091A1119091A21149E851E027E085
:101AB0000E9493068CE062E00E949F046091A31153
:101AC0007091A4118091A5119091A61149E851E05F
:101AD00027E00E9493068091C3128F3790F485E02F
:101AE00063E00E949F046091A7117091A8118091FA
:101AF000A9119091AA114FE851E026E00E949306A7
:101B000056C085E063E00E949F048FE392E04DC0E1
:101B1000CE01019666E372E00E9481A796E3E92E6A
:101B200092E0F92E0AC0CE0101966EE372E00E94A7
:101B300081A78EE3E82E82E0F82E84E060E00E9428
:101B40009F048E010F5F1F4FC8010E944B068CE05F
:101B500060E00E949F04C8010E944B0684E061E09F
:101B60000E949F04C8010E944B068CE061E00E9425
:101B70009F04C8010E944B0684E062E00E949F041B
:101B8000C8010E944B068CE062E00E949F04C801DD
:101B90000E944B06B7016F5F7F4FC8010E9481A76B
:101BA00085E063E00E949F04C8010E944B0682E129
:101BB00063E00E949F048091171290E0019665E90E
:101BC00071E042E00E944E0629960FB6F894DEBFFF
:101BD0000FBECDBFCF91DF911F910F91FF90EF907E
:101BE0000895EF92FF920F931F93CF93DF9384EFAB
:101BF00091E00E948905CAE7D1E1CE0160E270E080
:101C000044E150E00E9471A783E30E945E12BC0190
:101C1000FC0101900020E9F73197E81BF90BCE0198
:101C2000AF010E9468A716E51093851101E40093A7
:101C30008D1180E090E00E943906CE0160E270E0F4
:101C400044E150E00E9471A784E30E945E12BC014F
:101C5000FC0101900020E9F73197E81BF90BCE0158
:101C6000AF010E9468A71093851100938D1181E048
:101C700090E00E943906CE0160E270E044E150E05D
:101C80000E9471A787E30E945E12BC01FC010190D3
:101C90000020E9F73197E81BF90BCE01AF010E9454
:101CA00068A71093851100938D1182E090E00E9447
:101CB0003906CE0160E270E044E150E00E9471A775
:101CC0008AE30E945E12BC01FC0101900020E9F74A
:101CD0003197E81BF90BCE01AF010E9468A7109362
:101CE00085118FE30E945E12BC01FC01019000206F
:101CF000E9F73197E81BF90B2F96CE01AF010E944F
:101D000068A783E090E00E9439060E94920CDF9160
:101D1000CF911F910F91FF90EF90089581E00E9465
:101D2000E30508951F938091FB0D9091FC0DA09108
:101D3000FD0DB091FE0D20919411309195114091BF
:101D4000961150919711821B930BA40BB50B893CF4
:101D50009105A105B105F8F089E090E060E048E266
:101D600020E00E94F927182F8091E21280FD06C022
:101D7000112321F0113011F01A3111F48EE008C056
:101D80000E946D05181719F40E94BC0508C0812F28
:101D90000E94E30504C08FE891E10E9494461F91E0
:101DA00008950F931F93CF93DF93CAE7D1E1CE013C
:101DB00060E270E044E150E00E9471A781E00E947F
:101DC0005E12BC01FC0101900020E9F73197E81B8D
:101DD000F90B04E110E098012E1B3F0B3695279577
:101DE0002C0F3D1FC901AF010E9468A780E090E061
:101DF0000E943906CE0160E270E044E150E00E94AA
:101E000071A781E090E00E94390683E090E00E9493
:101E1000390680E00E945E12BC01FC0101900020A6
:101E2000E9F73197E81BF90B0E1B1F0B1695079569
:101E30000C0F1D1FC801AF010E9468A782E090E04F
:101E40000E94390686E70E945E122DB73EB72451E4
:101E500030400FB6F8943EBF0FBE2DBFEDB7FEB7B2
:101E60003196ADB7BEB71296DC93CE93119725E1AC
:101E700030E03383228322EB31E035832483978360
:101E8000868382E090E0918780878DE190E0938760
:101E9000828782E190E09587848789E090E0978748
:101EA000868780E290E0918B808B81E190E0938B3C
:101EB000828B0E94CEA72DB73EB72C5E3F4F0FB648
:101EC000F8943EBF0FBE2DBF80E063E00E949F04E8
:101ED000CE010E944B068FE891E10E94D646809188
:101EE000FB0D9091FC0DA091FD0DB091FE0D809326
:101EF000941190939511A0939611B0939711DF913F
:101F0000CF911F910F91089581E00E94E3050895FC
:101F10008091171280931A1280911E1280931D12C5
:101F20000E94010608950F931F93DF93CF93CDB7BF
:101F3000DEB728970FB6F894DEBF0FBECDBF8FE88F
:101F400091E10E9494468DB79EB708970FB6F8941A
:101F50009EBF0FBE8DBFEDB7FEB731968E010F5FEE
:101F60001F4FADB7BEB712961C930E93119788E022
:101F700090E0938382838091941190919511958341
:101F800084838091171290E00196978386830E9444
:101F9000CEA7F80101900020E9F78DB79EB708960B
:101FA0000FB6F8949EBF0FBE8DBFC8018E1B9F0B4E
:101FB00045969695879561E00E949F04C8010E940E
:101FC0004B0628960FB6F894DEBF0FBECDBFCF915B
:101FD000DF911F910F910895EF92FF920F931F933E
:101FE000CF93DF938BE00E945E12909395118093C4
:101FF0009411CAE7D1E1CE0160E270E044E150E023
:102000000E9471A781E00E945E12BC01FC01019058
:102010000020E9F73197E81BF90B04E110E0980183
:102020002E1B3F0B369527952C0F3D1FC901AF0185
:102030000E9468A780E090E00E943906CE0160E22D
:1020400070E044E150E00E9471A781E090E00E94BE
:10205000390687E10E945E12BC01FC01019000205C
:10206000E9F73197E81BF90BCE01AF010E9468A791
:1020700080E10E945E12BC01FC0101900020E9F7A2
:102080003197E81BF90B98012E1B3F0B36952795CE
:102090002C0F3D1FC901AF010E9468A78AE10E9471
:1020A0005E12BC01FC0101900020E9F73197E81BAA
:1020B000F90B0E1B1F0B0C0F1D1FC801AF010E9457
:1020C00068A782E090E00E943906CE0160E270E0ED
:1020D00044E150E00E9471A78BE10E945E12BC01B6
:1020E000FC0101900020E9F73197E81BF90B9E01F4
:1020F0002E5F3F4FC901AF010E9468A788E10E948F
:102100005E12BC01FC0101900020E9F73197E81B49
:10211000F90BCE1BDF0B6296CE01AF010E9468A7C0
:1021200083E090E00E9439068FE891E10E94D64654
:10213000DF91CF911F910F91FF90EF9008950F9332
:102140001F93CF93DF93CAE7D1E1CE0160E270E045
:1021500044E150E00E9471A781E00E945E12BC0140
:10216000FC0101900020E9F73197E81BF90B04E12D
:1021700010E098012E1B3F0B369527952C0F3D1F25
:10218000C901AF010E9468A780E090E00E94390673
:10219000CE0160E270E044E150E00E9471A781E06E
:1021A00090E00E943906CE0160E270E044E150E028
:1021B0000E9471A78FE00E945E12BC01FC01019099
:1021C0000020E9F73197E81BF90B0E1B1F0B169542
:1021D00007950C0F1D1FC801AF010E9468A782E080
:1021E00090E00E943906CE0160E270E044E150E0E8
:1021F0000E9471A783E090E00E9439068FE891E188
:102200000E94D646DF91CF911F910F9108950F93B1
:102210001F93DF93CF930F92CDB7DEB70E949F102D
:102220008CE10E945E128C0180E062E00E949F04BB
:10223000C8010E94E30480E20E945E12182FE82F7A
:10224000F92FDF010D900020E9F7EA1B8E2F8B5E3E
:1022500062E099830E949F04812F99810E94E30488
:102260008EE10E945E128C0182E063E00E949F0476
:10227000C8010E94E30481E20E945E12182FE82F39
:10228000F92FDF010D900020E9F7EA1B8E2F8D5EFC
:1022900063E099830E949F04812F99810E94E30447
:1022A0000E941A128BE00E945E1290939511809307
:1022B00094110F90CF91DF911F910F91089580E2BB
:1022C0000E94E305089585E20E94E305089584E2F3
:1022D0000E94E305089583E20E94E305089582E2E7
:1022E0000E94E305089581E20E94E30508958BE1D1
:1022F0000E94E30508950F931F93DF93CF93CDB70B
:10230000DEB728970FB6F894DEBF0FBECDBF8FE8BB
:1023100091E10E9494468DB79EB708970FB6F89446
:102320009EBF0FBE8DBFEDB7FEB731968E010F5F1A
:102330001F4FADB7BEB712961C930E93119788E04E
:1023400090E093838283809194119091951195836D
:1023500084838091171290E00196978386830E9470
:10236000CEA7F80101900020E9F78DB79EB7089637
:102370000FB6F8949EBF0FBE8DBFC8018E1B9F0B7A
:1023800045969695879561E00E949F04C8010E943A
:102390004B0628960FB6F894DEBF0FBECDBFCF9187
:1023A000DF911F910F9108950F931F93DF93CF93A8
:1023B0000F92CDB7DEB780911F12882311F480E20F
:1023C00005C080912012882321F48CE10E94D90558
:1023D0002BC00E949F108FE30E945E128C0182E04E
:1023E00063E00E949F04C8010E94E30486E10E940A
:1023F0005E12182FE82FF92FDF010D900020E9F76A
:10240000EA1B8E2F8D5E63E099830E949F04812FCB
:1024100099810E94E3040E941A128BE00E945E12CE
:1024200090939511809394110F90CF91DF911F910C
:102430000F9108951092F70D1092F60D80E092E042
:10244000E6EFFBE0DF019C011D9221503040E1F7F7
:1024500008950F931F93CF93DF93BC012091F60D46
:102460003091F70D89010A50144F8EEF91E0821BD5
:10247000930BEB0109900020E9F72197C61BD70BBE
:102480008C179D0708F4EC01C801AE010E9488A7D3
:102490008091F60D9091F70D01968C0F9D1FFC0118
:1024A000EA50F44F108201969093F70D8093F60D49
:1024B000C801DF91CF911F910F9108956F927F9284
:1024C0008F929F92AF92BF92CF92DF92EF92FF9244
:1024D0000F931F93DF93CF93CDB7DEB72B970FB634
:1024E000F894DEBF0FBECDBF8B3908F09DC0E090E1
:1024F000F60DF090F70D20E0E21622E0F20608F06B
:1025000093C087010A50144F5FEFC52E51E0D52EBE
:10251000CE18DF089091F80D992309F45DC0282F9B
:1025200030E04091F90D5091FA0D2417350708F06D
:1025300053C0C901880F991F0896BE016F5F7F4F76
:1025400042E00E94C84D89809A8036E1C316D104CA
:1025500014F024E102C02C2D21505801CC2433E08A
:10256000632E712C6C0E7D1E28C0D22E293010F0E7
:1025700098E0D92EC401B3014D2D2B870E94C84D80
:10258000F30180E090E04D2D50E02B850FC03081AD
:10259000D5013C9331910196332329F4FC01EC0DD4
:1025A000F11D6F0112C00894A11CB11C841795077E
:1025B00074F3CD0C2D19840E951E2223B1F6D5018E
:1025C0001C92DD240894C11CD11CCE0CDF1CD092BF
:1025D000F70DC092F60D2AC0E82FF0E0EE0FFF1FB6
:1025E000EA5BFD4F2081318121153105E9F080E062
:1025F00090E005C0F801E80FF91F40830196F9014A
:10260000E80FF91F4491442319F08C159D0594F3AC
:10261000F801E80FF91F108201968E0D9F1D90930F
:10262000F70D8093F60D02C00CE713E0C8012B965E
:102630000FB6F894DEBF0FBECDBFCF91DF911F91D3
:102640000F91FF90EF90DF90CF90BF90AF909F9051
:102650008F907F906F9008950F931F93DF93CF9388
:1026600000D000D0CDB7DEB780E090E08E010F5FE4
:102670001F4FB80144E00E94C84DC80161E372E0F9
:102680000E9478A79C0180E02115310509F481E0C2
:102690008093F80D882349F08091060090910700FF
:1026A00069EF7DE042E00E94C84D0F900F900F90BF
:1026B0000F90CF91DF911F910F9108958CE094E0DE
:1026C0000E94A264BC0180919011882321F0646073
:1026D0001092901104C06B7F81E0809390118CE088
:1026E00094E00E94046808958CE094E00E94A26443
:1026F00020918F11222329F0BC016E7F10928F113F
:1027000005C081E080938F1161E070E08CE094E07F
:102710000E9404680895CF93DF938CE094E00E94B8
:10272000A264EC01C2608CE094E0BE010E940468E7
:102730008FE79AE1A6E081509040A040E1F700C009
:102740000000BE016D7F8CE094E00E940468DF9180
:10275000CF9108950E9427530E943C530895EF9211
:10276000FF920F931F93CF93DF93CAE7D1E1CE017E
:1027700060E270E044E150E00E9471A76091931123
:1027800070919411DB01FD0101900020E9F7319770
:10279000EA1BFB0BCE01AF010E9468A7809190114C
:1027A000882329F06091991170919A1104C0609169
:1027B0009B1170919C11FB0101900020E9F731976A
:1027C000E61BF70B2EE831E1CAE7D1E12E1B3F0BE8
:1027D000C901AF010E9468A780E090E00E9439061D
:1027E000CE0160E270E044E150E00E9471A7609188
:1027F000951170919611DB01FD0101900020E9F720
:102800003197EA1BFB0BCE01AF010E9468A78091B4
:102810008F11882329F06091991170919A1104C049
:1028200060919B1170919C11FB0101900020E9F7D0
:102830003197E61BF70B04E110E098012E1B3F0BCC
:10284000CAE7D1E12C0F3D1FC901AF010E9468A763
:1028500081E090E00E943906CE0160E270E044E140
:1028600050E00E9471A76091951170919611DB0163
:10287000FD0101900020E9F73197EA1BFB0BCE0127
:10288000AF010E9468A76091971170919811DB01C8
:10289000FD0101900020E9F73197EA1BFB0B0E1BAD
:1028A0001F0B0C0F1D1FC801AF010E9468A782E01B
:1028B00090E00E943906CE0160E270E044E150E011
:1028C0000E9471A76091911170919211DB01FD013D
:1028D00001900020E9F73197EA1BFB0B2CE831E16E
:1028E0002E1B3F0BC901AF010E9468A783E090E057
:1028F0000E943906DF91CF911F910F91FF90EF90C9
:10290000089582E20E945E12909392118093911139
:102910008BE10E945E12909394118093931183E255
:102920000E945E12909396118093951184E20E940A
:102930005E1290939811809397118DE70E945E121A
:1029400090939A11809399118EE70E945E12909352
:102950009C1180939B118CE094E00E94A264282F2C
:10296000217020938F1196958795969587958095E0
:102970008170809390110E94AF13089580918F1100
:10298000882311F484E001C0815080938F11089551
:1029900080918F11843018F010928F1108958F5FFD
:1029A00080938F1108950E9427530E943C530895ED
:1029B000CF93DF93CAE7D1E1CE0160E270E044E15A
:1029C00050E00E9471A78DB79EB70E970FB6F8948E
:1029D0009EBF0FBE8DBFEDB7FEB73196ADB7BEB788
:1029E0001296DC93CE93119786E993E093838283CA
:1029F000809110129091111295838483809112120C
:102A000090E00196978386838091131280871186C8
:102A100080911412828713868091151284871586FF
:102A20000E940CA88DB79EB70E960FB6F8949EBF65
:102A30000FBE8DBF80E090E00E943906DF91CF91FC
:102A4000089580E192E10E94AC1B109216120E9440
:102A5000D8140895EF92FF92CF93DF9380E192E133
:102A60000E94AC1B109216120E94D814CAE7D1E142
:102A7000CE0160E270E044E150E00E9471A781E085
:102A800090E00E94390682E30E945E12BC01FC01C4
:102A900001900020E9F73197E81BF90B9E012E1BEE
:102AA0003F0B2C5E3F4FC901AF010E9468A782E037
:102AB00090E00E943906CE0160E270E044E150E00F
:102AC0000E9471A78BE10E945E12BC01FC01019083
:102AD0000020E9F73197E81BF90B9E012E5F3F4F6D
:102AE000C901AF010E9468A789E10E945E12BC0182
:102AF000FC0101900020E9F73197E81BF90BCE1B90
:102B0000DF0B6296CE01AF010E9468A783E090E0E0
:102B10000E943906DF91CF91FF90EF9008958AE7E8
:102B200091E160E270E044E150E00E9471A7809181
:102B30008F118230B9F0833018F4813029F40BC042
:102B40008330B9F08430E1F06091D0117091D111EF
:102B500021E030E01BC06091D2117091D31126E0CA
:102B600030E014C06091D4117091D51129E030E0AB
:102B70000DC06091D6117091D7112EE030E006C0E3
:102B80006091D8117091D91120E130E0FB010190E2
:102B90000020E9F73197E61BF70B26583E4EC90196
:102BA000AF010E9468A781E090E00E943906089575
:102BB0000E94D8140E948F15089580E192E10E942E
:102BC0000E190895EF92FF92CF93DF9380E192E187
:102BD0000E94AC1B1092161284E080938F110E9409
:102BE000D8140E948F15CAE7D1E1CE0160E270E0EF
:102BF00044E150E00E9471A78AE20E945E12BC018B
:102C0000FC0101900020E9F73197E81BF90BCE0198
:102C1000AF010E9468A782E30E945E12BC01FC0122
:102C200001900020E9F73197E81BF90B9E012E1B5C
:102C30003F0B2C5E3F4FC901AF010E9468A782E0A5
:102C400090E00E943906CE0160E270E044E150E07D
:102C50000E9471A78BE20E945E12BC01FC010190F0
:102C60000020E9F73197E81BF90B9E012E5F3F4FDB
:102C7000C901AF010E9468A788E10E945E12BC01F1
:102C8000FC0101900020E9F73197E81BF90BCE1BFE
:102C9000DF0B6296CE01AF010E9468A783E090E04F
:102CA0000E9439060E941A1285E20E945E129093D9
:102CB000D1118093D01186E20E945E129093D311BD
:102CC0008093D21187E20E945E129093D511809377
:102CD000D41188E20E945E129093D7118093D6118E
:102CE00089E20E945E129093D9118093D811DF91EE
:102CF000CF91FF90EF9008950E941A1285E20E94F2
:102D00005E129093D1118093D01186E20E945E12E0
:102D10009093D3118093D21187E20E945E12909318
:102D2000D5118093D41188E20E945E129093D7113E
:102D30008093D61189E20E945E129093D9118093FC
:102D4000D81180E192E10E940E198EE00E94E30505
:102D5000089580918F118230E1F0833018F4813032
:102D600029F412C0833031F1843071F18091101256
:102D70009091111227E08A3D920788F10197909374
:102D8000111280931012089580E192E10E944D1873
:102D9000089580911312823048F480E192E10E94FC
:102DA0004D1880E192E10E94C61701C081508093C6
:102DB0001312089580911412882311F487E101C041
:102DC000815080931412089580911512882321F464
:102DD0008BE3809315120895815080931512089506
:102DE00080E192E10E94D81780E192E10E94C6172B
:102DF00090911312891718F4981B90931312089549
:102E00001F9380918F118230D1F0833018F481307C
:102E100029F412C0833029F1843071F180911012AD
:102E20009091111227E08F3E920780F501969093C2
:102E30001112809310122AC00E94F01627C0109120
:102E4000131280E192E10E94C617181720F00E9429
:102E5000F01681E003C0809113128F5F80931312EC
:102E600015C080911412873118F0109214120EC000
:102E70008F5F809314120AC0809115128B3318F063
:102E80001092151203C08F5F809315121F91089541
:102E90001F920F920FB60F9211248F939F93AF93AF
:102EA000BF938091FB0D9091FC0DA091FD0DB09111
:102EB000FE0D0196A11DB11D8093FB0D9093FC0D9D
:102EC000A093FD0DB093FE0D88ED8093850083EFF8
:102ED00080938400BF91AF919F918F910F900FBE0F
:102EE0000F901F901895DC01CB012EE0B695A795A9
:102EF000979587952A95D1F78F719070A070B070D3
:102F000088319105A105B10520F087E190E0A0E0AE
:102F1000B0E00895BB27A92F982F872F8F7390704B
:102F2000A070B0708C339105A105B10520F08BE342
:102F300090E0A0E0B0E008951092800082E08093DD
:102F4000810088ED8093850083EF80938400109248
:102F500087001092860010928900109288001092CB
:102F60008B0010928A0010928D0010928C0081E0EC
:102F700080936F00089510926F00089520E0837091
:102F80009070009709F421E0822F0895FC0192814E
:102F900020813181E92FF0E0ED51FC4F80819130AB
:102FA00031F4237030702115310509F48DE1089555
:102FB000FC0182818B3058F08081918127E08F3E27
:102FC000920718F4019691838083128208958F5F8F
:102FD00082830895FC01828120813181A82FB0E095
:102FE000AD51BC4F9C91813031F42370307021156C
:102FF000310509F49DE18381860F8383981728F4B6
:10300000891B8383CF010E94D817089567E070E081
:103010000E94EA17089561E070E00E94EA1708959F
:103020000F931F93CF93DF93EC019B018C81280FAB
:10303000311DC90168E170E00E9442A6062F172FDA
:1030400088E1869F802D1124281B2C8305C0CE018A
:103050000E940B180150104001151105C1F7DF91B6
:10306000CF911F910F910895FC019B018581280F3D
:10307000311D2C33310578F0C9016CE370E00E94FA
:1030800042A68CE3689F802D1124281B2583CF0145
:103090000E941018089525830895FC0182818823D9
:1030A00059F48081918127E08A3D920718F00197B9
:1030B000918380838BE001C0815082830895EF92D9
:1030C000FF920F931F93FC016081718189ED97E05E
:1030D00020E030E0A9010FC0DC01A370B0701097B0
:1030E00029F422593E4F4F4F5F4F04C023593E4FA2
:1030F0004F4F5F4F01968617970770F3E280A3EE5C
:10310000B3E080E0637070700DC09C91813021F459
:103110006115710509F49DE1290F311D411D511DF6
:103120008F5F11968E1589F77381858190E0A0E0FD
:10313000B0E0BA2FA92F982F8827E480FF2400E061
:1031400010E06EE0EE0CFF1C001F111F6A95D1F716
:103150008E299F29A02BB12B6681660F660FE62E64
:10316000FF2400E010E08E299F29A02BB12B270F10
:10317000311D411D511D203060E2360760E04607D9
:1031800060E0560720F02FEF3FE140E050E063E1C0
:10319000220F331F441F551F6A95D1F7282B392B57
:1031A0004A2B5B2BB901CA011F910F91FF90EF9041
:1031B0000895CF92DF92EF92FF920F931F938AE0D0
:1031C00090E040E050E0BA010EEF1FEF2FEF3FEF2D
:1031D000CC24DD2476010E9462281F910F91FF907C
:1031E000EF90DF90CF900895DF93CF9300D000D081
:1031F000CDB7DEB769837A838B839C8380E094E0CC
:10320000BE016F5F7F4F42E050E00E94E4670F9085
:103210000F900F900F90CF91DF910895EF92FF9252
:103220000F931F930E945F187B018C010E94F4187A
:10323000C801B7014AE050E00E9424288091FB0DAC
:103240009091FC0DA091FD0DB091FE0D8093FF0DAE
:103250009093000EA093010EB093020E1F910F9158
:10326000FF90EF900895EF92FF920F931F93DF93DB
:10327000CF93CDB7DEB728970FB6F894DEBF0FBE59
:10328000CDBF05E0E02EF12CEC0EFD1E8E010F5F90
:103290001F4F80E094E0B70142E050E00E9482645A
:1032A00080E094E0B80142E050E00E94826429810D
:1032B0003A814B815C818D819E81AF81B8852817D1
:1032C00039074A075B0728F3B901CA0128960FB6E8
:1032D000F894DEBF0FBECDBFCF91DF911F910F914C
:1032E000FF90EF9008952F923F924F925F926F92CE
:1032F0007F928F929F92AF92BF92CF92DF92EF9286
:10330000FF920F931F93DF93CF93CDB7DEB728972C
:103310000FB6F894DEBF0FBECDBF182F0E94331931
:103320002B013C01113009F426C10E94D9189B01E0
:10333000AC015B016C01F3E1D694C794B794A794F8
:10334000FA95D1F7D301C201E3E1B695A795979518
:103350008795EA95D1F789549F4FAF4FBF4F8A1594
:103360009B05AC05BD0508F001C1112319F401E06E
:1033700010E019C1E090FB0DF090FC0D0091FD0DE7
:103380001091FE0D8091FF0D9091000EA091010E05
:10339000B091020EE81AF90A0A0B1B0BDA01C901F7
:1033A0007EE0B695A795979587957A95D1F78F7119
:1033B0009070A070B07088319105A105B10520F022
:1033C00087E190E0A0E0B0E0282E3324BB27A52FB2
:1033D000942F832F8F739070A070B0708C339105F1
:1033E000A105B10520F08BE390E0A0E0B0E0482E0D
:1033F0005524307040705070203F31054105510513
:1034000020F02FEE30E040E050E0622F70E078874F
:103410006F83C801B70120E036ED43E850E00E9419
:1034200056A629833A834B835C8369817A818B8199
:103430009C8120E036ED43E850E00E9417A6E61A92
:10344000F70A080B190BC801B70120E43EE745E075
:1034500050E00E9456A63E832D833901882499248A
:10346000C401B30120E43EE745E050E00E9417A606
:10347000E61AF70A080B190BC401B30120E737E17C
:1034800040E050E00E9417A6A8019701261B370BC9
:10349000480B590BCA01B90129E130E040E050E086
:1034A0000E9456A66F817885620F731F78876F839D
:1034B000603F710538F0605F704078876F830894D3
:1034C000411C511CC801B70120E737E140E050E042
:1034D0000E9456A6240D351D2C33310528F02C539F
:1034E00030400894211C311C8D819E81820D931DDA
:1034F0008831910530F048970894A11CB11CC11C7B
:10350000D11C422E552466247724762C652C542C0D
:1035100044247F81272F30E040E050E0422A532AA4
:10352000642A752A29813A814B815C81A20EB31EDF
:10353000C41ED51E33E1AA0CBB1CCC1CDD1C3A9565
:10354000D1F74A285B286C287D2890E0A0E0B0E005
:103550002EE0880F991FAA1FBB1F2A95D1F7482A72
:10356000592A6A2A7B2A01E010E007C0112319F4C6
:1035700000E010E018C000E010E0C301B2014AE032
:1035800050E00E9424288091FB0D9091FC0DA091A9
:10359000FD0DB091FE0D8093FF0D9093000EA09352
:1035A000010EB093020EC80128960FB6F894DEBF44
:1035B0000FBECDBFCF91DF911F910F91FF90EF9084
:1035C000DF90CF90BF90AF909F908F907F906F9043
:1035D0005F904F903F902F900895823018F482E0D2
:1035E0000E94731908956F927F928F929F92AF926B
:1035F000BF92CF92DF92EF92FF920F931F93CF93E0
:10360000DF937B018C01EA015B016C0133E1D6940D
:10361000C794B794A7943A95D1F787E0DA011D9241
:103620008A95E9F789ED97E09C01237030702115A8
:10363000310529F42EE631E040E050E004C02DE6EB
:1036400031E040E050E0BC016F5F7F4FA216B3064F
:10365000C406D50630F0A21AB30AC40AD50ACB01B3
:10366000E3CF998388831A829A8128813981E92F4F
:10367000F0E0ED51FC4F8081913031F423703070D7
:103680002115310509F48DE1682E772488249924C9
:103690006A147B048C049D0440F4CE010E94D81768
:1036A000A618B708C808D908DFCF9A2DAB828A15AB
:1036B00028F4981B9B83CE010E94D817D801C7011C
:1036C0002EE0B695A795979587952A95D1F78F7196
:1036D0009070A070B07088319105A105B10520F0FF
:1036E00087E190E0A0E0B0E08C83BB27A12F902F72
:1036F0008F2D8F739070A070B0708C339105A105E1
:10370000B10520F08BE390E0A0E0B0E08D838FEF77
:1037100090E0A0E0B0E0E822F9220A231B2390EF1A
:10372000E916F1040105110528F0AFEEEA2EF12C9F
:10373000012D112DE694E694EE82DF91CF911F9139
:103740000F91FF90EF90DF90CF90BF90AF909F9040
:103750008F907F906F900895CF93DF93EC010E943C
:103760003319AE010E94F31ADF91CF910895809131
:10377000FB0D9091FC0DA091FD0DB091FE0D2091DF
:103780008F11309190114091911150919211821BA3
:10379000930BA40BB50B20919311223048F4893E72
:1037A00023E0920720E0A20720E0B20748F4089542
:1037B0008D3221E0920720E0A20720E0B20710F04E
:1037C0000E94BC05089584E094E00E94A264BC01BC
:1037D000707F84E094E00E9404680E94BC05089514
:1037E000EF92FF920F931F93CF93DF9384E094E0C7
:1037F0000E94A264BC01707F84E094E00E9404688F
:103800008091FB0D9091FC0DA091FD0DB091FE0DEE
:1038100080938F1190939011A0939111B093921176
:1038200010929311CAE7D1E1CE0160E270E044E169
:1038300050E00E9471A784E00E945E12BC01FC016E
:1038400001900020E9F73197E81BF90B8E010C5F1E
:103850001F4FC801AF010E9468A780E090E00E945E
:103860003906CE0160E270E044E150E00E9471A7A9
:1038700085E00E945E12BC01FC0101900020E9F786
:103880003197E81BF90BC801AF010E9468A781E0DE
:1038900090E00E943906CE0160E270E044E150E021
:1038A0000E9471A785E40E945E12BC01FC01019098
:1038B0000020E9F73197E81BF90BCE01AF010E9418
:1038C00068A782E090E00E943906CE0160E270E0D5
:1038D00044E150E00E9471A783E090E00E94390625
:1038E00086EB96E060E00E945F4680E060E00E9428
:1038F0003C46DF91CF911F910F91FF90EF9008957B
:103900001F93182F1295107F8EEC98E060E0712FB6
:1039100040E050EF0E942F688EED98E060E0712F3C
:1039200040E050EF0E942F681F91089580E00E94B0
:10393000801C85E094E00E94A264BC01607F85E069
:1039400094E00E9404680895EF92FF92CF93DF9372
:1039500084E094E00E94A264BC01707F7A6084E0FD
:1039600094E00E940468809193118F5F809393117B
:10397000813009F066C08091FB0D9091FC0DA09103
:10398000FD0DB091FE0D80938F1190939011A09337
:103990009111B09392110E94961C80E00E940661E2
:1039A0008AE791E160E270E044E150E00E9471A793
:1039B00086E00E945E12BC01FC0101900020E9F744
:1039C0003197E81BF90BCEE7D1E1CE01AF010E94A0
:1039D00068A780E090E00E943906CE01049760E27B
:1039E00070E044E150E00E9471A787E00E945E12FF
:1039F000BC01FC0101900020E9F73197E81BF90BAD
:103A0000CE01AF010E9468A781E090E00E943906D4
:103A1000CE01049760E270E044E150E00E9471A79B
:103A200082E090E00E94390683E090E00E9439062F
:103A300086EB96E060E00E945F4680E060E00E94D6
:103A40003C46DF91CF91FF90EF9008950E94961C25
:103A500084E00E9406610E94BC05089585E094E020
:103A60000E94A264BC01607F656085E094E00E94D2
:103A7000046882E00E94801C0E94BC050895EF92B9
:103A8000FF92CF93DF938AE791E160E270E044E137
:103A900050E00E9471A783E00E945E12BC01FC010D
:103AA00001900020E9F73197E81BF90BCEE7D1E14F
:103AB000CE01AF010E9468A780E090E00E94390625
:103AC00081E160E00E949F048091171290E00196CE
:103AD0006FEE73E042E00E944E06CE01049760E272
:103AE00070E044E150E00E9471A78DE10E945E12F7
:103AF000BC01FC0101900020E9F73197E81BF90BAC
:103B0000CE01AF010E9468A785E094E00E94A26404
:103B10008F7090708530910511F481E801C082E8C2
:103B20000E945E12BC01FC0101900020E9F7319770
:103B3000E81BF90BC4E8D1E1CE01AF010E9468A7F0
:103B400081E090E00E9439062A97CE0160E270E0A1
:103B500044E150E00E9471A785E40E945E12BC011E
:103B6000FC0101900020E9F73197E81BF90BCE0129
:103B7000AF010E9468A787E40E945E12BC01FC01AD
:103B800001900020E9F73197E81BF90B2EE831E1AD
:103B90002E1B3F0BC901AF010E9468A782E090E095
:103BA0000E943906CE0160E270E044E150E00E94DC
:103BB00071A788E40E945E12BC01FC010190002004
:103BC000E9F73197E81BF90B2BE831E12E1B3F0B8E
:103BD000C901AF010E9468A783E090E00E94390606
:103BE00086EB96E060E00E945F4680E060E00E9425
:103BF0003C46DF91CF91FF90EF9008958AE10E94BB
:103C0000D905089589E10E94D9050895EF92FF92A0
:103C10000F931F93DF93CF93CDB7DEB728970FB6DF
:103C2000F894DEBF0FBECDBF8091FB0D9091FC0DCF
:103C3000A091FD0DB091FE0D80938F119093901186
:103C4000A0939111B0939211109293110AE711E190
:103C5000C80160E270E044E150E00E9471A782E098
:103C60000E945E12BC01FC0101900020E9F731972F
:103C7000E81BF90B98012B5F3F4FC901AF010E9470
:103C800068A780E090E00E943906C80160E270E019
:103C900044E150E00E9471A78DB79EB70A970FB616
:103CA000F8949EBF0FBE8DBFEDB7FEB731967E0173
:103CB0000894E11CF11CADB7BEB71296FC92EE92CF
:103CC000119788E090E09383828384EF93E095835B
:103CD000848382E090E0978386838DE190E09187F2
:103CE00080870E94CEA7F70101900020E9F7319765
:103CF000EE19FF099801285F3F4F8DB79EB70A96CE
:103D00000FB6F8949EBF0FBE8DBFC901B701AF01BA
:103D10000E9468A781E090E00E943906C80160E235
:103D200070E044E150E00E9471A785E40E945E12B9
:103D3000BC01FC0101900020E9F73197E81BF90B69
:103D4000C801AF010E9468A786E40E945E12BC0110
:103D5000FC0101900020E9F73197E81BF90B98016D
:103D60002E1B3F0B2C5E3F4FC901AF010E9468A77D
:103D700082E090E00E943906C80160E270E044E110
:103D800050E00E9471A78FE10E945E12BC01FC010D
:103D900001900020E9F73197E81BF90B0E1B1F0B70
:103DA0000E5E1F4FC801AF010E9468A783E090E03C
:103DB0000E94390686EB96E060E00E945F4680E054
:103DC00060E00E943C4628960FB6F894DEBF0FBE16
:103DD000CDBFCF91DF911F910F91FF90EF9008958C
:103DE000E0919811F0E0EF5FFA4E80818F3F11F47F
:103DF00081E309C0893311F481E405C0863411F4EC
:103E000080E301C08F5F808308952091981130E096
:103E1000F901EF5FFA4E80818F3F11F0803329F472
:103E20002F5F3A4E86E4F90105C0813411F489E32D
:103E300001C081508083089580919811882311F0EA
:103E4000815001C083E0809398110895809198116A
:103E5000833020F48F5F8093981108951092981109
:103E600008958FEF809301158093021580930315B9
:103E700080930415089580E09091A611992309F488
:103E800081E08093A611089580E09091A711992375
:103E900009F481E08093A7110895AF92BF92CF9269
:103EA000DF92EF92FF920F931F93CF93DF93809156
:103EB000A711C82FD0E0CC0FDD1FCC0FDD1FC157DD
:103EC000DE4E6D817E818F81988520E030E040E874
:103ED0005FE30E944DA36D837E838F8398878091DB
:103EE000A711C82FD0E0CC0FDD1FCC0FDD1FC157AD
:103EF000DE4EAD80BE80CF80D884E090A011F090DF
:103F0000A1110091A2111091A311C601B501A80140
:103F100097010E9400A51816B4F4C801B7012091BA
:103F20009C1130919D1140919E1150919F110E94C2
:103F30004CA39B01AC01C601B5010E944CA36D834B
:103F40007E838F83988781E08093A9118091AA1145
:103F5000863099F085E08093AA118091FB0D9091B5
:103F6000FC0DA091FD0DB091FE0D8093AB119093CF
:103F7000AC11A093AD11B093AE11DF91CF911F9111
:103F80000F91FF90EF90DF90CF90BF90AF9008958A
:103F9000AF92BF92CF92DF92EF92FF920F931F9357
:103FA000CF93DF938091A711C82FD0E0CC0FDD1FF6
:103FB000CC0FDD1FC157DE4E6D817E818F819885CC
:103FC00020E030E040E85FE30E944CA36D837E83F5
:103FD0008F8398878091A711C82FD0E0CC0FDD1F69
:103FE000CC0FDD1FC157DE4EAD80BE80CF80D884A0
:103FF000E0909C11F0909D1100919E1110919F11E5
:10400000C601B501A80197010E94B1A38823B4F4A9
:104010006091A0117091A1118091A2119091A311B2
:10402000A80197010E944CA39B01AC01C601B501F8
:104030000E944DA36D837E838F83988781E0809358
:10404000A9118091AA11883099F087E08093AA1174
:104050008091FB0D9091FC0DA091FD0DB091FE0D96
:104060008093AB119093AC11A093AD11B093AE11AE
:10407000DF91CF911F910F91FF90EF90DF90CF9044
:10408000BF90AF900895AF92BF92CF92DF92EF9220
:10409000FF920F931F93CF93DF938091A711C82FA7
:1040A000D0E0CC0FDD1FCC0FDD1FC157DE4E6D8180
:1040B0007E818F8198852DEC3CEC4CEC5DE30E9479
:1040C0004CA36D837E838F8398878091A711C82F1F
:1040D000D0E0CC0FDD1FCC0FDD1FC157DE4EAD8011
:1040E000BE80CF80D884E0909C11F0909D1100910B
:1040F0009E1110919F11C601B501A80197010E9460
:10410000B1A38823B4F46091A0117091A1118091A2
:10411000A2119091A311A80197010E944CA39B01A9
:10412000AC01C601B5010E944DA36D837E838F83D0
:10413000988781E08093A9118091AA118C3099F021
:104140008BE08093AA118091FB0D9091FC0DA091C2
:10415000FD0DB091FE0D8093AB119093AC11A09327
:10416000AD11B093AE11DF91CF911F910F91FF90E0
:10417000EF90DF90CF90BF90AF900895AF92BF9235
:10418000CF92DF92EF92FF920F931F93CF93DF9323
:104190008091A711C82FD0E0CC0FDD1FCC0FDD1F01
:1041A000C157DE4E6D817E818F8198852DEC3CEC70
:1041B0004CEC5DE30E944DA36D837E838F839887D3
:1041C0008091A711C82FD0E0CC0FDD1FCC0FDD1FD1
:1041D000C157DE4EAD80BE80CF80D884E090A01164
:1041E000F090A1110091A2111091A311C601B50187
:1041F000A80197010E9400A58823B4F0C801B70167
:1042000020919C1130919D1140919E1150919F11D0
:104210000E944CA39B01AC01C601B5010E944CA3B6
:104220006D837E838F83988781E08093A91180912D
:10423000AA118A3099F089E08093AA118091FB0D30
:104240009091FC0DA091FD0DB091FE0D8093AB11EE
:104250009093AC11A093AD11B093AE11DF91CF91BB
:104260001F910F91FF90EF90DF90CF90BF90AF9094
:104270000895E091A711F0E0EE0FFF1FE157FE4E09
:104280008581968120919A1130919B118217930715
:1042900014F4019604C0809198119091991196831D
:1042A000858381E08093A9119091AA11923091F0B9
:1042B0008093AA118091FB0D9091FC0DA091FD0DB2
:1042C000B091FE0D8093AB119093AC11A093AD1102
:1042D000B093AE110895E091A711F0E0EE0FFF1F2B
:1042E000E157FE4E85819681209198113091991168
:1042F0002817390714F4019704C080919A119091FE
:104300009B119683858381E08093A9118091AA11E6
:10431000843099F083E08093AA118091FB0D9091F5
:10432000FC0DA091FD0DB091FE0D8093AB1190930B
:10433000AC11A093AD11B093AE11089584E991E151
:1043400061E075E144E050E00E945BA70097C1F195
:1043500020E030E080910415863411F421E030E053
:1043600080E090E040910315463411F481E090E044
:104370002823392390E080910215863409F491E0D6
:1043800080E040910115463409F481E0892390E0F2
:1043900082239323009761F48FEF8093011580931C
:1043A00002158093031580930415109298110895B7
:1043B00081E095E160E070E044E050E00E941A285E
:1043C0000E94BC050895809101158F3F61F4809192
:1043D00002158F3F41F4809103158F3F21F48091A6
:1043E00004158F3F89F081E095E160E070E044E0E2
:1043F00050E00E941A288FEF8093011580930215D8
:10440000809303158093041582E00E94E3050895CC
:104410008AE00E94E305089584E00E94E305089580
:104420008AE791E160E270E044E150E00E9471A708
:104430008BE580937A11809101158F3F09F480E21A
:1044400080937B11809102158F3F09F480E2809365
:104450007C11809103158F3F09F480E280937D11D8
:10446000809104158F3F09F480E280937E118DE5E1
:1044700080937F1181E090E00E943906809198112D
:104480008F5F61E00E949F048EE00E9435040895D2
:104490008DE50E945E129093B0118093AF118CE570
:1044A0000E945E129093B2118093B1110895EF9221
:1044B000FF920F931F93CF93DF938FEF809301159C
:1044C0008093021580930315809304151092981120
:1044D000CAE7D1E1CE0160E270E044E150E00E9421
:1044E00071A788E00E945E12BC01FC0101900020CF
:1044F000E9F73197E81BF90B04E110E098012E1B56
:104500003F0B369527952C0F3D1FC901AF010E9427
:1045100068A780E090E00E9439060E941022CE0138
:1045200060E270E044E150E00E9471A78AE20E94DC
:104530005E12BC01FC0101900020E9F73197E81BF5
:10454000F90BCE01AF010E9468A78DE40E945E12B4
:10455000BC01FC0101900020E9F73197E81BF90B41
:104560000E1B1F0B0C0F1D1FC801AF010E9468A777
:1045700082E090E00E943906CE0160E270E044E102
:1045800050E00E9471A78BE20E945E12BC01FC0108
:1045900001900020E9F73197E81BF90B9E012E5F8F
:1045A0003F4FC901AF010E9468A78CE40E945E12D0
:1045B000BC01FC0101900020E9F73197E81BF90BE1
:1045C000CE1BDF0B6296CE01AF010E9468A783E08D
:1045D00090E00E943906DF91CF911F910F91FF90DB
:1045E000EF900895CF93DF93CAE7D1E1CE0160E267
:1045F00070E044E150E00E9471A781E00E945E12E9
:10460000BC01FC0101900020E9F73197E81BF90B90
:1046100024E130E02E1B3F0B369527952C0F3D1FD4
:10462000C901AF010E9468A780E090E00E943906AE
:10463000CE0160E270E044E150E00E9471A781E0A9
:1046400090E00E943906DF91CF91089580E061E00B
:1046500041E00E94ED6008958BE00E94D905089525
:1046600080919911882319F084E10E94D905089559
:1046700082E10E94D90508958FE00E94D90508952E
:104680000F931F93DF93CF93CDB7DEB728970FB665
:10469000F894DEBF0FBECDBF8DB79EB708970FB69B
:1046A000F8949EBF0FBE8DBFEDB7FEB731968E0159
:1046B0000F5F1F4FADB7BEB712961C930E931197A5
:1046C00088E090E0938382838091D0119091D11102
:1046D0009583848380911A1290E001969783868354
:1046E0000E94CEA7F80101900020E9F78DB79EB790
:1046F00008960FB6F8949EBF0FBE8DBFC8018E1BE3
:104700009F0B45969695879561E00E949F04C8018E
:104710000E944B0628960FB6F894DEBF0FBECDBFA1
:10472000CF91DF911F910F9108950E9440238FE850
:1047300091E10E9494460895EF92FF92CF93DF9308
:104740000E94F222CAE7D1E1CE0160E270E044E1CA
:1047500050E00E9471A78AE50E945E12BC01FC0134
:1047600001900020E9F73197E81BF90BCE01AF016A
:104770000E9468A781E10E945E12BC01FC010190C9
:104780000020E9F73197E81BF90B24E130E02E1BFC
:104790003F0B369527952C0F3D1FC901AF010E9495
:1047A00068A782E090E00E943906CE0160E270E0E6
:1047B00044E150E00E9471A78BE10E945E12BC01AF
:1047C000FC0101900020E9F73197E81BF90B9E01ED
:1047D0002E5F3F4FC901AF010E9468A78BE50E9481
:1047E0005E12BC01FC0101900020E9F73197E81B43
:1047F000F90BCE1BDF0B6296CE01AF010E9468A7BA
:1048000083E090E00E9439068FE891E10E94D6464D
:104810000E941A128BE00E945E129093D111809335
:10482000D0110E949523DF91CF91FF90EF900895D2
:104830001F930E94402380911A126EE00E949A6694
:10484000192F80911A126CE00E949A6692959170CD
:1048500012951170910F909399118AE791E160E29E
:1048600070E044E150E00E9471A76091D211709114
:10487000D311DB01FD0101900020E9F73197EA1B1C
:10488000FB0B2CE731E1C901AF010E9468A78091C1
:1048900099118823A1F06091D4117091D511DB0199
:1048A000FD0101900020E9F73197EA1BFB0B2CE892
:1048B00031E12E1B3F0BC901AF010E9468A783E0C5
:1048C00090E00E9439068FE891E10E9494461F9182
:1048D0000895EF92FF92CF93DF9384E991E160E036
:1048E00070E044E050E00E945828809194118F3F7E
:1048F000B9F4809195118F3F99F4809196118F3F73
:1049000079F4809197118F3F59F481E391E3DC01B1
:104910008093941190939511A0939611B093971151
:1049200084E991E161E075E144E050E00E945BA719
:10493000009779F00E946D05823021F48BE00E948F
:10494000D9056EC083E00E947B058BE00E94E305E1
:1049500067C00E94F222CAE7D1E1CE0160E270E0B6
:1049600044E150E00E9471A78AE40E945E12BC01FB
:10497000FC0101900020E9F73197E81BF90B7E015B
:10498000CE01AF010E9468A781E10E945E12BC01C6
:10499000FC0101900020E9F73197E81BF90BC4E115
:1049A000D0E09E012E1B3F0B369527952E0D3F1D07
:1049B000C901AF010E9468A786E10E945E12BC0196
:1049C000FC0101900020E9F73197E81BF90BCE1BA1
:1049D000DF0BCE0DDF1DCE01AF010E9468A782E084
:1049E00090E00E9439068FE891E10E94D6460E942D
:1049F0001A128BE00E945E129093D1118093D01115
:104A00008BE40E945E129093D3118093D2118FE4B5
:104A10000E945E129093D5118093D4110E941824A5
:104A2000DF91CF91FF90EF900895EF92FF920F9357
:104A30001F93CF93DF938091AA11882309F4B5C007
:104A40000E944409882309F4B0C08091AA118730DC
:104A500040F48530A8F4813008F4A7C0833068F0B2
:104A600009C08B3018F48930A8F40FC08D3008F0DD
:104A70009CC015C0CBE6D1E20AC0C9E3D1E202C0B6
:104A8000CDE4DFE180E091E00EC0C8ECDFE180E83A
:104A900090E009C0CEEBD0E280E290E004C0C3E435
:104AA000D0E280E490E00E944F09882309F47FC09F
:104AB0008091AA11863009F450C0873088F4833081
:104AC00009F1843030F48130E9F0823009F06DC0B2
:104AD00044C0843009F441C0853009F066C012C07A
:104AE000893081F08A3030F4873061F0883009F005
:104AF0005CC033C08B3031F08B3078F18C3009F0F2
:104B000054C02BC08091FB0D9091FC0DA091FD0D28
:104B1000B091FE0D2091AB113091AC114091AD11CF
:104B20005091AE117C018D01E21AF30A040B150BB2
:104B3000A80197012536310541055105C0F1809343
:104B4000AB119093AC11A093AD11B093AE118091C5
:104B5000AA118F5F8093AA112AC08091FB0D9091BA
:104B6000FC0DA091FD0DB091FE0D2091AB11309187
:104B7000AC114091AD115091AE117C018D01E21A42
:104B8000F30A040B150BA80197012B3031054105E1
:104B9000510568F08093AB119093AC11A093AD11C7
:104BA000B093AE11FE01099502C01092AA11DF91D7
:104BB000CF911F910F91FF90EF9008958091171260
:104BC000882311F48091070E815080931712089565
:104BD00080911A12882311F48BE001C081508093D8
:104BE0001A120895809117128F5F9091070E8917FE
:104BF00018F010921712089580931712089580915B
:104C00001A128F5F8C3018F010921A120895809348
:104C10001A12089510921712089581E080931712C6
:104C2000089582E080931712089583E0809317120D
:104C3000089590911F12992359F080911E12882394
:104C400021F4915090931E120895815080931E126A
:104C5000089580911D12882311F481E001C08150D4
:104C600080931D12089580911E128F5F90911F12E4
:104C7000891718F010921E12089580931E1208953D
:104C800080911D128F5F823018F010921D120895CE
:104C900080931D12089510921E12089580911F1284
:104CA000882319F081E080931E12089580911912D3
:104CB000882311F483E001C0815080931912089574
:104CC000809119128F5F843018F010921912089594
:104CD00080931912089580911812882311F485E0A9
:104CE00001C08150809318120895809118128F5F2F
:104CF000863018F0109218120895809318120895B3
:104D000010921B128091080E8823F1F485E090E048
:104D100060E04CE02CE00E94F9278093201291E0A3
:104D200090931F12843008F484E08093070E90E083
:104D300001972091171230E0281739070CF4C901A8
:104D40008093171210921E120E94F08C0E94F85A43
:104D500008951F93182F8230E8F48091171264E0B1
:104D600070E00E94EC2780911E1266E070E00E94C5
:104D7000EC278091080E882389F08091201265E04D
:104D800070E00E94EC2780911F1267E070E00E94A3
:104D9000EC2704C0843011F40E948026812F0E94E9
:104DA000CD58812F0E940F841F91089585E094E0D3
:104DB0000E94A2648F7090708530910509F0E8C060
:104DC00080911B128130D9F0813010F08430B0F125
:104DD0008091FB0D9091FC0DA091FD0DB091FE0D09
:104DE0008093030E9093040EA093050EB093060ECD
:104DF00081E080931B1282E00E94066108950E9468
:104E0000285C8091FB0D9091FC0DA091FD0DB0915F
:104E1000FE0D2091030E3091040E4091050E50912D
:104E2000060E821B930BA40BB50B86399105A105C9
:104E3000B10508F4AFC082E080931B1280E798E0D0
:104E40000E94A2649F708F339105E9F1803491052F
:104E5000A0F48730910589F18830910538F48130CC
:104E6000910549F183309105E1F523C08F3091051B
:104E700031F18F319105A9F524C021E08F3F9207D0
:104E800041F122E08030920738F48F379105E9F044
:104E90008F3F910531F51BC027E08F3F9207E9F066
:104EA0002FE08F3F9207D9F023E08F3F9207C9F49C
:104EB00012C082E017C081E015C083E013C084E017
:104EC00011C085E00FC086E00DC087E00BC088E010
:104ED00009C089E007C08AE005C08BE003C08CE010
:104EE00001C080E08093201280E798E00E94A264D5
:104EF00081E080931F128093080E809120128430ED
:104F000008F484E08093070E90E001972091171237
:104F100030E0281739070CF4C9018093171210925A
:104F20001E1280911B12833030F58091FB0D909101
:104F3000FC0DA091FD0DB091FE0D2091030E30915E
:104F4000040E4091050E5091060E821B930BA40B8C
:104F5000B50B843F21E0920720E0A20720E0B207D2
:104F600050F083E080931B120E94AF470E94254BB4
:104F700083E00E9406610E94285C0E9444480E94CF
:104F80005C590E944F850E94494D0E94FE8C0895F5
:104F90000E948026089584E090E060E04BE020E0ED
:104FA0000E94F9278093171280931A1286E090E0EE
:104FB00060E041E020E00E94F92780931E12809378
:104FC0001D120E9480260E94AF470E94254B0E941E
:104FD00036590E944F8508951F93282FCB011FB784
:104FE000F894622F0E94BCA817FF01C078941F910B
:104FF00008951F93DF93CF9300D00F92CDB7DEB704
:105000001FB7F8942B834A8369830E94AAA82B8137
:105010004A81698117FF01C07894861718F04817F4
:1050200008F0282F822F0F900F900F90CF91DF91D3
:105030001F9108951F931FB7F8940E94B2A817FFFD
:1050400001C078941F910895DF93CF9300D000D0D2
:10505000CDB7DEB769837A838B839C83BA01CE0197
:10506000019644E050E00E941A280F900F900F9094
:105070000F90CF91DF910895DF93CF9300D0CDB7FC
:10508000DEB79A838983CE01019642E050E00E9408
:105090001A280F900F90CF91DF91089544E050E0CF
:1050A0000E941A28089544E050E00E941A280895AA
:1050B0001F931FB7F8940E949AA817FF01C0789415
:1050C0001F9108954F925F926F927F928F929F925D
:1050D000AF92BF92CF92DF92EF92FF920F931F9306
:1050E000DF93CF9300D000D0CDB7DEB7FC012A010B
:1050F0003B0148015901CE010196BF0144E050E057
:105100000E94582889819A81AB81BC8184159505BC
:10511000A605B70538F088169906AA06BB0610F052
:105120006C017D01B601C7010F900F900F900F9099
:10513000CF91DF911F910F91FF90EF90DF90CF9073
:10514000BF90AF909F908F907F906F905F904F90A7
:105150000895EF92FF920F931F93DF93CF9300D0A8
:1051600000D0CDB7DEB7FC017B018A01CE010196EC
:10517000BF0142E050E02B833C830E945828898184
:105180009A812B813C818E159F0520F00817190705
:1051900008F09C01C9010F900F900F900F90CF91D4
:1051A000DF911F910F91FF90EF9008950F931F9340
:1051B000DF93CF9300D000D0CDB7DEB7BC018E0116
:1051C0000F5F1F4FC80144E050E00E9458288981BA
:1051D0008F3F91F4F8013196D80111968C91119777
:1051E0008F3F51F4DF01119681818F3F29F4119691
:1051F0008C9111978F3F51F089819A81AB81BC814D
:105200002A2F220F2B2F221F2F3F19F480E090E02E
:10521000DC01682F792F8A2F9B2F0F900F900F9012
:105220000F90CF91DF911F910F9108952F923F9290
:105230004F925F926F927F928F929F92AF92BF92A6
:10524000CF92DF92EF92FF920F931F93DF93CF9352
:1052500000D000D0CDB7DEB7FC011A012B01380118
:105260004901560167017E010894E11CF11CC70148
:10527000BF0144E050E00E94582889818F3F91F49B
:10528000F7013196D70111968C9111978F3F51F408
:10529000DF01119681818F3F29F411968C9111972E
:1052A0008F3FE1F0E980FA800B811C81802F880F0D
:1052B000812F881F8F3F91F0C801B701A201910192
:1052C0000E94B1A387FD0AC0C801B701A4019301E0
:1052D0000E9400A5181614F0570168016A2D7B2D55
:1052E0008C2D9D2D0F900F900F900F90CF91DF91EF
:1052F0001F910F91FF90EF90DF90CF90BF90AF90F4
:105300009F908F907F906F905F904F903F902F90E5
:1053100008956F927F928F929F92AF92BF92CF9299
:10532000DF92EF92FF920F931F93DF93CF93CDB74E
:10533000DEB72A970FB6F894DEBF0FBECDBF8C0143
:105340005B01DC018C91843309F4CBC1853308F512
:105350008B3009F47EC08C3070F4843009F44BC07B
:10536000853018F48823D1F136C0853009F450C057
:10537000863089F550C0813309F42DC1823318F489
:10538000803349F5F8C0823309F440C1833319F5FD
:105390005EC1813409F4E6C2823460F4863309F4D4
:1053A000A0C1863308F400C2873309F4FDC18034FC
:1053B00091F4A1C2803609F457C0813630F48035AB
:1053C00009F4F2C2813539F4B2C4813609F478C0E7
:1053D000803D09F4E0C4EE24FF2424C5FB011082C3
:1053E0008FEF818380E081938F5F8733E1F717E34D
:1053F000E12EF12C17C5DB01F80187E001900D9239
:105400008150E1F785EAD50117968C93179707C568
:10541000FB01808304C5DB018C9382E011968C93A1
:1054200011978DE112968C93129780E213968C93CC
:10543000139781E114968C93149782E115968C93BF
:10544000159789E016968C93169717961C921797C6
:10545000E6C4F8016181D5018C9311966C9385E0C7
:1054600040E00E94ED60DBC485E094E00E94A2640D
:10547000BC01606285E094E00E940468F8016281EA
:1054800070E080E090E0CB0177276627238130E051
:1054900040E050E0542F432F322F2227622B732BF2
:1054A000842B952B248130E040E050E0622B732B5D
:1054B000842B952BA8014B5F5F4F21810E945E9F3B
:1054C00085E094E00E94A264BC01606285E094E003
:1054D0000E940468D80111962C911197E22EFF24A6
:1054E000E5E0F0E0EE0EFF1E12966C901297772426
:1054F0008824992443017724662413968C9190E0A4
:10550000A0E0B0E0BA2FA92F982F8827682A792A1F
:105510008A2A9B2AD80114968C9190E0A0E0B0E0F2
:10552000682A792A8A2A9B2AD501F80185E0019008
:105530000D928150E1F7A5014B5F5F4F2223B1F43B
:10554000C401B30148875A870E94B69E0E94709E8C
:10555000082FC401B30148855A8524E60E94DB9ECA
:10556000F50106830783008701875CC4C401B3018A
:105570000E94DB9E57C4D8011196DC9011971296B9
:105580009C91129780E01396EC90FF24E82AF92A68
:10559000B8016C5F7F4FC7014D2D0E943B4EF7FC59
:1055A0001AC0ED0CF11CB1E0EB16B0E6FB0698F06A
:1055B00081E08093C0148091FB0D9091FC0DA0912F
:1055C000FD0DB091FE0D8093191390931A13A093C3
:1055D0001B13B0931C13F8014181E42EFF2485E0D6
:1055E00090E0E80EF91E328120E0838190E0608037
:1055F000718082809380D5016D927D928D929D9273
:10560000BD01822B932B0E94C84D0CC4F80161810F
:10561000603190F06C3109F0FBC382818C31B9F4B8
:1056200083818330A1F4C801029661EF72E04EE1FC
:1056300050E00E941A280BC070E0660F771F660FBB
:10564000771F62567D4FC80102960E945328D801E9
:105650008C91F501808311968C911197818311961D
:105660008C9111978031E8F08C3109F0D1C38CE531
:1056700091E161EF72E04EE150E00E94582883EE24
:1056800092E161EF72E04EE150E00E945828D501AE
:105690001296E3EEF2E18CE101900D928150E1F778
:1056A000ADC390E0880F991F880F991FFC01E35745
:1056B000FB4FC080D180E280F38082569D4F40E056
:1056C00050E068E472EC00E010E028E432E40E946C
:1056D0001629D50112966D937D938D939C93159702
:1056E0009EC3F8016181862F829586958695837089
:1056F00090E0823091050CF08BC33081262F2695E7
:1057000026952695343329F5277030E0243031056D
:105710000CF07EC3677070E0633071050CF078C3E5
:10572000660F771F660F771FE6EAF0E08E9FA001F5
:105730008F9F500D9E9F500D1124640F751F6A5A44
:105740007E4F54E0220F331F5A95E1F7620F731F0B
:1057500027C0277030E0263031050CF059C3677040
:1057600070E0643071050CF053C3660F771F660F4D
:10577000771FE6EAF0E08E9FA0018F9F500D9E9F5D
:10578000500D1124640F751F6D567E4FC901B4E092
:10579000880F991FBA95E1F7820F931F680F791F41
:1057A000C80102960E945328D8018C91F50180838C
:1057B00011968C911197818311969C911197692F65
:1057C000629566956695637070E0623071050CF0C5
:1057D0001FC38C918453492F469546954695823038
:1057E00008F043C0477050E0443051050CF010C33E
:1057F0009770E92FF0E0E330F1050CF009C39F0149
:10580000220F331F220F331FA6EAB0E06A9FC001A8
:105810006B9F900D7A9F900D1124280F391F2A5AE3
:105820003E4FCA0154E0880F991F5A95E1F7EE0FD9
:10583000FF1FEE0FFF1FE353FB4FC080D180E280BC
:10584000F380820F931F40E050E068E472EC00E0C8
:1058500010E028E432E40E941629D50112966D93D7
:105860007D938D939C93159742C0477050E04630CE
:1058700051050CF0CDC29770E92FF0E0E430F1054E
:105880000CF0C6C2CF01880F991F880F991FA6EA96
:10589000B0E06A9F90016B9F300D7A9F300D11240C
:1058A000820F931F8D569E4F9A0114E0220F331FD3
:1058B0001A95E1F7240F351FEE0FFF1FEE0FFF1FA4
:1058C000E752FB4FC080D180E280F380820F931FAC
:1058D00040E050E068E472EC00E010E028E432E4DC
:1058E0000E941629F5016283738384839583A6E061
:1058F000EA2EF12C97C2D8011196DC901197D6941C
:1059000012969C91129780E01396EC90FF24E82A5F
:10591000F92AB8016C5F7F4FC7014D2D50E00E94FE
:10592000E467B2E0EB16B4E0FB06E0F4ED0CF11C2A
:10593000E1E0EE16E4E0FE06A8F081E08093C014FA
:105940002091FB0D3091FC0D4091FD0D5091FE0D0D
:105950002093191330931A1340931B1350931C1365
:1059600080935112D80111964C9111974695129639
:105970003C91129720E013968C91139790E0ED9054
:10598000FD900D911C91F501E082F1820283138359
:10599000542F550F5183B5016C5F7F4F822B932B92
:1059A00050E00E9482642AC285EA95EADB018D9369
:1059B0009C93F80180819181A281B381FB01808356
:1059C0009183A283B383D80111968C911197853A64
:1059D00009F494C0863A30F4882351F08E3109F0EE
:1059E0001EC231C08A3C69F08E3F09F018C21AC04D
:1059F000F801828193810E943909F4E0EF2EF12CA5
:105A000011C2D80112968C91129713966C910E9434
:105A10003C6F482F4E7FF801828163810E94056FA1
:105A20008FE46DC0D80112968C91129713966C91E9
:105A30000E943C6F482F4160F801828163810E947F
:105A4000056F83E45CC0D80112968C91129756EAD8
:105A5000859FC001112413966C9131E1639FB001C1
:105A60001124860F971F8E569E4F60E04BE022E078
:105A700039875A870E94F927982FF801828163811C
:105A800098870E943C6FE82ED80112966C9112976D
:105A900013968C91139739855A859885E1FE14C029
:105AA000659FB0011124839F90011124620F731F21
:105AB0006E567E4F892F8D700E94EC274E2D4D70B3
:105AC000F8018281638116C0659FB0011124839F14
:105AD00090011124620F731F6E567E4F892F8260D2
:105AE0000E94EC274E2D4260D80112968C9112979D
:105AF00013966C910E94056F84E501C08EE4F80155
:105B00009181D50111969C9311979FE516969C93D0
:105B1000169722812F5C17962C93179718969C93B3
:105B2000189723812F5C19962C9319971A969C939A
:105B30001A971B968C931B97EFE2EE2E1C96EC9215
:105B40007DE0C72ED12CCA0CDB1CCE0101960E9431
:105B5000AC1BEDB7FEB770970FB6F894FEBF0FBE43
:105B6000EDBF3196ADB7BEB71296DC92CE921197CB
:105B700089EE94E09383828389819A8195838483DB
:105B80008B8190E00196978386838C818087118634
:105B90008D81828713868E81848715868F81868783
:105BA00017860E940CA8F501E1A262E2C62ED12C54
:105BB000CA0CDB1C8DB79EB740960FB6F8949EBFFB
:105BC0000FBE8DBFC8010296D80112966C91129734
:105BD00013964C910E941778EDB7FEB73A970FB61F
:105BE000F894FEBF0FBEEDBF2DB73EB72F5F3F4FFE
:105BF000D282C18288E090E0D90113969C938E9363
:105C0000129788E095E015969C938E931497F8016F
:105C100082859385A485B585F90186839783A087BE
:105C2000B1870E94CEA7D5019996EC92C5018A96BC
:105C30002DB73EB72F5F3F4FEDB7FEB792838183FD
:105C400087E090E0D90113969C938E9312978EE093
:105C500095E015969C938E931497F8018281938119
:105C6000A481B581F90186839783A087B1870E94BB
:105C7000CEA7D501D096EC92EDB7FEB73A960FB607
:105C8000F894FEBF0FBEEDBFD80195968C91959705
:105C900095012E5C3F4F882321F081E3F50181AB14
:105CA00004C080E3D501D1968C93D9018FE28D9306
:105CB000F80184A1AD014F5F5F4F882331F081E38C
:105CC000D90111968C93119703C080E3F901818368
:105CD000FA018FE28193D80196968C9196977F0175
:105CE0000894E11CF11C8A3050F081E3DA0111962E
:105CF0008C93D80196968C9196978A5D09C080E323
:105D0000DA0111968C93D80196968C919697805DC6
:105D10008183F70131968FE2808356E0E52EF12CE6
:105D2000EE0EFF1EEA18FB08F501E5827BC0DB01E1
:105D30008C9311961C9211978091CF11882321F09A
:105D400042E0E42EF12C6EC0F80111811F70DB01DE
:105D500011961C931197EE24FF2400E015C010FF4C
:105D60000BC0602F70E06E5F7F4F6A0D7B1DC70117
:105D700044E10E940D060C5E0894E11CF11CB4E0A5
:105D8000EB16F10419F01695112349F7E02EFF24C4
:105D9000E2E0F0E03AC0D80112963C91129720E080
:105DA0001396EC901397FF24E22AF32A11960C9194
:105DB00011970695FB018083802F880F8183F282E3
:105DC000E38234E0C32ED12CC60ED71E15C0102F8F
:105DD000093008F018E0C701B601412F50E00E94D9
:105DE0008264011B812F90E0880F991FC80ED91E75
:105DF00080E190E0E80EF91E002349F7D5011196E5
:105E0000EC901197FF24E4E0F0E0EE0EFF1E0AC0D4
:105E100087E0D5018C9384E011968C93119788E0EC
:105E2000E82EF12CC7012A960FB6F894DEBF0FBEFC
:105E3000CDBFCF91DF911F910F91FF90EF90DF9039
:105E4000CF90BF90AF909F908F907F906F9008956C
:105E50000E94152580E060E00E949F04E091A71158
:105E6000F0E0EE0FFF1FE155FE4E808191810E9410
:105E70004B0683E061E00E949F04E091A811F0E0EE
:105E8000EE0FFF1FE053FE4E808191810E944B0672
:105E900008950E94282F8BE061E00E949F04E0910A
:105EA000A711F0E0EE0FFF1FE157FE4E85819681AE
:105EB00064E175E046E00E944E0681E161E00E94E7
:105EC0009F0481E40E94B2040895CF93DF9310925F
:105ED000AA11CAE7D1E1CE0160E270E044E150E0EE
:105EE0000E9471A78EE50E945E12BC01FC01019028
:105EF0000020E9F73197E81BF90B2AE030E02E1B70
:105F00003F0B36952795265F3F4F2C0F3D1FC9014C
:105F1000AF010E9468A780E090E00E943906CE01A0
:105F200060E270E044E150E00E9471A781E090E0FF
:105F30000E943906DF91CF9108950E94482289E599
:105F40000E945E129093D1118093D01183E30E943E
:105F50005E129093D3118093D21185E30E945E125A
:105F60009093D5118093D41184E30E945E12909394
:105F7000D7118093D61186E30E945E129093D911B7
:105F80008093D81189E80E945E129093DB11809370
:105F9000DA118AE80E945E129093DD118093DC1181
:105FA0008BE80E945E129093DF118093DE118DE8E2
:105FB0000E945E129093E1118093E0118CE80E94A0
:105FC0005E129093E3118093E2110895EF92FF9295
:105FD000CF93DF930E94652F8AE20E945E12BC017C
:105FE000FC0101900020E9F73197E81BF90BCAE7A3
:105FF000D1E1CE01AF010E9468A782E090E00E944B
:106000003906CE0160E270E044E150E00E9471A7E1
:106010008BE20E945E12BC01FC0101900020E9F7B6
:106020003197E81BF90B2296CE01AF010E9468A7B9
:1060300083E090E00E9439060E941A120E949D2F70
:10604000DF91CF91FF90EF900895EF92FF92CF9361
:10605000DF930E94652F8EE20E945E12BC01FC015C
:1060600001900020E9F73197E81BF90BCAE7D1E16D
:10607000CE01AF010E9468A780E30E945E12BC01BE
:10608000FC0101900020E9F73197E81BF90B9E0114
:106090002E1B3F0B2C5E3F4FC901AF010E9468A72A
:1060A00082E090E00E943906CE0160E270E044E1B7
:1060B00050E00E9471A78FE20E945E12BC01FC01B9
:1060C00001900020E9F73197E81BF90B9E012E5F44
:1060D0003F4FC901AF010E9468A781E30E945E1291
:1060E000BC01FC0101900020E9F73197E81BF90B96
:1060F000CE1BDF0B6296CE01AF010E9468A783E042
:1061000090E00E9439060E941A120E949D2FDF9192
:10611000CF91FF90EF90089580E10E94E3050895EC
:106120001F938091A911882309F49CC08091A81124
:10613000823051F1833020F4813009F093C007C0E0
:10614000833009F44AC0843009F08CC063C04091A8
:1061500094115091951160919611709197118091C1
:106160001A1290E020E00E94D3694091981150915A
:10617000991160919A1170919B1180911A1290E07F
:1061800020E00E94B9696EC010911A1220919411FA
:1061900030919511B901882777FD8095982F0E943D
:1061A00050A4AB01BC01812F90E020E00E9458690F
:1061B00010911A122091961130919711B9018827E8
:1061C00077FD8095982F0E9450A4AB01BC01812FD0
:1061D00090E020E00E94296945C0409194115091BF
:1061E0009511609196117091971180911A1290E01B
:1061F00020E00E949F6940919811509199116091FF
:106200009A1170919B1180911A1290E020E00E94E7
:10621000856928C010911A1220919411309195111E
:10622000B901882777FD8095982F0E9450A4AB0173
:10623000BC01812F90E020E00E94FC6810911A12AE
:106240002091961130919711B901882777FD80959B
:10625000982F0E9450A4AB01BC01812F90E020E058
:106260000E94CD681F9108958091A811823009F194
:10627000833020F4813009F099C006C08330F1F1F9
:10628000843009F093C06EC080911A1290E060E0F3
:106290000E944C67609394117093951180939611AE
:1062A0009093971180911A1290E060E00E944067ED
:1062B00039C080911A1290E060E00E9411670E943C
:1062C0001DA4709395116093941180911A1290E01F
:1062D00060E00E94FA660E941DA47093971160937B
:1062E000961184ED9EEF90939911809398118CE212
:1062F00091E090939B1180939A11089580911A12C6
:1063000090E060E00E94346760939411709395115F
:10631000809396119093971180911A1290E060E00B
:106320000E942867609398117093991180939A1135
:1063300090939B1180E090E0DC0180939C119093FE
:106340009D11A0939E11B0939F1180E090E0A6E96B
:10635000B2E48093A0119093A111A093A211B093E5
:10636000A311089580911A1290E060E00E94E36604
:106370000E941DA4709395116093941180911A123C
:1063800090E060E00E94CC660E941DA4709397117B
:106390006093961184ED9EEF9093991180939811DC
:1063A0008CE291E090939B1180939A110895CF9382
:1063B000DF930E9490308091A811833049F084309F
:1063C00069F0823019F0CFE0D0E00DC081E007C065
:1063D00082E08093A811C1E1D0E005C083E0809302
:1063E000A811C0E1D0E00E9434311092A91110929E
:1063F000A7118C2F0E94E305DF91CF910895CF93D1
:10640000DF930E9490308091A811833061F0843036
:1064100081F0823011F082E007C083E08093A81100
:10642000C0E1D0E00AC084E08093A811C1E1D0E0CF
:1064300004C01092A811C3E0D0E00E943431109241
:10644000A9111092A7118C2F0E94E305DF91CF9123
:1064500008950E94282F8BE061E00E949F04E09144
:10646000A711F0E0EE0FFF1FEE0FFF1FE157FE4EEA
:10647000658176818781908548E155E027E00E941B
:10648000930682E161E00E949F0486E50E94B204C7
:106490000895413051F4662311F46EE001C06CE0C0
:1064A00040E050E120E030E009C0662311F46EE0E6
:1064B00001C06CE040E050E020E030E10E94526812
:1064C0000895E091A611F0E0E157FE4E158A609123
:1064D0001A128BE1689FB00111249091A6118DE0F2
:1064E000989FC0011124680F791F615F7F4F80E082
:1064F0000E94EC2780911A126091A61140E00E9440
:1065000049320895E091A611F0E0E157FE4E84E093
:10651000858B60911A128BE1689FB00111249091D4
:10652000A6118DE0989FC0011124680F791F615F4B
:106530007F4F84E00E94EC2780911A126091A6118F
:1065400044E00E9449320895E091A611F0E0E1573D
:10655000FE4E83E0858B60911A128BE1689FB0013B
:1065600011249091A6118DE0989FC0011124680F0D
:10657000791F615F7F4F83E00E94EC2780911A12A0
:106580006091A61143E00E9449320895E091A6115E
:10659000F0E0E157FE4E82E0858B60911A128BE1AC
:1065A000689FB00111249091A6118DE0989FC001C1
:1065B0001124680F791F615F7F4F82E00E94EC27F2
:1065C00080911A126091A61142E00E94493208950A
:1065D000E091A611F0E0E157FE4E81E0858B6091DD
:1065E0001A128BE1689FB00111249091A6118DE0E1
:1065F000989FC0011124680F791F615F7F4F81E070
:106600000E94EC2780911A126091A61141E00E942D
:1066100049320895CF93DF938091A611882329F002
:10662000C091D611D091D71104C0C091D211D09190
:10663000D3118FE060E00E949F04CE010E94E3042A
:10664000E091A611F0E0E157FE4EE589F0E0EE0F93
:10665000FF1FE652FE4EC081D1818DE061E00E94B5
:106660009F04CE010E944B068FE891E10E94944660
:10667000DF91CF910895FF920F931F93082FF62E6D
:10668000662311F06CE001C06EE00E949A66192F3B
:10669000129511702BE1029F90011124215F3F4F51
:1066A0008DE04F2D489FC0011124820F931F60E0A1
:1066B00044E020E00E94F927813011F4812F02C0CC
:1066C000111181E01F910F91FF900895EF92FF92B9
:1066D0000F931F93CF93DF9380911A1260E00E9473
:1066E0003B338093A41180911A1261E00E943B33E6
:1066F0008093A5111092A61181E08093A8111092A9
:10670000A9111092A7110E943431CAE7D1E1CE013C
:1067100060E270E044E150E00E9471A789E00E94CD
:106720005E12BC01FC0101900020E9F73197E81BE3
:10673000F90B04E110E098012E1B3F0B36952795CD
:106740002C0F3D1FC901AF010E9468A780E090E0B7
:106750000E943906CE0160E270E044E150E00E9400
:1067600071A781E090E00E9439068EE40E945E12DB
:10677000BC01FC0101900020E9F73197E81BF90BFF
:10678000CE01AF010E9468A789E50E945E12BC019C
:10679000FC0101900020E9F73197E81BF90B980103
:1067A0002E1B3F0B369527952C0F3D1FC901AF01BE
:1067B0000E9468A783E50E945E12BC01FC01019063
:1067C0000020E9F73197E81BF90B0E1B1F0B0C0F8C
:1067D0001D1FC801AF010E9468A782E090E00E94DF
:1067E0003906CE0160E270E044E150E00E9471A7FA
:1067F00081E50E945E12BC01FC0101900020E9F7D6
:106800003197E81BF90B9E012E5F3F4FC901AF0185
:106810000E9468A785E50E945E12BC01FC01019000
:106820000020E9F73197E81BF90BCE1BDF0B6296CE
:10683000CE01AF010E9468A783E090E00E94390674
:106840000E941A120E949D2F8FE891E10E94D64665
:10685000DF91CF911F910F91FF90EF90089590914C
:106860008F11892F882311F48BE001C08150E82F0C
:10687000F0E0E75FFC4E2081222331F080938F11FE
:1068800081E0809390110895891761F708959091A0
:106890008F11892F8F5F8C3008F080E0E82FF0E0B7
:1068A000E75FFC4E2081222331F080938F1181E03D
:1068B000809390110895891769F70895AF92BF9258
:1068C000CF92DF92EF92FF920F931F93DF93CF93BC
:1068D000CDB7DEB72A970FB6F894DEBF0FBECDBF97
:1068E000809117138823F1F48091FB0D9091FC0D9A
:1068F000A091FD0DB091FE0D20919111309192115A
:106900004091931150919411821B930BA40BB50BE2
:10691000893C9105A105B10510F00E94BC051092BB
:106920009011DEC080919011882309F4D9C08AE7C4
:1069300091E160E270E044E150E00E9471A700E064
:1069400010E020E030E05E010894A11CB11C48E09A
:10695000C42ED12C96E6E92E95E0F92EF801E75FDA
:10696000FC4E8081882399F18DB79EB708970FB6AA
:10697000F8949EBF0FBE8DBFEDB7FEB73196ADB791
:10698000BEB71296BC92AE921197D382C282F582A4
:10699000E482C80101969783868329873A870E94FB
:1069A000CEA729853A85F901E658FE4E89819A815C
:1069B000918380832D5F3F4F8DB79EB708960FB6AA
:1069C000F8949EBF0FBE8DBF233131052CF40F5FAD
:1069D0001F4F0C30110511F681E090E00E9439063E
:1069E000E0918F11F0E0E75FFC4E8081882311F485
:1069F0000E9447340AE711E1C80160E270E044E117
:106A000050E00E9471A7E0918F11F0E0E75FFC4E2B
:106A1000808190E00E94EA8CE82FF0E0EE0FFF1FEB
:106A2000EB56FE4E60817181DB01FD01019000207B
:106A3000E9F73197EA1BFB0BC801AF010E9468A779
:106A4000ADB7BEB718970FB6F894BEBF0FBEADBFB7
:106A5000EDB7FEB731968E010F5F1F4F12961C9354
:106A60000E93119788E090E0938382838AE695E005
:106A70009583848380918F1190E00196978386831C
:106A80000E94CEA7F80101900020E9F73197E01BA2
:106A9000F10B2EE831E12E1B3F0B8DB79EB7089608
:106AA0000FB6F8949EBF0FBE8DBFC901B801AF01EC
:106AB0000E9468A783E090E00E943906109290112E
:106AC0008091FB0D9091FC0DA091FD0DB091FE0DFC
:106AD0008093911190939211A0939311B09394117C
:106AE0002A960FB6F894DEBF0FBECDBFCF91DF91CF
:106AF0001F910F91FF90EF90DF90CF90BF90AF90DC
:106B00000895EF92FF92CF93DF938BE080938F11E4
:106B10000E94473481E0809390118091FB0D909109
:106B2000FC0DA091FD0DB091FE0D809391119093FD
:106B30009211A0939311B0939411CAE7D1E1CE01C1
:106B400060E270E044E150E00E9471A784E10E949D
:106B50005E12BC01FC0101900020E9F73197E81BAF
:106B6000F90BCE01AF010E9468A780E090E00E947F
:106B70003906CE0160E270E044E150E00E9471A766
:106B800081E090E00E94390682E090E00E943906A0
:106B900083E090E00E9439060E941A128AE90E945E
:106BA0005E12909396118093951189E90E945E126E
:106BB000909398118093971188E90E945E129093A8
:106BC0009A1180939911DF91CF91FF90EF900895E2
:106BD00080911613882359F00E946505873221F4AD
:106BE00081E080939011089587E20E94E305089563
:106BF000EF92FF920F931F93DF93CF930F92CDB736
:106C0000DEB78091FB0D9091FC0DA091FD0DB09130
:106C1000FE0D20910A0E30910B0E40910C0E5091FA
:106C20000D0E7C018D01E21AF30A040B150BA8016D
:106C30009701253131054105510508F4B1C0809314
:106C40000A0E90930B0EA0930C0EB0930D0E809134
:106C5000090E823009F45FC0833009F48CC0BE0194
:106C60006F5F7F4F813039F1198285E898E30E9488
:106C70008B5C198183E094E00E94A264BC016F7375
:106C80007F73123071F0133018F4113071F40CC0AE
:106C9000133029F0143049F46068706806C06068E9
:106CA00004C06068706401C0706483E094E00E9476
:106CB000046881E05DC019828BE997E30E948B5CD8
:106CC000198183E094E00E94A264BC01637F737F1A
:106CD000143091F0153038F4123061F0133050F464
:106CE000113099F409C0163061F0163038F01730C1
:106CF00061F40AC06C6009C0646007C064607460BD
:106D000004C06C607C6001C07C6083E094E00E9401
:106D1000046882E02DC0198281EE96E3BE016F5FA8
:106D20007F4F0E948B5C198183E094E00E94A264F3
:106D3000BC016F7C7F7C133081F0143028F411305B
:106D400051F0123081F405C0143051F0153059F46F
:106D500009C0606108C0606306C06061706103C003
:106D6000706101C0706383E094E00E94046883E076
:106D70008093090E15C083E094E00E94A264BC01D8
:106D80006C7F7C7F80911713882319F480911513F1
:106D90008111716083E094E00E9404681092090EF2
:106DA0000F90CF91DF911F910F91FF90EF90089579
:106DB00083E094E060E070E00E9404681092090EA5
:106DC0000895CF92DF92EF92FF920F931F93CF938C
:106DD000DF93182F662319F421E030E0A2C0E42EDF
:106DE000E7017E01F52EE701812F6EE00E949A6691
:106DF00094FF43C0812F62E00E949A6696FF02C012
:106E000001E03CC0812F6EE00E949A666C01812FE8
:106E100063E00E949A66D4FE04C095FD02C002E0C1
:106E20002DC080911B12833041F5812F60E00E94BC
:106E30006A556B017C0120E030E040E450E40E94A0
:106E4000B1A3882314F405E019C0C701B60120E0FE
:106E500030E040EF50E40E94B1A3882314F404E032
:106E60000DC0C701B60120E030E040E751E40E94C8
:106E7000B1A3882314F403E001C000E0812F6CE08B
:106E80000E949A6694FF43C0812F62E00E949A6636
:106E900096FF02C081E03CC0812F6EE00E949A669E
:106EA0006C01812F63E00E949A66D4FE04C095FDB8
:106EB00002C082E02DC080911B12833041F5812FEA
:106EC00060E00E946A556B017C0120E030E040E404
:106ED00050E40E94B1A3882314F485E019C0C701CF
:106EE000B60120E030E040EF50E40E94B1A38823D7
:106EF00014F484E00DC0C701B60120E030E040E7A3
:106F000051E40E94B1A3882314F483E001C080E01F
:106F1000801708F4802F9881981708F4888320E060
:106F200030E0C901DF91CF911F910F91FF90EF9059
:106F3000DF90CF9008952F923F924F925F926F9281
:106F40007F928F929F92AF92BF92CF92DF92EF92F9
:106F5000FF920F931F93DF93CF9300D000D0CDB754
:106F6000DEB7182F662319F421E030E0B6C01A010D
:106F700090E00E9487674B015C01812F90E00E94A6
:106F8000D3676B017C01812F90E00E9481672B0108
:106F90003C01812F90E00E94CD6769837A838B83C7
:106FA0009C83C501B401A70196010E9404A56B0151
:106FB0007C01C301B20129813A814B815C810E942D
:106FC00004A59B01AC01C701B6010E944DA3D62EBA
:106FD000E72EF82E092F20E030E04AEF53EC0E9414
:106FE000B1A3181614F003E070C06D2D7E2D8F2D07
:106FF000902F20E030E048EC52EC0E94B1A318162C
:1070000014F004E062C06D2D7E2D8F2D902F20E0B6
:1070100030E84BEB54E40E9400A5181614F407E086
:1070200054C06D2D7E2D8F2D902F20E030E04AEF43
:1070300053E40E9400A5181614F406E046C06D2D16
:107040007E2D8F2D902F20E030E048EC52E40E94FE
:1070500000A5181614F405E038C0812F62E00E94E4
:107060009A6695FD02C000E014C0812F90E00E9456
:10707000D3676B017C01812F90E061E00E94116772
:107080009B01AC01C701B6010E94B1A387FD1CC0E2
:1070900001E0812F65E00E949A6695FF16C0812F5E
:1070A00090E00E94CD676B017C01812F90E061E050
:1070B0000E94E3669B01AC01C701B6010E94B1A327
:1070C00087FD02C001E001C002E0F101808180176C
:1070D00010F4F101008320E030E0C9010F900F901F
:1070E0000F900F90CF91DF911F910F91FF90EF9034
:1070F000DF90CF90BF90AF909F908F907F906F90D8
:107100005F904F903F902F900895EF92FF921F93C2
:10711000CF93DF93182F662319F421E030E032C0BB
:10712000E42EE7017E01F52EE701812F6BE00E943E
:10713000896693FF02C084E01FC0812F6BE00E942C
:10714000896692FF10C0812F6AE00E94896695FFD0
:1071500012C0812F6BE00E94896694FD02C082E01C
:107160000BC083E009C0812F6AE00E94896695FF09
:1071700002C081E001C080E09881981708F48883FC
:1071800020E030E0C901DF91CF911F91FF90EF9097
:10719000089583E10E94E30508958091A911882351
:1071A000E1F18091A811813019F08230B1F51BC056
:1071B0004091941150919511609196117091971191
:1071C00080911A1290E00E94B468409198115091F9
:1071D000991160919A1170919B1180911A1290E00F
:1071E0000E94996808954091941150919511609171
:1071F00096117091971180911A1290E00E94836805
:10720000409198115091991160919A1170919B1130
:1072100080911A1290E00E94686808958091A811E8
:10722000813019F08230B1F51BC080911A1290E0C4
:107230000E94C46660939411709395118093961187
:107240009093971180911A1290E00E94BB66609310
:1072500098117093991180939A1190939B110895AE
:1072600080911A1290E00E94B0666093941170931E
:107270009511809396119093971180911A1290E036
:107280000E94A166609398117093991180939A114E
:1072900090939B1108950E94CD388091A81182305F
:1072A00021F082E10E94E305089581E08093A81116
:1072B0000E940E391092A9111092A71108950E94F0
:1072C000CD388091A811823051F082E08093A811CE
:1072D0000E940E391092A9111092A711089583E00F
:1072E0000E94E3050895CF93DF930E94152580E067
:1072F00060E00E949F04CFE8D1E1E091A711F0E0A7
:107300007096EE0FFF1FEC0FFD1F808191810E9490
:107310004B0683E061E00E949F04E091A811F0E039
:10732000EE0FFF1FE053FE4E808191810E944B06BD
:107330008BE061E00E949F04E091A711F0E0EE0F66
:10734000FF1FEE0FFF1FEC0FFD1F65817681878108
:1073500090854AE855E027E00E94930682E161E0CB
:107360000E949F0486E50E94B204DF91CF910895A8
:10737000EF92FF92CF93DF931092AA1180E090E0FA
:10738000DC0180939C1190939D11A0939E11B0936A
:107390009F1180E090E0A6E9B2E48093A011909361
:1073A000A111A093A211B093A3110E94482289E5D4
:1073B0000E945E129093D1118093D01188E30E94B5
:1073C0005E129093D3118093D21189E30E945E12D2
:1073D0009093D5118093D411CAE7D1E1CE0160E238
:1073E00070E044E150E00E9471A78EE50E945E12B9
:1073F000BC01FC0101900020E9F73197E81BF90B73
:107400002AE030E02E1B3F0B36952795265F3F4F35
:107410002C0F3D1FC901AF010E9468A780E090E0DA
:107420000E943906CE0160E270E044E150E00E9423
:1074300071A781E090E00E9439068EE20E945E1200
:10744000BC01FC0101900020E9F73197E81BF90B22
:10745000CE01AF010E9468A780E30E945E12BC01CA
:10746000FC0101900020E9F73197E81BF90B9E0120
:107470002E1B3F0B2C5E3F4FC901AF010E9468A736
:1074800082E090E00E943906CE0160E270E044E1C3
:1074900050E00E9471A78FE20E945E12BC01FC01C5
:1074A00001900020E9F73197E81BF90B9E012E5F50
:1074B0003F4FC901AF010E9468A781E30E945E129D
:1074C000BC01FC0101900020E9F73197E81BF90BA2
:1074D000CE1BDF0B6296CE01AF010E9468A783E04E
:1074E00090E00E943906DF91CF91FF90EF900895D0
:1074F0001092A41160911A128BE1689FB0011124BF
:10750000625F7F4F80E00E94EC27089584E08093C3
:10751000A41160911A128BE1689FB0011124625F7F
:107520007F4F84E00E94EC27089583E08093A411AC
:1075300060911A128BE1689FB0011124625F7F4F46
:1075400083E00E94EC27089582E08093A41160916B
:107550001A128BE1689FB0011124625F7F4F82E0B5
:107560000E94EC27089581E08093A41160911A1283
:107570008BE1689FB0011124625F7F4F81E00E9420
:10758000EC270895CF93DF93E091A411F0E0EE0F84
:10759000FF1FEA52FE4EC081D1818DE061E00E9462
:1075A0009F04CE010E944B068FE891E10E94944611
:1075B000DF91CF910895EF92FF920F931F93CF9396
:1075C000DF9390911A128BE1989FC00111240E96BF
:1075D00060E044E020E00E94F9278093A41181E05C
:1075E0008093A8111092A9111092A7110E940E3930
:1075F000CAE7D1E1CE0160E270E044E150E00E94D0
:1076000071A78AE00E945E12BC01FC01019000207B
:10761000E9F73197E81BF90B04E110E098012E1B04
:107620003F0B369527952C0F3D1FC901AF010E94D6
:1076300068A780E090E00E943906CE0160E270E029
:1076400044E150E00E9471A781E090E00E94390679
:1076500086E50E945E12BC01FC0101900020E9F762
:107660003197E81BF90BCE01AF010E9468A789E5AD
:107670000E945E12BC01FC0101900020E9F73197E5
:10768000E81BF90B98012E1B3F0B369527952C0F05
:107690003D1FC901AF010E9468A788E50E945E12E4
:1076A000BC01FC0101900020E9F73197E81BF90BC0
:1076B0000E1B1F0B0C0F1D1FC801AF010E9468A7F6
:1076C00082E090E00E943906CE0160E270E044E181
:1076D00050E00E9471A785E50E945E12BC01FC018A
:1076E00001900020E9F73197E81BF90B9E012E5F0E
:1076F0003F4FC901AF010E9468A787E50E945E1253
:10770000BC01FC0101900020E9F73197E81BF90B5F
:10771000CE1BDF0B6296CE01AF010E9468A783E00B
:1077200090E00E9439060E941A1289E80E945E12B7
:107730009093D7118093D6118FE80E945E12909398
:10774000D9118093D8118DE80E945E129093DB11BD
:107750008093DA1180E90E945E129093DD1180938C
:10776000DC118EE80E945E129093DF118093DE118F
:107770008FE891E10E94D646DF91CF911F910F9142
:10778000FF90EF9008958CE08093941181E08093B6
:107790009611089588E18093941181E08093961169
:1077A000089584E28093941181E080939611089566
:1077B00080919111823030F081508093911181E05D
:1077C00080939611089580919111803230F48F5FEB
:1077D0008093911181E08093961108958091971183
:1077E000909198112FEF843F9207F0F40A969093AE
:1077F0009811809397118091901185508230E0F01C
:1078000085E0809390118091FB0D9091FC0DA091EB
:10781000FD0DB091FE0D80939B1190939C11A09350
:107820009D11B0939E1108C0109290118EEF9FEFA2
:10783000909398118093971181E080939611089509
:1078400080919711909198118A309105F0F00A97E4
:107850009093981180939711809190118750823066
:10786000D0F087E0809390118091FB0D9091FC0DFA
:10787000A091FD0DB091FE0D80939B1190939C11F2
:10788000A0939D11B0939E1106C01092901110927A
:1078900098111092971181E080939611089580912C
:1078A0009711909198112FEF8D3F9207F0F4019668
:1078B000909398118093971180919011815082300C
:1078C000E0F081E0809390118091FB0D9091FC0D90
:1078D000A091FD0DB091FE0D80939B1190939C1192
:1078E000A0939D11B0939E1108C0109290118EEF3D
:1078F0009FEF909398118093971181E08093961158
:10790000089580919711909198110097F1F0019747
:1079100090939811809397118091901183508230A9
:10792000D0F083E0809390118091FB0D9091FC0D3D
:10793000A091FD0DB091FE0D80939B1190939C1131
:10794000A0939D11B0939E1106C0109290111092B9
:1079500098111092971181E0809396110895EF92FB
:10796000FF920F931F93CF93DF9380919011882301
:1079700009F499C00E944409882309F494C08091B5
:107980009011853030F4833050F4813008F48BC08E
:107990000BC0873070F0893008F085C00FC080E4DC
:1079A00090E0C1E8DCE30EC080E290E0CFE4DCE3ED
:1079B00009C080E091E0CEEEDBE304C080E890E017
:1079C000C0E2DCE30E944F09882309F46EC0809175
:1079D0009011843009F43FC0853040F48230D9F1F1
:1079E000833070F4813009F05EC00AC0863099F1AE
:1079F000863030F0873021F0883009F054C02BC039
:107A00008091FB0D9091FC0DA091FD0DB091FE0DAC
:107A100020919B1130919C1140919D1150919E118C
:107A20007C018D01E21AF30A040B150BA8019701E2
:107A30002536310541055105C0F180939B11909386
:107A40009C11A0939D11B0939E11809190118F5F16
:107A5000809390112AC08091FB0D9091FC0DA09114
:107A6000FD0DB091FE0D20919B1130919C11409124
:107A70009D1150919E117C018D01E21AF30A040BB5
:107A8000150BA80197012B3031054105510568F010
:107A900080939B1190939C11A0939D11B0939E1184
:107AA000FE01099502C010929011C0919711D091DA
:107AB00098118091991190919A11C817D90761F185
:107AC00082E061E00E949F04CE0160EC75E045E039
:107AD0000E944E068BE061E00E949F04BE0180E0A0
:107AE00090E00E944EA420E030E040E752E40E9483
:107AF00004A520E030E04AE754E40E94B5A344EC3A
:107B000055E028E00E94930680919711909198117A
:107B100090939A1180939911DF91CF911F910F91BA
:107B2000FF90EF900895CF92DF92EF92FF920F9324
:107B30001F93CF93DF9381E080938F111092901168
:107B40008FEF9FEF90939A11809399111092961155
:107B500090911A128BE1989FC001112430911C1250
:107B60002DE0329F90011124820F931F449640E034
:107B700050E0BA0100E21EEF2FE63AE40F2EF0E0EB
:107B8000CF2EF0E8DF2EFBEBEF2EF5E4FF2EF02DED
:107B90000E94162920E030E040E752E40E94B5A39D
:107BA0007B018C017F2D912F20E030E0A9010E9404
:107BB000B1A318162CF010929811109297111FC0B3
:107BC0006E2D7F2D802F912F20E03FEF4FE757E460
:107BD0000E9400A518163CF48EEF9FEF9093981129
:107BE000809397110CC06E2D7F2D802F912F0E94B6
:107BF00067A50E9422A470939811609397110AE7D9
:107C000011E1C80160E270E044E150E00E9471A718
:107C100087E60E945E12BC01FC0101900020E9F79A
:107C20003197E81BF90B2AE030E02E1B3F0B36950D
:107C30002795200F311FC901AF010E9468A788E670
:107C40000E945E12BC01FC0101900020E9F731970F
:107C5000E81BF90BC4E1D0E09E012E1B3F0B200F67
:107C6000311FC901AF010E9468A780E090E00E9427
:107C70003906C80160E270E044E150E00E9471A75B
:107C800081E090E00E9439068CE20E945E12BC0105
:107C9000FC0101900020E9F73197E81BF90BC801BE
:107CA000AF010E9468A78AE20E945E12BC01FC013B
:107CB00001900020E9F73197E81BF90BCE1BDF0B91
:107CC000C00FD11FCE01AF010E9468A782E090E0F3
:107CD0000E943906C80160E270E044E150E00E9471
:107CE00071A78DE20E945E12BC01FC010190002090
:107CF000E9F73197E81BF90B0E5F1F4FC801AF0181
:107D00000E9468A78BE20E945E12BC01FC010190F8
:107D10000020E9F73197E81BF90B2CE831E12E1B25
:107D20003F0BC901AF010E9468A783E090E00E9469
:107D30003906DF91CF911F910F91FF90EF90DF9067
:107D4000CF9008950F931F9380919611882361F12E
:107D500060911A120BE1609FB001112480911C12F6
:107D60001DE0819FC0011124680F791F605F7F4F64
:107D7000809191110E94EC2760911A12609FB001CE
:107D8000112480911C12819FC0011124680F791F5A
:107D90006F5E7F4F809194110E94EC2780911A12A0
:107DA00060911C120E942C561F910F9108951F93F1
:107DB000DF93CF9300D000D0CDB7DEB7182F8091DE
:107DC0008F11882319F08130B9F503C00E94A23EBB
:107DD00033C080919611882379F1209197113091C9
:107DE00098118CE390E0289FB001299F700D389F77
:107DF000700D112480E090E00E944EA469837A8384
:107E00008B839C8360911A128BE1689FB0011124CF
:107E100090911C128DE0989FC0011124680F791F6A
:107E20006C5E7F4FCE0101960E94532880911A12FA
:107E300060911C120E942C56812F0E94E3050F9026
:107E40000F900F900F90CF91DF911F910895809127
:107E50008F11813011F083E001C084E10E94D73E90
:107E6000089580918F11882311F086E101C085E18A
:107E70000E94D73E08950F931F9380911A120BE131
:107E8000809FC001112420911C121DE0219F9001B0
:107E90001124820F931F409661E040E221E00E948E
:107EA000F9278093911180911A12809FC0011124AB
:107EB00020911C12219F90011124820F931F419643
:107EC0006CE044E22CE00E94F92780939411109218
:107ED00096111F910F91089580911C12882361F4CF
:107EE00080919311882391F00E94A23E81E08093BB
:107EF0001C120E943B3F089580919211882331F01B
:107F00000E94A23E10921C120E943B3F0895EF92E5
:107F1000FF920F931F93DF93CF93CDB7DEB72997CF
:107F20000FB6F894DEBF0FBECDBF82E160E00E94C5
:107F30009F048091911190E06BEC75E042E00E940B
:107F40004E060AE711E1C80160E270E044E150E04A
:107F50000E9471A780911A122BE1829FC001112407
:107F600040911C123DE0439FA0011124840F951FF6
:107F7000429660E044E020E039870E94F927E82F2C
:107F8000F0E0EE0FFF1FE852FE4E60817181DB01D1
:107F9000FD0101900020E9F73197EA1BFB0BC801B6
:107FA000AF010E9468A78DB79EB708970FB6F894E7
:107FB0009EBF0FBE8DBFEDB7FEB731967E01089410
:107FC000E11CF11CADB7BEB71296FC92EE92119770
:107FD00088E090E0938382838091D0119091D111B9
:107FE0009583848380911A1290E00196978386830B
:107FF0000E94CEA7F70101900020E9F73197EE1912
:10800000FF0904E110E0A8014E1B5F0B5695479550
:1080100046585E4E8DB79EB708960FB6F8949EBF31
:108020000FBE8DBFCA01B701AF010E9468A7809142
:108030001A12ABE18A9FC001112420911C123985CC
:10804000239F90011124820F931F439660E043E029
:1080500020E00E94F927E82FF0E0EE0FFF1FEE511D
:10806000FE4E60817181DB01FD0101900020E9F786
:108070003197EA1BFB0B0E1B1F0B06581E4EC80147
:10808000AF010E9468A781E090E00E94390688E075
:1080900063E00E949F048091941190E06BEC75E086
:1080A00042E00E944E0680919511882329F40091A8
:1080B000D2119091D31109C0E0911C12F0E0EE0FA3
:1080C000FF1FEC52FE4E00819181E02FF92FDF015E
:1080D0000D900020E9F7EA1B8E2F8B5E62E09987F6
:1080E0000E949F04802F99850E944B0629960FB607
:1080F000F894DEBF0FBECDBFCF91DF911F910F91DE
:10810000FF90EF900895EF92FF92CF93DF9310923C
:108110008F1180911A126EE00E949A66929591706A
:108120009093921180911A126CE00E949A66929537
:1081300091709093931180919211292F280F209381
:108140009511992311F0882319F010921C1203C085
:1081500081E080931C120E943B3FCAE7D1E1CE012F
:1081600060E270E044E150E00E9471A786E60E9460
:108170005E12BC01FC0101900020E9F73197E81B79
:10818000F90BCE01AF010E9468A780E090E00E9449
:108190003906CE0160E270E044E150E00E9471A730
:1081A0008FE30E945E12BC01FC0101900020E9F700
:1081B0003197E81BF90B9E01295F3F4FC901AF01C1
:1081C0000E9468A781E090E00E943906CE0160E23B
:1081D00070E044E150E00E9471A781E90E945E12C4
:1081E000BC01FC0101900020E9F73197E81BF90B75
:1081F000CE01AF010E9468A782E090E00E9439069C
:10820000CE0160E270E044E150E00E9471A782E993
:108210000E945E12BC01FC0101900020E9F7319739
:10822000E81BF90B2296CE01AF010E9468A783E9F3
:108230000E945E12BC01FC0101900020E9F7319719
:10824000E81BF90B2CE831E12E1B3F0BC901AF01F4
:108250000E9468A786E58093841183E090E00E94E5
:1082600039060E941A128BE00E945E129093D1117F
:108270008093D01189E50E945E129093D311809370
:10828000D21187E80E945E129093D5118093D41189
:1082900088E80E945E129093D7118093D611CAE3AA
:1082A000D2E0D093D911C093D81189E60E945E1212
:1082B0009093DB118093DA118BE60E945E1290930B
:1082C000DD118093DC118AE60E945E129093DF112B
:1082D0008093DE118CE60E945E129093E1118093F0
:1082E000E011D093E311C093E2118FE60E945E1279
:1082F0009093E5118093E4118EE60E945E129093B4
:10830000E7118093E61180E70E945E129093E911D5
:108310008093E811DF91CF91FF90EF9008951F9324
:108320008091A811813021F08230B1F511E001C0B7
:1083300010E09091A61180911A12409194115091E1
:1083400095116091961170919711992399F090E091
:10835000212F0E949F69409198115091991160912D
:108360009A1170919B1180911A1290E0212F0E9416
:10837000856912C090E0212F0E94D3694091981125
:108380005091991160919A1170919B1180911A12DC
:1083900090E0212F0E94B9691F9108951F93809149
:1083A000A811813021F08230B1F511E001C010E058
:1083B0009091A61180911A12992399F090E0612F63
:1083C0000E94346760939411709395118093961175
:1083D0009093971180911A1290E0612F0E94286764
:1083E00012C090E0612F0E944C67609394117093CB
:1083F0009511809396119093971180911A1290E0A5
:10840000612F0E9440676093981170939911809337
:108410009A1190939B111F9108950E948F41809112
:10842000A811823021F085E10E94E305089581E0E2
:108430008093A8111092A9111092A7110E94CE4109
:1084400008950E948F418091A811823051F082E0FE
:108450008093A8111092A9111092A7110E94CE41E9
:10846000089587E10E94E30508951F93DF93CF935A
:108470000F92CDB7DEB70E94152580E060E00E9424
:108480009F04E091A711F0E0EE0FFF1FE155FE4EB3
:10849000808191810E944B068091A811813029F43E
:1084A0001091D0119091D11104C01091D2119091DE
:1084B000D311E12FF92FDF010D900020E9F79F0183
:1084C0002A1B3B0B255F3F4F36952795822F61E096
:1084D00099830E949F04812F99810E944B068BE013
:1084E00061E00E949F04E091A711F0E0EE0FFF1FF2
:1084F000EE0FFF1FE157FE4E6581768187819085E3
:1085000040E056E027E00E94930682E161E00E948D
:108510009F0486E50E94B2040F90CF91DF911F91D6
:108520000895EF92FF92CF93DF9381E08093A8119B
:108530001092A9111092A71180911A126CE00E945A
:108540009A66929591709093A6111092AA1180E06C
:1085500090E0DC0180939C1190939D11A0939E115B
:10856000B0939F1180E090E0A8E4B2E48093A01162
:108570009093A111A093A211B093A3110E94CE4198
:10858000CAE7D1E1CE0160E270E044E150E00E9430
:1085900071A78EE50E945E12BC01FC0101900020D3
:1085A000E9F73197E81BF90B2AE030E02E1B3F0B6F
:1085B00036952795265F3F4F2C0F3D1FC901AF0110
:1085C0000E9468A780E090E00E943906CE0160E238
:1085D00070E044E150E00E9471A781E090E00E94C9
:1085E00039068EE20E945E12BC01FC01019000205F
:1085F000E9F73197E81BF90BCE01AF010E9468A79C
:1086000080E30E945E12BC01FC0101900020E9F7AA
:108610003197E81BF90B9E012E1B3F0B2C5E3F4F41
:10862000C901AF010E9468A782E090E00E9439066C
:10863000CE0160E270E044E150E00E9471A78FE259
:108640000E945E12BC01FC0101900020E9F7319705
:10865000E81BF90B9E012E5F3F4FC901AF010E943D
:1086600068A781E30E945E12BC01FC01019000201A
:10867000E9F73197E81BF90BCE1BDF0B6296CE01B1
:10868000AF010E9468A783E090E00E9439060E9433
:108690001A120E94482284E90E945E129093D1111E
:1086A0008093D01185E90E945E129093D31180933C
:1086B000D211DF91CF91FF90EF900895EF92FF924A
:1086C0000F931F93CF93DF9310929411CAE7D1E1D8
:1086D000CE0160E270E044E150E00E9471A789E6BB
:1086E0000E945E12BC01FC0101900020E9F7319765
:1086F000E81BF90BCE01AF010E9468A785E10E943B
:108700005E12BC01FC0101900020E9F73197E81BE3
:10871000F90B04E110E098012E1B3F0B36952795CD
:108720002C0F3D1FC901AF010E9468A78AE60E9475
:108730005E12BC01FC0101900020E9F73197E81BB3
:10874000F90B0E1B1F0B0C0F1D1FC801AF010E9460
:1087500068A782E090E00E943906CE0160E270E0F6
:1087600044E150E00E9471A78BE60E945E12BC01BA
:10877000FC0101900020E9F73197E81BF90B9E01FD
:108780002E5F3F4FC901AF010E9468A78CE60E948F
:108790005E12BC01FC0101900020E9F73197E81B53
:1087A000F90BCE1BDF0B6296CE01AF010E9468A7CA
:1087B00083E090E00E943906DF91CF911F910F91E5
:1087C000FF90EF90089580919411882319F40E94EE
:1087D000BC0508950E945E430895EF92FF92CF93E7
:1087E000DF9381E080939411CAE7D1E1CE0160E28A
:1087F00070E044E150E00E9471A78DE60E945E1295
:10880000BC01FC0101900020E9F73197E81BF90B4E
:10881000CE01AF010E9468A78EE60E945E12BC01E5
:10882000FC0101900020E9F73197E81BF90B9E014C
:108830002E1B3F0B2C5E3F4FC901AF010E9468A762
:1088400082E090E00E943906CE0160E270E044E1EF
:1088500050E00E9471A78FE60E945E12BC01FC01ED
:1088600001900020E9F73197E81BF90B9E012E5F7C
:108870003F4FC901AF010E9468A780E70E945E12C6
:10888000BC01FC0101900020E9F73197E81BF90BCE
:10889000CE1BDF0B6296CE01AF010E9468A783E07A
:1088A00090E00E943906DF91CF91FF90EF900895FC
:1088B00080919411882349F480919511813029F495
:1088C0000E941A120E94ED4308950E940106089525
:1088D0000F931F939091941160911A1280911C1222
:1088E000992311F593E0909395110BE1609FB001EE
:1088F00011241DE0819FC0011124680F791F6E5E55
:108900007F4F83E00E94EC2760911A12609FB001B4
:10891000112480911C12819FC0011124680F791FBE
:108920006D5E7F4F80E010C092E0909396119BE1C6
:10893000699FB00111249DE0899FC0011124680F37
:10894000791F6D5E7F4F82E00E94EC2780911A12A2
:1089500060911C120E942C560E9401061F910F91DB
:1089600008950F931F939091941160911A12809122
:108970001C12992311F594E0909395110BE1609FDF
:10898000B00111241DE0819FC0011124680F791FDF
:108990006E5E7F4F84E00E94EC2760911A12609F08
:1089A000B001112480911C12819FC0011124680F15
:1089B000791F6D5E7F4F80E010C093E09093961119
:1089C0009BE1699FB00111249DE0899FC0011124A2
:1089D000680F791F6D5E7F4F83E00E94EC278091C6
:1089E0001A1260911C120E942C560E9401061F91BF
:1089F0000F9108950F931F939091941160911A1203
:108A000080911C12992311F592E0909395110BE13E
:108A1000609FB00111241DE0819FC0011124680FE7
:108A2000791F6E5E7F4F82E00E94EC2760911A12E0
:108A3000609FB001112480911C12819FC0011124FC
:108A4000680F791F6D5E7F4F80E010C091E09093BA
:108A500096119BE1699FB00111249DE0899FC0019F
:108A60001124680F791F6D5E7F4F81E00E94EC2713
:108A700080911A1260911C120E942C560E940106CD
:108A80001F910F91089580919411882301F581E041
:108A90008093951160911A128BE1689FB0011124A7
:108AA00090911C128DE0989FC0011124680F791FCE
:108AB0006E5E7F4F81E00E94EC2780911A126091D8
:108AC0001C120E942C560E941A120E94ED43089517
:108AD0008FE891E10E9494460895EF92FF920F93E0
:108AE0001F93DF93CF93CDB7DEB728970FB6F894D7
:108AF000DEBF0FBECDBF80911A121BE1819FC00166
:108B0000112420911C120DE0209F90011124820F4E
:108B1000931F429660E044E020E00E94F927809392
:108B2000951160911A1220911C12813089F4619F75
:108B3000C0011124209F80011124800F911F4396B2
:108B400060E043E020E00E94F927809396110FC077
:108B500010929611619FB0011124209F8001112471
:108B6000600F711F6D5E7F4F80E00E94EC278AE7E7
:108B700091E160E270E044E150E00E9471A781E081
:108B80000E945E12BC01FC0101900020E9F73197C0
:108B9000E81BF90B04E110E098012E1B3F0B369502
:108BA000279526583E4EC901AF010E9468A780E074
:108BB00090E00E9439068AE791E160E270E044E1CA
:108BC00050E00E9471A78BE00E945E122DB73EB765
:108BD000285030400FB6F8943EBF0FBE2DBFEDB702
:108BE000FEB731967E010894E11CF11CADB7BEB70B
:108BF0001296FC92EE92119728E030E033832283A4
:108C00009583848380911A1290E0019697838683DE
:108C10000E94CEA7F70101900020E9F73197EE19E5
:108C2000FF090E1B1F0B1695079506581E4E2DB7F4
:108C30003EB7285F3F4F0FB6F8943EBF0FBE2DBF23
:108C4000C801B701AF010E9468A781E090E00E94CF
:108C500039060E945E438FE891E10E94D64628962D
:108C60000FB6F894DEBF0FBECDBFCF91DF911F913D
:108C70000F91FF90EF900895FF920F931F93082F8D
:108C8000F62E8430C0F4862F602F0E949F0410E0DF
:108C9000812F0E942B041F5F1430D1F7033059F04D
:108CA000602F6F5F8F2D0E949F04812F0E942B04E5
:108CB0001F5F1830D1F71F910F91FF900895AF9269
:108CC000BF92CF92DF92EF92FF921F93CF93DF93E9
:108CD0007C01162FC0E0D0E08C2F612F0E94900401
:108CE0006E0183E0CC0CDD1C8A95E1F7CE0CDF1C15
:108CF000AA24BB24F60181916F010E942B040894E1
:108D0000A11CB11CF8E0AF16B104A1F72196C83040
:108D1000D10511F7DF91CF911F91FF90EF90DF9078
:108D2000CF90BF90AF900895CF93DF93EC016C810B
:108D30002091FB0D3091FC0D4091FD0D5091FE0DE9
:108D400088819981AA81BB81662371F4281B390B24
:108D50004A0B5B0B203531054105510520F181E0BF
:108D60008C8386E796E00CC0281B390B4A0B5B0B03
:108D70002431310541055105B0F01C8286E396E0AF
:108D800060E00E945F4680E060E00E943C46809187
:108D9000FB0D9091FC0DA091FD0DB091FE0D88830F
:108DA0009983AA83BB83DF91CF910895CF93DF93FB
:108DB000EC0186E396E060E00E945F4680E060E0C0
:108DC0000E943C468091FB0D9091FC0DA091FD0D01
:108DD000B091FE0D88839983AA83BB831C82DF91A7
:108DE000CF9108958091FB0D9091FC0DA091FD0D08
:108DF000B091FE0D20918F11309190114091911101
:108E000050919211821B930BA40BB50B893E23E06A
:108E1000920720E0A20720E0B20710F00E94BC05F4
:108E2000089580E060E041E00E94ED600895EF92D7
:108E3000FF920F931F93CF93DF938091FB0D90913F
:108E4000FC0DA091FD0DB091FE0D80938F119093BC
:108E50009011A0939111B0939211CAE7D1E1CE0184
:108E600060E270E044E150E00E9471A782E10E945C
:108E70005E12BC01FC0101900020E9F73197E81B6C
:108E8000F90B8E010B5F1F4FC801AF010E9468A74D
:108E900080E090E00E943906CE0160E270E044E19B
:108EA00050E00E9471A783E10E945E12BC01FC01A8
:108EB00001900020E9F73197E81BF90BC801AF01D9
:108EC0000E9468A781E090E00E943906CE0160E22E
:108ED00070E044E150E00E9471A781E70E945E12B9
:108EE000BC01FC0101900020E9F73197E81BF90B68
:108EF000CE01AF010E9468A782E70E945E12BC010A
:108F0000FC0101900020E9F73197E81BF90B9E0165
:108F10002E1B3F0B2C5E3F4FC901AF010E9468A77B
:108F200082E090E00E943906CE0160E270E044E108
:108F300050E00E9471A783E090E00E94390686EB22
:108F400096E060E00E945F4680E060E00E943C4660
:108F5000DF91CF911F910F91FF90EF900895809135
:108F600017128093230E2091FB0D3091FC0D409140
:108F7000FD0D5091FE0D285230404040504020934E
:108F80000E0E30930F0E4093100E5093110E90E082
:108F90000E9487676093311270933212809333126C
:108FA000909334128091230E90E00E94D3679B012E
:108FB000AC0160932112709322128093231290933C
:108FC000241260913112709132128091331290917B
:108FD00034120E9404A56093291270932A12809380
:108FE0002B1290932C128091230E90E00E948167A7
:108FF0006093351270933612809337129093381223
:109000008091230E90E00E94CD679B01AC0160939C
:109010002512709326128093271290932812609144
:1090200035127091361280913712909138120E9449
:1090300004A560932D1270932E1280932F1290939B
:1090400030121092120E1092130E1092140E1092F3
:10905000150E1092160E1092170E1092180E1092F6
:10906000190E10921A0E10921B0E10921C0E1092D6
:109070001D0E10921E0E10921F0E1092200E1092B6
:10908000210E1092220E0895CF92DF92EF92FF925E
:109090000F931F93909117128091230E981711F040
:1090A0000E94AF478091FB0D9091FC0DA091FD0DAA
:1090B000B091FE0D20910E0E30910F0E4091100ECA
:1090C0005091110E7C018D01E21AF30A040B150B6D
:1090D000A8019701223331054105510508F4AEC1BD
:1090E00080930E0E90930F0EA093100EB093110E5E
:1090F000E090120EF090130E0091140E1091150EC8
:109100008091230E60E00E949A66A0E0B0E09F701C
:10911000A070B0708E0D9F1DA01FB11F8093120E06
:109120009093130EA093140EB093150EE090160EAC
:10913000F090170E0091180E1091190E8091230EC9
:1091400064E00E949A66A0E0B0E09F70A070B070EA
:109150008E0D9F1DA01FB11F8093160E9093170EAA
:10916000A093180EB093190EE0901A0EF0901B0EFB
:1091700000911C0E10911D0E8091230E65E00E943F
:109180008D67AA2797FDA095BA2F8E0D9F1DA01F52
:10919000B11F80931A0E90931B0EA0931C0EB093D8
:1091A0001D0EE0901E0EF0901F0E0091200E1091EB
:1091B000210E8091230E62E00E948D67AA2797FD01
:1091C000A095BA2F8E0D9F1DA01FB11F80931E0E5C
:1091D00090931F0EA093200EB093210E8091220E2B
:1091E0008F5F8093220E843008F428C1C0908D04D4
:1091F000D0908E04E0908F04F09090048EE992E07D
:1092000040E050E068E472EC00E010E028E432E472
:109210000E9416297B018C016091120E7091130E31
:109220008091140E9091150E0E9450A49B01AC01E8
:10923000C801B7010E9404A520E030E040E85EE3E9
:109240000E9404A5609331127093321280933312FE
:1092500090933412C0909104D0909204E0909304C3
:10926000F090940482EA92E040E050E068E472EC0E
:1092700000E010E028E432E40E9416297B018C0112
:109280006091160E7091170E8091180E9091190E24
:109290000E9450A49B01AC01C801B7010E9404A523
:1092A00020E030E040E85EE30E9404A560933512C0
:1092B000709336128093371290933812C0909504B1
:1092C000D0909604E0909704F090980486EA92E09B
:1092D00040E050E068E472EC00E010E028E432E4A2
:1092E0000E9416297B018C0160911A0E70911B0E51
:1092F00080911C0E90911D0E0E9450A49B01AC0108
:10930000C801B7010E9404A520E030E040E85EE318
:109310000E9404A56093211270932212809323125D
:1093200090932412C0909904D0909A04E0909B04EA
:10933000F0909C048AEA92E040E050E068E472EC2D
:1093400000E010E028E432E40E9416297B018C0141
:1093500060911E0E70911F0E8091200E9091210E33
:109360000E9450A49B01AC01C801B7010E9404A552
:1093700020E030E040E85EE30E9404A57B018C0120
:10938000862F9F2DA02FB12F809325129093261208
:10939000A0932712B093281260913112709132126B
:1093A0008091331290913412209121123091221227
:1093B00040912312509124120E9404A56093291217
:1093C00070932A1280932B1290932C126091351275
:1093D0007091361280913712909138122E2D3F2DB8
:1093E000402F512F0E9404A560932D1270932E12CE
:1093F00080932F12909330121092120E1092130E2F
:109400001092140E1092150E1092160E1092170E46
:109410001092180E1092190E10921A0E10921B0E26
:1094200010921C0E10921D0E10921E0E10921F0E06
:109430001092200E1092210E1092220E1F910F9169
:10944000FF90EF90DF90CF9008952F923F924F9230
:109450005F926F927F928F929F92AF92BF92CF92C4
:10946000DF92EF92FF920F931F935A016B017801E5
:109470008901E82FF0E0EE0FFF1FEE0FFF1FE75B03
:10948000FD4E208031804280538060E070E088ECA7
:1094900092E4A20191010E944CA39B01AC01C8017E
:1094A000B7010E9404A5A60195010E94B5A320E082
:1094B00030E048EC52E40E94B5A3962E872E782E19
:1094C000692EA62EB72EC82ED92E8C2D880F8D2D45
:1094D000881F8F3FA9F0692D782D872D962D20E0CC
:1094E00030E0A9010E94B1A387FD0AC0692D782D43
:1094F000872D962DA80197010E9400A5181684F4C7
:10950000C801B701A20191010E9404A520E030E04A
:1095100048EC52E40E94B5A3A62EB72EC82ED92E31
:109520006A2D7B2D8C2D9D2D1F910F91FF90EF901B
:10953000DF90CF90BF90AF909F908F907F906F9073
:109540005F904F903F902F9008956F927F928F92EF
:109550009F92AF92BF92CF92DF92EF92FF920F93C2
:109560001F933B014C01CA01B901A80197010E9458
:1095700004A5A60195010E94B5A39B01AC01C401FD
:10958000B3010E944DA31F910F91FF90EF90DF90C8
:10959000CF90BF90AF909F908F907F906F900895E5
:1095A000882359F4809117126EE00E949A6694FF06
:1095B00017C08091171262E00CC0813089F480914D
:1095C00017126CE00E949A6694FF0AC080911712ED
:1095D00065E00E949A66892F82958695817008952C
:1095E00080E008951F93CF93DF93182F0E94D04AF5
:1095F000212F30E0F901E75DF14F8083220F331F07
:10960000220F331FF901EF5BFD4E80E090E0DC019B
:1096100080839183A283B383F901E75BFD4E80834E
:109620009183A283B383F901E75CFD4E2F5D3D4E2C
:10963000E90188819981AA81BB8180839183A2837A
:10964000B383DF91CF911F9108958091171280937A
:10965000280E80E00E94F24A81E00E94F24A0895BA
:109660004F925F926F927F928F929F92AF92BF9232
:10967000CF92DF92EF92FF920F931F93CF93DF93DE
:10968000B82E8091FB0D9091FC0DA091FD0DB09135
:10969000FE0D2091240E3091250E4091260E509102
:1096A000270E7C018D01E21AF30A040B150BA801A9
:1096B0009701243631054105510508F4D9C180933D
:1096C000240E9093250EA093260EB093270E0B2DFB
:1096D00010E0E801C75DD14F8B2D0E94D04A782E53
:1096E0008881871521F08B2D0E94F24A78828DE0C7
:1096F00090E0089FE001099FD00D189FD00D112424
:10970000909117128BE1989FC001112440968C0F05
:109710009D1F61E040E221E00E94F927A82E8823E6
:1097200011F4AA24A394909117128BE1989FC00181
:10973000112444968C0F9D1F40E050E0BA0100E2D6
:109740001EEF2FE63AE40F2EF0E0CF2EF0E8DF2EEA
:10975000FBEBEF2EF5E4FF2EF02D0E9416297B0186
:109760008C012A2D30E0B901882777FD8095982F4C
:109770000E9450A4A80197010E9404A520E030E0B7
:1097800040E752E40E94B5A3A62E172F082F692E9A
:109790008B2C9924E401CC0FDD1FCC0FDD1FFE01C3
:1097A000EF5DFD4EC080D180E280F380E894F7F851
:1097B000772009F435C18091171262E00E949A6601
:1097C00096FF12C08091171265E00E949A6696FF7C
:1097D0000BC0C75BDD4E80E090E0A8ECB2E488836C
:1097E0009983AA83BB8310C0809117126B2D0E94AE
:1097F0006A55F401EE0FFF1FEE0FFF1FE75BFD4EF2
:1098000060837183828393838B2DB701A601F80156
:109810000A2D1F2F2E2F362D0E94254A2B013C0189
:10982000C701B60120E030E040E85FE30E94B1A349
:1098300088232CF460E070E080E89FE3E5C0C70176
:10984000B60120E030E040E251E40E94B1A3882359
:10985000ECF4C701B60120E030E040E85FE30E948D
:109860004CA37B018C0160E070E080E89FE32DEC6D
:109870003CEC4CE45FEB0F2EF0E0AF2EF0E0BF2E9F
:10988000F0E1CF2EF1E4DF2EF02DBCC0C701B60110
:1098900020E030E040E751E40E94B1A388239CF42B
:1098A000C701B60120E030E040E251E40E944CA341
:1098B0007B018C016DEC7CEC8CE49EE320E73EECBC
:1098C00048E05DEB95C0C701B60120E030E040EA1A
:1098D00051E40E94B1A388239CF4C701B60120E0A3
:1098E00030E040E751E40E944CA37B018C0161E32E
:1098F00079E98AE29EE328EB3CEF47E05DEB78C034
:10990000C701B60120E030E048EC51E40E94B1A369
:1099100088239CF4C701B60120E030E040EA51E41E
:109920000E944CA37B018C0163E07AE988E09EE30E
:109930002CEA33E140ED5CEB5BC0C701B60120E0EF
:1099400030E040EF51E40E94B1A388239CF4C701AA
:10995000B60120E030E048EC51E40E944CA37B01CA
:109960008C016BE17FE28DED9DE323E133E840E480
:109970005DEB3EC0C701B60120E030E04CE052E4B0
:109980000E94B1A388239CF4C701B60120E030E017
:1099900040EF51E40E944CA37B018C0163E27BED1C
:1099A00089E79DE324E430E645E65CE321C0C70196
:1099B000B60120E030E040E252E40E94B1A387FD0E
:1099C00005C065E975E688E89DE31EC0C701B601DC
:1099D00020E030E04CE052E40E944CA37B018C017B
:1099E0006AE979E989E99DE328E230EA49E05CEB3C
:1099F0000F2EF0E0AF2EF0E0BF2EF0EACF2EF0E415
:109A0000DF2EF02D0E94A54AE401CC0FDD1FCC0F04
:109A1000DD1FCF5BDD4EA30192010E9404A524C08F
:109A2000809117126B2D0E946A559B01AC0169E46D
:109A3000862E62E1962E8C0E9D1E60E070E088EC12
:109A400092E40E944CA3F401608371838283938328
:109A50008B2DB701A601F8010A2D1F2F2E2F362DB1
:109A60000E94254ACF5BDD4E688379838A839B837E
:109A7000DF91CF911F910F91FF90EF90DF90CF90EA
:109A8000BF90AF909F908F907F906F905F904F901E
:109A900008959091280E80911712981711F00E9446
:109AA000254B809117126EE00E949A6694FF03C0C6
:109AB00080E00E94304B809117126CE00E949A6601
:109AC00094FF03C081E00E94304B0895249A2C9AA1
:109AD000089580E58CBD8DB581608DBD2C9886E0A4
:109AE0000E940D052C9A089580E58CBD8DB581608E
:109AF0008DBD2C9885E00E940D058FEF0E940D050D
:109B00002C9A08951F931FB7F8940E94744D17FF65
:109B100001C078941F9108951F93CF93DF931FB7CF
:109B2000F89480912B0E882381F0C0E0D0E4F89463
:109B30000E94824D80FF02C0219719F410922B0ED3
:109B400004C017FFF4CF7894F2CF812FDF91CF912B
:109B50001F9108950F931F93082F0E948C4D182F6B
:109B60000E94694D80E58CBD8DB581608DBD2C98BE
:109B700081E00E940D05802F0E940D052C9A81E046
:109B800080932B0E17FF01C078941F910F910895B9
:109B9000EF92FF920F931F93DF93CF9300D0CDB737
:109BA000DEB7182F7B014A8399830E948C4D082FC2
:109BB00080E58CBD8DB581608DBD2C9883E00E94C1
:109BC0000D059981892F0E940D05812F0E940D0599
:109BD000C7014A81642F70E00E9413052C9A07FF89
:109BE00001C078940F900F90CF91DF911F910F914A
:109BF000FF90EF900895DF93CF930F92CDB7DEB72C
:109C0000BE016F5F7F4F41E00E94C84D89810F9078
:109C1000CF91DF910895EF92FF921F93DF93CF933F
:109C200000D0CDB7DEB7182F7B014A8399830E94FD
:109C3000694D80E58CBD8DB581608DBD2C9882E02D
:109C40000E940D059981892F0E940D05812F0E9488
:109C50000D05C7014A81642F70E00E9423052C9AEC
:109C600081E080932B0E0F900F90CF91DF911F9189
:109C7000FF90EF900895CF92DF92EF92FF920F93B3
:109C80001F93CF93DF93EC017B01142F80E4D82E38
:109C900020C0CE018F73082F812F90E0800F911D7F
:109CA0008134910514F4012F03C09D2D901B092FC1
:109CB0000E948C4DC82ECE01B701402F0E940B4E42
:109CC000C7FE01C07894C05CDF4FC07CE00EF11C81
:109CD000101B1123F1F6DF91CF911F910F91FF908F
:109CE000EF90DF90CF900895DF93CF930F92CDB791
:109CF000DEB76983BE016F5F7F4F41E00E943B4E3C
:109D00000F90CF91DF91089581E080930E07089521
:109D10001092E900E0EFF0E0808188608083089590
:109D20001F920F920FB60F920BB60F9211242F9322
:109D30003F934F935F936F937F938F939F93AF93D3
:109D4000BF93EF93FF938091F40080FF0CC080914C
:109D5000F4008E7F8093F4000E9474548091E80098
:109D6000877F8093E8008091F40082FF1BC082E02F
:109D70008093E9008091E8008E7F8093E8008091D5
:109D8000F00080FF0FC08091F4008B7F8093F4007F
:109D90006091561270915712809154129091551201
:109DA0000E94AF528091F40081FF35C081E0809322
:109DB000E9008091F00082FF2EC08091F4008D7F39
:109DC0008093F4008091E80085FF25C08091F20027
:109DD0009091F3000097F9F08DE29EE063E171E06D
:109DE0000E9414528823B9F48DE29EE060E47FE083
:109DF0000E948929BC01009771F082E08093E900FC
:109E00008091E80085FF05C080E49FE00E94AF528A
:109E100002C00E946554FF91EF91BF91AF919F9155
:109E20008F917F916F915F914F913F912F910F9003
:109E30000BBE0F900FBE0F901F9018950E94655497
:109E40000895F8940E944453809151121092511237
:109E50007894882319F081E00E9473190895CF93B4
:109E6000DF9380915A12833089F1843030F481304D
:109E700059F0823009F082C060C08A3009F449C0CC
:109E80008B3009F07BC02FC080915912813A09F0C4
:109E900075C0C0E4DFE08DE29EE0BE010E9489292A
:109EA000BC01181619060CF069C08091E800877F84
:109EB0008093E800CE010E94525283E191E0FE01BE
:109EC0009C01119221503040E1F74FC0809159120E
:109ED000813A09F053C08091E800877F8093E800C1
:109EE00080910E0735C080915912813209F046C029
:109EF0008091E800877F8093E80010920E078091A0
:109F00005B1290915C12009789F081E080930E07BC
:109F10000DC080915912813289F58091E800877FC8
:109F20008093E80080915C1280932C0E0E943C523A
:109F30008091E800982F9E7F1CC080915912813A31
:109F4000E9F48091E800877F8093E80080912C0EEF
:109F50008093F1008091E800982F9E7F9093E80015
:109F60008F778093E8000E9447528091E800982FF5
:109F70009B7F9093E8008F778093E800DF91CF91EB
:109F8000089582E061EC46E30E94C25180E00E94A5
:109F9000EC5181E060EC46E30E94C251E0EFF0E05A
:109FA000808184608083089581E00E94EC5108954F
:109FB0009330C1F0943030F4913051F0923009F088
:109FC0003BC00BC0913271F1923209F035C02FC005
:109FD00022E130E08FEB94E033C029E230E081ED04
:109FE00094E02EC0813061F0813028F0823071F031
:109FF000833011F510C08AEF94E0FC01249104C075
:10A000008EEF94E0FC01249130E01AC084E295E0E8
:10A01000FC012491F9CFECE4F5E0249130E083EEEB
:10A0200092E10EC029E030E083EE94E009C024E321
:10A0300030E08BE894E004C020E030E080E090E085
:10A04000FA0191838083C9010895DF93CF9300D0F3
:10A05000CDB7DEB7E9E5F2E18091F100819342E10D
:10A06000E136F407C9F79091591280915A12853060
:10A0700009F474C0863040F48130B9F1813070F059
:10A08000833009F033C131C0883009F4F6C089301B
:10A0900009F413C1863009F029C179C0903821F044
:10A0A000923809F023C108C080915212882311F020
:10A0B00083E011C081E00FC080915D128093E900C0
:10A0C0008091EB0090E025E0969587952A95E1F741
:10A0D00081701092E9009091E800977F9093E800DA
:10A0E0008093F1001092F100D3C0923009F0FEC0CD
:10A0F00090915B12992331F590915D12937009F460
:10A10000F7C09093E9002091EB0020FF1BC0813045
:10A11000A1F48091EB0080618093EB0021E030E0BE
:10A1200002C0220F331F9A95E2F72093EA001092A3
:10A13000EA008091EB00886003C08091EB008062B0
:10A140008093EB001092E9008091E800877F809374
:10A15000E8008091E800982F9E7FA9C0992309F01C
:10A16000C5C08091E800877F8093E8008091E80077
:10A17000982F9E7F9093E8008F778093E8000E944D
:10A180003C5280915B1280688093E300B1C090588C
:10A19000923008F0ABC080915B1290915C1260919C
:10A1A0005D12AE014F5F5F4F0E94D84F009709F4D8
:10A1B0009FC02091E800277F2093E80020915F1244
:10A1C000309160128217930720F49093601280936D
:10A1D0005F1220915B1230915C1280E041C080914F
:10A1E000E80082FD60C08091E80080FFF8CF19C0D0
:10A1F000E981FA8143E02330340731F44191FA8355
:10A20000E9834093F10008C0AF014F5F5F4F5A836D
:10A210004983E491E093F100019790936012809359
:10A220005F1280915F1290916012009739F0409117
:10A23000F2005091F30048305105D0F24091F20005
:10A240005091F30080E04830510509F481E090918D
:10A25000E800492F4E7F4093E8009F779093E800F5
:10A2600040915F12509160124115510509F0BBCF2A
:10A270008823B9F00E943C520BC09038B9F5809108
:10A28000E800877F8093E800809153128093F1006B
:10A290008091E800982F9E7F9093E8008F778093BD
:10A2A000E8000E9447528091E800982F9B7F90938E
:10A2B000E8008F778093E8001BC09923B9F4909150
:10A2C0005B129230A8F48091E800877F8093E800C9
:10A2D000909353128091E800982F9E7F9093E8000E
:10A2E0008F778093E8000E94C14F02C00E942F4FD9
:10A2F0008091E80083FF0AC08091EB008062809328
:10A30000EB008091E800877F8093E8000F900F902A
:10A31000CF91DF9108959C019091E1009B7F9093F4
:10A32000E1008091E80085FD1DC0809158128823CE
:10A3300011F482E008958091EB0085FF02C081E076
:10A3400008958091E10082FFECCF8091E1008B7F46
:10A350008093E1002115310511F483E00895215027
:10A360003040DFCF80E00895AC0128E030E080E0AD
:10A3700003C08F5F220F331F24173507D0F3829558
:10A38000807F08958093E9008091EB008160809345
:10A39000EB001092ED006093EC004093ED00809193
:10A3A000EE00881F8827881F08951092F40080E02F
:10A3B0008093E9001092F0001092E8009091ED0077
:10A3C0009D7F9093ED009091EB009E7F9093EB002A
:10A3D0008F5F873069F7089520915412309155129C
:10A3E0002115310501F19091E9001092551210925A
:10A3F00054121092571210925612882341F081E0A5
:10A400008093E9008091F00084608093F00082E006
:10A410008093E9008091F0008E7F8093F000892F77
:10A4200083708093E90008950F931F93CF93DF9378
:10A430008C01EB0184E690E00E948B518823B9F4F3
:10A44000202F312FF90108C09091E80095FF06C038
:10A450009091F100919321972097B1F79091E800A6
:10A46000292F2B7F2093E8009F779093E800DF91BE
:10A47000CF911F910F91089580E197E22091E8001C
:10A4800020FD04C0009711F00197F8CF089580E1F6
:10A4900097E22091E80022FD04C0009711F0019797
:10A4A000F8CF0895EF92FF920F931F93CF93DF930E
:10A4B000082F192F80915F1290916012E62EE7010C
:10A4C0007E01F72EE7018E159F0508F4EC0180E070
:10A4D00023C00E943C5207C0F80181918F018093F4
:10A4E000F100219739F08091F2009091F3008830CB
:10A4F000910590F32091F2003091F30080E0283034
:10A50000310509F481E09091E800292F2E7F2093F6
:10A51000E8009F779093E800209721F09091E80061
:10A5200092FFD7CF9091E80092FF02C085E010C063
:10A53000882359F00E943C528091E800982F9E7F1A
:10A540009093E8008F778093E8000E94475280E064
:10A55000DF91CF911F910F91FF90EF900895CF92CF
:10A56000DF92EF92FF920F931F93CF93DF938C01B3
:10A57000EB0184E690E00E948B51F82E882309F0CD
:10A5800057C0CC24DD2408C0F80181918F0180934D
:10A59000F1000894C11CD11CCC16DD0620F480917A
:10A5A000E80085FDF1CFC114D10411F00E948E9511
:10A5B0008091F4008B7F8093F4008091E800982FC5
:10A5C0009E7F9093E8008F778093E800CC19DD0997
:10A5D00049F4C114D10461F1FFE3CF22DD24C11499
:10A5E000D10431F580E290E00E948B51E82E88235F
:10A5F00041F283E0E816C9F4109355120093541207
:10A60000D0935712C093561281E08093E900809155
:10A61000F0008B7F8093F00082E08093E9008091CE
:10A62000F00081608093F00008C00E94655401C072
:10A63000EF2C81E00E94EC51FE2C8F2DDF91CF9109
:10A640001F910F91FF90EF90DF90CF9008950E949F
:10A65000D44FE0EEF0E0808181608083E8EDF0E0AF
:10A6600080818062808319BCE7EDF0E080818E7F7D
:10A6700080831092581208950E94F65381E08093CF
:10A6800058120E94844E08958091D9008170909153
:10A690005812992329F4882319F00E943C530895F5
:10A6A00090915812992321F0882311F40E94275386
:10A6B00008951F920F920FB60F920BB60F921124AE
:10A6C0002F933F934F935F936F937F938F939F93BA
:10A6D000AF93BF93EF93FF938091DA0080FF0BC09D
:10A6E0008091D80080FF07C08091DA008E7F809330
:10A6F000DA000E9444538091E10080FF19C08091EC
:10A70000E20080FF15C08091E1008E7F8093E10020
:10A710008091E2008E7F8093E2008091E200806170
:10A720008093E2008091D80080628093D80019BCA9
:10A730008091E10084FF20C08091E20084FF1CC072
:10A740008CE089BD89B5826089BD09B400FEFDCF6A
:10A750008091D8008F7D8093D8008091E1008F7E1A
:10A760008093E1008091E2008F7E8093E2008091EF
:10A77000E20081608093E2008091E10083FF23C0CA
:10A780008091E20083FF1FC08091E100877F80936A
:10A79000E100109253128091E1008E7F8093E100DE
:10A7A0008091E2008E7F8093E2008091E2008061E0
:10A7B0008093E2000E94D55180E060E042E00E9478
:10A7C000C2510E94884EFF91EF91BF91AF919F912E
:10A7D0008F917F916F915F914F913F912F910F904A
:10A7E0000BBE0F900FBE0F901F9018958091D80050
:10A7F0008C7F8093D8001092E2001092DA001092C1
:10A80000E10010925812109253121092521280E0EE
:10A810000E94EC518CE089BD89B5826089BD09B484
:10A8200000FEFDCF8091D800982F9F779093D8009D
:10A8300080688093D8008091D70081608093D70092
:10A840008091D8008F7D8093D8008091E0008B7F2D
:10A850008093E0008091D80081608093D80080913F
:10A86000E0008E7F8093E0008091E2008160809321
:10A87000E2008091E20088608093E2000895809178
:10A880005812882311F00E94D44F8091E00081601B
:10A890008093E0008091D8008C7F8093D800109244
:10A8A000E2001092DA001092E10010925812109219
:10A8B00053128091D8008F778093D80019BC809173
:10A8C000D8008F7E8093D80008950E943F54E7ED12
:10A8D000F0E08081806880830E94F653E8EDF0E02C
:10A8E00080818061808308950F931F938091581217
:10A8F000882381F01091E9001092E9008091E8002E
:10A9000083FF05C00FB7F8940E9425500FBF137046
:10A910001093E9001F910F910895EF92FF920F930A
:10A920001F9390E0880F991F860F911DFC01EE0F79
:10A93000FF1FEE0FFF1FED5AFF4EE080F1800281F6
:10A940001381FA01E082F1820283138389549F4EBE
:10A95000FC018081F90180831F910F91FF90EF909E
:10A9600008959BE1899FC001112440962DE0629FCC
:10A97000B0011124860F971F61E040E221E00E94A0
:10A98000F927882309F481E00895AF92BF92CF920E
:10A99000DF92EF92FF920F931F93B82EA62E2BE11A
:10A9A000829F900111242C5E3F4F8DE0689FC00173
:10A9B0001124820F931F40E050E0BA0100E21EEF25
:10A9C0002FE63AE40F2EF0E0CF2EF0E8DF2EFBEB7F
:10A9D000EF2EF5E4FF2EF02D0E9416297B018C014D
:10A9E0008B2D6A2D0E94B154282F30E0B9018827A1
:10A9F00077FD8095982F0E9450A49B01AC01C8015F
:10AA0000B7010E9404A51F910F91FF90EF90DF9076
:10AA1000CF90BF90AF900895BF92CF92DF92EF9208
:10AA2000FF920F931F93082F162F0E94B154B82E38
:10AA30002BE1029F900111242C5E3F4F8DE0189F67
:10AA4000C0011124820F931F40E050E0BA0100E2E0
:10AA50001EEF2FE63AE40F2EF0E0CF2EF0E8DF2EC7
:10AA6000FBEBEF2EF5E4FF2EF02D0E9416297B0163
:10AA70008C0120E030E040E752E40E94B1A387FD62
:10AA80000AC0C801B70120E030E64AEE56E40E9451
:10AA900000A5181654F40F2EF0E0EF2EF0E8FF2E6C
:10AAA000FBEB0F2FF5E41F2FF02D2B2D30E0B9011C
:10AAB000882777FD8095982F0E9450A4A8019701C0
:10AAC0000E9404A51F910F91FF90EF90DF90CF900F
:10AAD000BF900895EF92FF920F931F93E82FF0E03D
:10AAE000EE0FFF1FE60FF11DEE0FFF1FEE0FFF1F12
:10AAF000EF59FD4EE080F180028113810E940C55D8
:10AB00009B01AC01C801B7010E94B5A37B018C0178
:10AB1000802F880F812F881F8F3F09F1C801B7014F
:10AB200020E030E0A9010E94B1A387FD18C0C80150
:10AB3000B70120E030E040E85FE30E9400A518166E
:10AB40002CF460E070E088EC92E40DC0C801B7011D
:10AB500020E030E048EC52E40E9404A504C060E02C
:10AB600070E080E090E01F910F91FF90EF900895CA
:10AB7000AF92BF92CF92DF92EF92FF920F931F930B
:10AB8000DF93CF9300D000D0CDB7DEB7082F162FBC
:10AB900080911B127E010894E11CF11C8330F9F0B6
:10ABA00080E090E0DC0189839A83AB83BC836BE116
:10ABB000069FB0011124685E7F4F8DE01802C0012E
:10ABC0001124680F791FC7010E944E2880E090E889
:10ABD000ABE3B5E489839A83AB83BC8326C0802F23
:10ABE0000E94E75C5B016C01802F612F0E940C5575
:10ABF000A60195010E9404A520E030E048EC52E453
:10AC00000E94B5A369837A838B839C836BE1069F43
:10AC1000B0011124685E7F4F8DE01802C00111243D
:10AC2000680F791FC7010E944E2859814A813B81D4
:10AC30002C81652F742F832F922F0F900F900F90E0
:10AC40000F90CF91DF911F910F91FF90EF90DF90C8
:10AC5000CF90BF90AF9008950F931F93CF93DF9342
:10AC6000082F10E0C62FDD27C7FDD0950E94B855EC
:10AC70009B01AC01000F111F0C0F1D1FC801880F95
:10AC8000991F880F991FFC01EF59FD4E20833183D6
:10AC9000428353838D5A9F4EFC011082118212828F
:10ACA000138209541F4EF8011082DF91CF911F913A
:10ACB0000F9108952F923F924F925F926F927F92E1
:10ACC0008F929F92AF92BF92CF92DF92EF92FF92BC
:10ACD0000F931F93DF93CF93CDB7DEB72A970FB6AD
:10ACE000F894DEBF0FBECDBF8D836E834A0139015C
:10ACF00017012801AF82B886C986DA86FA01E0809A
:10AD0000F18002811381F9016081718182819381D7
:10AD1000A80197010E944CA3D62EC72EB82EA92EAB
:10AD2000C201B101D601F5012B2F3A2F4F2F5E2F13
:10AD30000E9404A59B01AC01C801B7010E944DA36C
:10AD4000F40160837183828393836F817885898521
:10AD50009A85D601F5012B2F3A2F4F2F5E2F0E9497
:10AD600004A59B01AC01C801B7010E944DA3B62EFA
:10AD7000C72ED82EE92E862F9C2DAD2DBE2DF3018A
:10AD800080839183A283B3838D816E810E94B154AD
:10AD9000282F30E0B901882777FD8095982F0E94F1
:10ADA00050A49B01AC016B2D7C2D8D2D9E2D0E94FE
:10ADB000B5A369837A838B839C836BE1FD81F69FC6
:10ADC000B00111246C5E7F4F8DE02E81289FC00161
:10ADD0001124680F791FCE0101960E9453282A96EC
:10ADE0000FB6F894DEBF0FBECDBFCF91DF911F919C
:10ADF0000F91FF90EF90DF90CF90BF90AF909F901A
:10AE00008F907F906F905F904F903F902F9008951C
:10AE10002F923F924F925F926F927F928F929F926A
:10AE2000AF92BF92CF92DF92EF92FF920F931F9358
:10AE3000DF93CF93CDB7DEB72E970FB6F894DEBF72
:10AE40000FBECDBFA82EB62E442E882E9924662381
:10AE5000E9F4C0909504D0909604E0909704F090A7
:10AE6000980486EA92E040E050E068E472EC00E08A
:10AE700010E028E432E40E9416297B018C01F401E1
:10AE800023E0EE0FFF1F2A95E1F71FC0C090990441
:10AE9000D0909A04E0909B04F0909C048AEA92E09F
:10AEA00040E050E068E472EC00E010E028E432E4B6
:10AEB0000E9416297B018C01F401EE0FFF1FEB0DA0
:10AEC000F11DEE0FFF1FEE0FFF1FED5AFF4E6081C9
:10AED0007181828193810E9450A49B01AC01C801C1
:10AEE000B7010E9404A5962EC72ED82EE92E642DF8
:10AEF00070E080E090E00E944EA49B01AC01692DBF
:10AF00007C2D8D2D9E2D0E94B5A3D62EC72E982E5A
:10AF1000892E2A2C33242B2D30E03A872987C10132
:10AF2000880F991F820F931F9C01220F331F220F3E
:10AF3000331FF901ED5AFF4E1082118212821382E3
:10AF400089549F4EDC011C922F593D4EF9016081BE
:10AF5000718182819381D601F4012B2F3A2F4F2FDB
:10AF60005E2F0E944CA3262F372F482F592F29835D
:10AF70003A834B835C8320E030E0A9010E94B1A3B7
:10AF800088233CF480E090E0DC0189839A83AB83E2
:10AF9000BC838A2D6B2D0E940C552B013C016D83C7
:10AFA0007E838F8398878A2D6B2D0E94E75C7B01BF
:10AFB0008C01A6019401652F7C2D832F982D20E014
:10AFC00030E040E050E40E94B1A388230CF04BC075
:10AFD00089819A81AB81BC818B879C87AD87BE8735
:10AFE000C301B2012FE832EC45EF5CE30E9404A5F7
:10AFF0009B01AC016B857C858D859E850E94B1A3EC
:10B000001816CCF0C801B70120E030E040E450E46D
:10B010000E94B1A318163CF5C801B7012D813E81ED
:10B020004F8158850E9404A520E030E048EC52E4AE
:10B030000E94B5A314C0C801B70120E030E040E48D
:10B0400050E40E94B1A3181674F06B857C858D8541
:10B050009E852DEC3CEC4CE45FE30E9404A56983E3
:10B060007A838B839C8369817A818B819C812D81FA
:10B070003E814F8158850E9400A5181654F5C801DD
:10B08000B70120E030E042EC52E40E9400A59E01AE
:10B090002B5F3F4FAE014F5F5F4F88231CF08A2D1F
:10B0A0006B2D37C08A2D6B2D0F2EF6E6EF2EF6E6B0
:10B0B000FF2EF6EE0F2FFEE31F2FF02D0F2EF3E3E2
:10B0C000AF2EF3E3BF2EF3E7CF2EFFE3DF2EF02DFD
:10B0D00034C0A6019401652F7C2D832F982D20E08C
:10B0E00030E040E050EC0E9400A5181644F5C8017D
:10B0F000B70120E030E042EC52E40E9400A5882332
:10B10000F4F08A2D6B2DAE014F5F5F4F9E012B5FD8
:10B110003F4F0F2EFDECEF2EFCECFF2EFCE40F2F2B
:10B12000FEE31F2FF02D0F2EFDECAF2EFCECBF2EFB
:10B13000FCE4CF2EFFE3DF2EF02D0E945A56F101E2
:10B14000EE0FFF1FA985BA85EA0FFB1FEE0FFF1F49
:10B15000EE0FFF1FEF59FD4E89819A81AB81BC81B3
:10B1600080839183A283B3832E960FB6F894DEBFBB
:10B170000FBECDBFCF91DF911F910F91FF90EF9048
:10B18000DF90CF90BF90AF909F908F907F906F9007
:10B190005F904F903F902F9008954F925F927F92D3
:10B1A0008F929F92AF92BF92CF92DF92EF92FF92D7
:10B1B0000F931F93DF93CF930F92CDB7DEB78230FB
:10B1C00050F451E6E52E52E1F52E48E1842E912C03
:10B1D000442455242EC08430C1F5F3CFF80180817A
:10B1E000882359F0872D622F4CE329830E9408574A
:10B1F000C601B5010E944E2829812F5F0F5F1F4FA6
:10B2000084E090E0C80ED91EEDE0F0E0AE0EBF1E67
:10B21000223021F70894411C511C88E090E0E80E90
:10B22000F91EEBE1F0E08E0E9F1EFCE04F1651047C
:10B2300051F0742C8201000F111F09541F4E54014C
:10B24000670120E0CBCF1092D1100F90CF91DF910A
:10B250001F910F91FF90EF90DF90CF90BF90AF9034
:10B260009F908F907F905F904F9008958091D11024
:10B27000882309F580911B128330E9F486E79AE56B
:10B2800060E070E00E948B5C8091FB0D9091FC0D62
:10B29000A091FD0DB091FE0D8093B3109093B4106A
:10B2A000A093B510B093B6101092CF101092D0109A
:10B2B00081E08093D11008955F926F927F928F9278
:10B2C0009F92AF92BF92CF92DF92EF92FF920F9335
:10B2D0001F93CF93DF938091FB0D9091FC0DA09174
:10B2E000FD0DB091FE0D2091B3103091B41040913E
:10B2F000B5105091B6107C018D01E21AF30A040BCF
:10B30000150BA8019701243631054105510508F4B4
:10B3100068C08093B3109093B410A093B510B0930D
:10B32000B6100E9436598091D110882309F459C073
:10B3300081E09AE560E070E00E948B5C8091CF1024
:10B340008F5F8093CF108C3308F44BC01092CF10D6
:10B350008091D0108F5F8093D010893610F4EE2446
:10B3600004C01092D010EE24E394E1E6CE2EE2E188
:10B37000DE2E78E1672E712CC0E0D0E028C0F80105
:10B380004081442351F0852D6F2D0E940857EE20F7
:10B3900021F0C501B4010E944E28F3940F5F1F4FA6
:10B3A00084E090E0A80EB91EEDE0F0E08E0E9F1E46
:10B3B000F2E0FF1621F7219608E010E0C00ED11E42
:10B3C0008BE190E0680E791ECC30D10551F05C2EF7
:10B3D0008E01000F111F09541F4E43015601FF2417
:10B3E000CECFDF91CF911F910F91FF90EF90DF9023
:10B3F000CF90BF90AF909F908F907F906F905F9015
:10B400000895AF92BF92CF92DF92EF92FF921F9377
:10B41000CF93DF93182F662319F421E030E05BC04F
:10B420006EE00E949A6694FF26C0E12EFF24E70199
:10B4300083E0CC0FDD1F8A95E1F7CD5ADF4EA8805F
:10B44000B980CA80DB80812F65E00E948D67AA27C2
:10B4500097FDA095BA2F8A0D9B1DAC1DBD1D88833D
:10B460009983AA83BB83F701EE0FFF1FE954FF4EB8
:10B4700080818F5F8083812F6CE00E949A6694FFA9
:10B4800028C0C12FD0E0CC0FDD1F7E01EE0CFF1CC9
:10B49000EE0CFF1C87E590E1E80EF91EF701A08095
:10B4A000B180C280D380812F62E00E948D67AA277D
:10B4B00097FDA095BA2F8A0D9B1DAC1DBD1DF701F0
:10B4C00080839183A283B383C954DF4E89818F5FC8
:10B4D000898320E030E0C901DF91CF911F91FF9077
:10B4E000EF90DF90CF90BF90AF9008955F926F92F2
:10B4F0007F928F929F92AF92BF92CF92DF92EF9204
:10B50000FF920F931F93CF93DF93A82E562E8BE1BC
:10B510009A2D989FE00111246896CA2CDD24C6015B
:10B5200043E0880F991F4A95E1F731E6832E32E117
:10B53000932E880E991E23E5622E20E1722E680E4E
:10B54000791ECC0CDD1CE7EBF0E1CE0EDF1EBB2438
:10B55000CE010E94D6287B018C0120E030E040E73C
:10B5600052E40E94B1A387FD0AC0C801B70120E0E0
:10B5700030E64AEE56E40E9400A518169CF45520C9
:10B5800059F40F2EF0E0EF2EF0E8FF2EFBE30F2F23
:10B59000F5E41F2FF02D06C08A2D6B2D0E94B855A3
:10B5A0007B018C01F401E192F192019311934F011F
:10B5B000F30111921192119211923F01F601119231
:10B5C0006F01B3942D96F2E0BF1611F680E090E083
:10B5D000DF91CF911F910F91FF90EF90DF90CF906F
:10B5E000BF90AF909F908F907F906F905F900895E5
:10B5F0008FEF8093C1128FE78093C2128093C312A2
:10B600000895FC018FEF80838FE781838283089503
:10B61000CF93DF93C82FD0E0CC57DF4F84E0CC0F1F
:10B62000DD1F8A95E1F7CE0182579F4F0E94A264E9
:10B63000292F22952F7030E02230310511F090E053
:10B640000AC0CE018A579D4F0E94A26490E08F707D
:10B650008F3009F091E0892FDF91CF91089590917B
:10B660001B12923010F480E0089590E024E0880FDF
:10B67000991F2A95E1F78A53954F0E94A264892F5A
:10B68000911181E008951F93CF93DF93C4ECDAE02A
:10B6900010E080E00E942F5B882371F0CE010E94B1
:10B6A000A26484FF09C0812F0E94085B882329F0CF
:10B6B0001F5F6096123069F781E0DF91CF911F9193
:10B6C00008950F931F93CF93DF93082F0E94435B3E
:10B6D0008823D9F010E015C0812F60E80E949A6697
:10B6E000EC01812F63E80E949A66C070DE702EE044
:10B6F000C030D20729F48F7090708F30910529F0F7
:10B700001F5F101748F381E001C080E0DF91CF9107
:10B710001F910F91089590E034E0880F991F3A959A
:10B72000E1F78C53954F0E94A26485FD02C081E031
:10B7300008958CE00E94615B811181E00895CF92B1
:10B74000DF92EF92FF920F931F93CF93DF93EC0161
:10B750007B0180E00E948B5B882341F080E00E94A7
:10B760002F5B882319F081E090E002C080E090E038
:10B77000182F00E0802F612FA701FE0109956C01B1
:10B780001123E1F00097C9F40023B9F480E00E948E
:10B79000085B182F882391F081E00E948B5B88233F
:10B7A00041F081E00E942F5B882319F081E090E056
:10B7B00002C080E090E0182F01C011E00F5F02305E
:10B7C00019F0C114D104B1F2C601DF91CF911F91DC
:10B7D0000F91FF90EF90DF90CF900895CF92DF927E
:10B7E000EF92FF921F93CF93DF93182FEB0160E846
:10B7F0000E949A666C01812F61E80E949A667C0122
:10B80000812F63E80E949A669883960165E03695D9
:10B8100027956A95E1F72077382F3F70232B2983EE
:10B8200054E0969587955A95E1F78F70970145E01A
:10B83000369527954A95E1F7922F9077892B8A8341
:10B84000DF91CF911F91FF90EF90DF90CF900895FF
:10B85000EF92FF920F931F938091FB0D9091FC0D3F
:10B86000A091FD0DB091FE0D2091D2103091D3101A
:10B870004091D4105091D5107C018D01E21AF30A49
:10B88000040B150BA80197012B303105410551051B
:10B89000E8F08093D2109093D310A093D410B0937B
:10B8A000D510809117120E94615B882349F48FEFB5
:10B8B0008093C1128FE78093C2128093C31206C097
:10B8C0008091171261EC72E10E94EE5B1F910F9163
:10B8D000FF90EF9008951F93182F80911B128230D4
:10B8E000B8F0812F6FE00E948966009789F0812F60
:10B8F00067E80E949A66009759F0812F61E80E94DC
:10B900009A6680E092959F70191719F481E001C042
:10B9100080E01F9108958F929F92AF92BF92CF9235
:10B92000DF92EF92FF920F931F93DF93CF9300D09C
:10B930000F92CDB7DEB76C015B010E94435B882399
:10B9400041F080E00E946B5C882319F001E010E078
:10B9500002C000E010E010E07E010894E11CF11C40
:10B96000812F602FA501F60109954C010023C1F03C
:10B970000097B1F41B30A1F0812F60E80E949A6615
:10B9800097FF0DC0812FB7010E94EE5B8A818F3730
:10B9900030F4812F8F5F0E946B5C082F01C000E0A4
:10B9A0001F5F1C3019F081149104D1F2C4010F9073
:10B9B0000F900F90CF91DF911F910F91FF90EF901B
:10B9C000DF90CF90BF90AF909F908F9008952F926F
:10B9D0003F924F925F926F927F928F929F92AF921F
:10B9E000BF92CF92DF92EF92FF920F931F93DF935C
:10B9F000CF9300D000D0CDB7DEB7182F062F662327
:10BA000081F46EE00E949A6694FF3CC1812F90E021
:10BA10000E9487676B017C01812F90E00E94D367B1
:10BA20000FC06CE00E949A6694FF2CC1812F90E0B9
:10BA30000E9481676B017C01812F90E00E94CD679D
:10BA40002B013C012BE1129F900111242F5E3F4FEF
:10BA50008DE0089FC0011124820F931F6CE044E227
:10BA60002CE00E94F927082FC701B60120E030E042
:10BA700040E151E40E94B1A388230CF41EC1C70128
:10BA8000B60120E030E048E851E40E94B1A38823E9
:10BA900014F411E00FC0C701B60120E030E040EF20
:10BAA00051E40E94B1A3182F111F1127111F83E029
:10BAB000811B182F083189F0043219F00C30C1F5C0
:10BAC00022C0C701B60120E030E048ED51E40E94F9
:10BAD00000A588236CF113E02BC0C701B60120E05C
:10BAE00030E040E951E40E9400A588230CF1C70131
:10BAF000B60120E030E040EE51E40E94B1A31816F8
:10BB0000BCF012E015C0C701B60120E030E040E112
:10BB100051E40E9400A588235CF0C701B60120E033
:10BB200030E040E651E40E94B1A318160CF011E099
:10BB3000212F30E0B901882777FD8095982F0E944A
:10BB400050A44B015C01C701B601A50194010E94FC
:10BB5000B5A3062F372E282E9983C301B2019F77F4
:10BB6000A50194010E94B5A3862EA72EC82E192FD9
:10BB70002DEC3CEC40E051E40E9400A588232CF021
:10BB80008FE097E09C838B8315C0682D7A2D8C2DD8
:10BB9000912F20E030E048EB50E40E9400A587FFA1
:10BBA00005C0A7E6B7E0BC83AB8304C0EBE3F7E0D6
:10BBB000FC83EB838B809C80AA24BB2414E6D401F5
:10BBC000CD90DD90ED90FC90C701B6017980202FDB
:10BBD000332D422D572D0E94B1A318160CF447C0E7
:10BBE000AA2029F460E070E088EC92E44FC0612F55
:10BBF00070E080E090E00E944EA4162F872E982ED1
:10BC00009A83C701B601A1013981402E552E642EB9
:10BC1000732EA30192010E944CA320E030E040E289
:10BC200051E40E9404A52B013C01F5013197EE0F70
:10BC3000FF1FEE0FFF1F8B819C81E80FF91FC701CB
:10BC4000B60120813181428153810E944CA39B0126
:10BC5000AC01C301B2010E94B5A39B01AC01CA8033
:10BC6000612F782D892D9C2D0E944DA30FC0089423
:10BC7000A11CB11CA4E0B0E08A0E9B1E112311F0A0
:10BC80001A509DCF60E070E080E090E00F900F9040
:10BC90000F900F90CF91DF911F910F91FF90EF9038
:10BCA000DF90CF90BF90AF909F908F907F906F90DC
:10BCB0005F904F903F902F90089510E0FBCE8091C1
:10BCC0001C12813039F480919011882319F0109260
:10BCD0001C1208950E94BC05089580911C128823AF
:10BCE00041F480919111882321F081E080931C120E
:10BCF00008950E94BC0508958091171260911C124E
:10BD00000E942C5608958091171280938F116EE037
:10BD10000E949A669295917090939011809117125B
:10BD20006CE00E949A66929591709093911199237C
:10BD300021F080919011882319F010921C1208951F
:10BD400081E080931C120895AF92BF92CF92DF9250
:10BD5000EF92FF920F931F93DF93CF9300D000D009
:10BD600000D0CDB7DEB79091171280918F11981740
:10BD700011F00E94835E8AE060E00E949F04E091DF
:10BD80001C12F0E0EE0FFF1FE157FE4E83819481FD
:10BD90000E944B0682E160E00E949F04809117128E
:10BDA00090E0019663E977E042E00E944E0684E06D
:10BDB00060E00E949F0460911C12E62FF0E0E157C2
:10BDC000FE4E8181882309F457C0809117120E948A
:10BDD000C55420E030E040E752E40E94B5A38B0157
:10BDE000B82EA92E9501712F832F922F48E957E085
:10BDF00026E00E94930684E061E00E949F04809107
:10BE00001C12E0911712F0E0EE0FFF1FE80FF11D7A
:10BE1000EE0FFF1FEE0FFF1FEF59FD4E6081718186
:10BE20008281938120E030E040E752E40E94B5A394
:10BE30006B017C017D2D9F2D48E957E026E00E9493
:10BE400093068BE061E00E949F046C2D7D2D8E2D6A
:10BE50009F2D20E030E048EC52E40E9404A5F5015B
:10BE6000202F312F4F2F5E2F0E94B5A34EE957E0B0
:10BE700025E00E94930614C087E392E00E944B06DF
:10BE800084E061E00E949F0487E392E00E944B06F9
:10BE90008BE061E00E949F0488E392E00E944B06E1
:10BEA00090911C1280911712992349F40E94D36734
:10BEB0007B018C01C0909611D090971109C090E041
:10BEC0000E94CD677B018C01C0909811D090991190
:10BED00080E062E00E949F04C6010E944B0684E05D
:10BEE00062E00E949F04E0911C12F0E0E157FE4ED8
:10BEF0008181882309F470C0C801B70148E957E07F
:10BF000026E00E9493068EE062E00E949F048091EA
:10BF1000171260911C120E94E75C4EE957E025E081
:10BF20000E9493068091171260911C12AE014E5F21
:10BF30005F4F9E012F5F3F4F0E948D5480911C12D6
:10BF4000882359F4C0909504D0909604E09097040B
:10BF5000F090980486EA92E00AC0C0909904D090CC
:10BF60009A04E0909B04F0909C048AEA92E040E0FE
:10BF700050E068E472EC00E010E028E432E40E9453
:10BF800016297B018C016A817B818C819D810E94B5
:10BF900050A49B01AC01C801B7010E9404A5F62E74
:10BFA000072F182F84E063E09E830E949F049E81E8
:10BFB0006F2D702F812F48E957E026E00E949306ED
:10BFC0008BE063E00E949F04898190E064EA77E05F
:10BFD00042E00E944E061CC087E392E00E944B069E
:10BFE0008EE062E00E949F0488E392E00E944B068C
:10BFF00084E063E00E949F0487E392E00E944B0686
:10C000008BE063E00E949F048BE392E00E944B066A
:10C0100026960FB6F894DEBF0FBECDBFCF91DF914D
:10C020001F910F91FF90EF90DF90CF90BF90AF9056
:10C030000895CF92DF92EF92FF920F931F93CF93C9
:10C04000DF9384EF91E00E9489050E94835ECAE736
:10C05000D1E1CE0160E270E044E150E00E9471A7BE
:10C060008EE40E945E12BC01FC0101900020E9F701
:10C070003197E81BF90BCE01AF010E9468A74AE394
:10C08000F42EF0927D118FE30E945E12BC01FC0140
:10C0900001900020E9F73197E81BF90B8E01015F51
:10C0A0001F4FC801AF010E9468A780E090E00E9486
:10C0B0003906CE0160E270E044E150E00E9471A7D1
:10C0C00085E70E945E12BC01FC0101900020E9F7A7
:10C0D0003197E81BF90BCE01AF010E9468A7F092DF
:10C0E0007D1135E2E32EE0928A1181E090E00E941A
:10C0F0003906CE0160E270E044E150E00E9471A791
:10C10000F0927D1181E480938411E0928D1182E0A0
:10C1100090E00E943906CE0160E270E044E150E018
:10C120000E9471A784E70E945E12BC01FC0101908D
:10C130000020E9F73197E81BF90BCE01AF010E940F
:10C1400068A7F0927D1184E20E945E12BC01FC019E
:10C1500001900020E9F73197E81BF90BC801AF0106
:10C160000E9468A783E090E00E94390687E80E9459
:10C170005E12909393118093921188E80E945E1250
:10C18000909395118093941185E30E945E12909391
:10C1900097118093961186E30E945E1290939911F5
:10C1A000809398110E94A45EDF91CF911F910F910F
:10C1B000FF90EF90DF90CF900895E8ECF7E008C093
:10C1C000208131812817390711F46283089533964D
:10C1D00027E0EA3DF207A1F708956093D71091E0B8
:10C1E0009093D61083FD02C090E401C090E6877062
:10C1F000892B98E10FB6F894A895909360000FBE34
:10C200008093600078944111FFCF08951F93CF93DE
:10C21000DF93182FC0ECD7E004C0E991F991812F8A
:10C22000099587E0C83CD807C1F7DF91CF911F91EE
:10C2300008958091D610882319F4A8950E94B59589
:10C2400008950F931F93CF93DF9384B78093E212E7
:10C2500098E10FB6F89490936000109260000FBEC2
:10C2600020E090E80FB6F89490936100209361006D
:10C270000FBE80FF06C08FE493EC0197F1F700C07A
:10C28000000018E101E60FB6F894A895109360003D
:10C290000FBE0093600078940E9409620E9400051E
:10C2A0000E949C170E941E4F0E94664D8CE00E94C7
:10C2B0003F048FE39DE0A3E081509040A040E1F770
:10C2C00000C000008CE00E943F040E94CB270E9427
:10C2D000A0090E94D8360E94ED690E942C130E948A
:10C2E00007090E944D8D0E946D95129A129A14BEF4
:10C2F00078948CE591E161EF72E04EE150E00E94AC
:10C3000058280FB6F894A895109360000FBE0093BC
:10C3100060007894C8ECD7E007C08A81813019F4B6
:10C32000E881F9810995239697E0CA3DD907A9F7D5
:10C330000E94196182B1847082B98BB184708BB90B
:10C340006297F2CF1F920F920FB60F920BB60F9219
:10C3500011242F933F934F935F936F937F938F930A
:10C360009F93AF93BF93CF93DF93EF93FF9381E0BE
:10C370000E9406618091D710882319F4C0E0D0E0B4
:10C3800008C083E094E065E570E00E940468C0E0C6
:10C39000D0EF84B7877F84BF88E10FB6F89480938D
:10C3A0006000109260000FBE0E94BB170E943F54B5
:10C3B0008FE39DE0A3E081509040A040E1F700C0F2
:10C3C0000000FE01099583FD03C020E030E002C0BB
:10C3D00020E038E0613069F4B90160507E4F43FFDE
:10C3E00003C0B90160587D4F47705070462B572BE2
:10C3F00004C04F785070422B532B9C012770307033
:10C4000084E0220F331F8A95E1F7242B352BC901D5
:10C410000895209A2898089588E58CBD8DB581608F
:10C420008DBD289A089528980895CF92DF92EF92B3
:10C43000FF920F931F93CF93DF93EC01C0909D0465
:10C44000D0909E04E0909F04F090A0048EEA92E0C9
:10C4500040E050E068E472EC00E010E028E432E4F0
:10C460000E9416296B017C01DF70BE0180E090E024
:10C470000E944EA4A70196010E9404A5DF91CF91CE
:10C480001F910F91FF90EF90DF90CF900895CF9282
:10C49000DF92EF92FF920F931F93CF93DF93EC0104
:10C4A000C0909904D0909A04E0909B04F0909C0472
:10C4B0008AEA92E040E050E068E472EC00E010E0CC
:10C4C00028E432E40E9416296B017C01BE01882712
:10C4D00077FD8095982F0E9450A49B01AC01C70165
:10C4E000B6010E9404A5DF91CF911F910F91FF909B
:10C4F000EF90DF90CF900895CF92DF92EF92FF926E
:10C500000F931F93CF93DF93EC01C0909504D090CD
:10C510009604E0909704F090980486EA92E040E058
:10C5200050E068E472EC00E010E028E432E40E949D
:10C5300016296B017C01BE01882777FD8095982F15
:10C540000E9450A49B01AC01C701B6010E9404A542
:10C55000DF91CF911F910F91FF90EF90DF90CF90DF
:10C560000895CF92DF92EF92FF920F931F93CF9394
:10C57000DF93EC01C0909104D0909204E09093047A
:10C58000F090940482EA92E040E050E068E472ECBB
:10C5900000E010E028E432E40E9416296B017C01DF
:10C5A000DF70BE0180E090E00E944EA4A7019601DA
:10C5B0000E9404A5DF91CF911F910F91FF90EF9002
:10C5C000DF90CF900895CF92DF92EF92FF920F937A
:10C5D0001F93CF93DF93EC01C0908D04D0908E0415
:10C5E000E0908F04F09090048EE992E040E050E0FB
:10C5F00068E472EC00E010E028E432E40E941629BE
:10C600006B017C01DF70BE0180E090E00E944EA4CF
:10C61000A70196010E9404A5DF91CF911F910F9170
:10C62000FF90EF90DF90CF9008958F929F92AF92FE
:10C63000BF92CF92DF92EF92FF920F931F934B0125
:10C640005C0120E030E0A9010E94B1A388231CF422
:10C6500060E070E02BC0C501B40120E030EF4FE78F
:10C6600055E40E9400A518161CF46FEF7FE01EC071
:10C67000C0909D04D0909E04E0909F04F090A00490
:10C680008EEA92E040E050E068E472EC00E010E0F6
:10C6900028E432E40E9416299B01AC01C501B401D3
:10C6A0000E94B5A30E9467A50E9422A4CB011F91FE
:10C6B0000F91FF90EF90DF90CF90BF90AF909F9041
:10C6C0008F9008958F929F92AF92BF92CF92DF92F8
:10C6D000EF92FF920F931F934B015C01C09099045E
:10C6E000D0909A04E0909B04F0909C048AEA92E037
:10C6F00040E050E068E472EC00E010E028E432E44E
:10C700000E9416299B01AC01C501B4010E94B5A38A
:10C710000E9467A50E941DA4CB011F910F91FF905D
:10C72000EF90DF90CF90BF90AF909F908F90089543
:10C730008F929F92AF92BF92CF92DF92EF92FF9231
:10C740000F931F934B015C01C0909504D090960409
:10C75000E0909704F090980486EA92E040E050E080
:10C7600068E472EC00E010E028E432E40E9416294C
:10C770009B01AC01C501B4010E94B5A30E9467A54D
:10C780000E941DA4CB011F910F91FF90EF90DF90AD
:10C79000CF90BF90AF909F908F9008958F929F926F
:10C7A000AF92BF92CF92DF92EF92FF920F931F93BF
:10C7B0004B015C0120E030E0A9010E94B1A31816F2
:10C7C0001CF060E070E02BC0C501B40120E030EF48
:10C7D0004FE755E40E9400A588231CF06FEF7FE02F
:10C7E0001EC0C0909104D0909204E0909304F09009
:10C7F000940482EA92E040E050E068E472EC00E0E9
:10C8000010E028E432E40E9416299B01AC01C50126
:10C81000B4010E94B5A30E9467A50E9422A4CB0187
:10C820001F910F91FF90EF90DF90CF90BF90AF904E
:10C830009F908F9008958F929F92AF92BF92CF92C8
:10C84000DF92EF92FF920F931F934B015C0120E068
:10C8500030E0A9010E94B1A318161CF060E070E05E
:10C860002BC0C501B40120E030EF4FE755E40E9432
:10C8700000A588231CF06FEF7FE01EC0C0908D04E0
:10C88000D0908E04E0908F04F09090048EE992E0B6
:10C8900040E050E068E472EC00E010E028E432E4AC
:10C8A0000E9416299B01AC01C501B4010E94B5A3E9
:10C8B0000E9467A50E9422A4CB011F910F91FF90B7
:10C8C000EF90DF90CF90BF90AF909F908F900895A2
:10C8D0001F931FB7F89488E58CBD8DB581608DBD21
:10C8E000289A82E094E00E943405289817FF01C03E
:10C8F00078941F9108950E946864892F8295869587
:10C9000081700895EF92FF921F93CF93DF93EB0115
:10C910007A011FB7F89428E52CBD2DB521602DBDF7
:10C92000289A9F770E943405CE01B7010E943705EF
:10C93000289817FF01C07894DF91CF911F91FF9045
:10C94000EF900895DF93CF9300D0CDB7DEB7BE014F
:10C950006F5F7F4F41E050E00E94826489819A813D
:10C960000F900F90CF91DF9108950E94E3610E9494
:10C97000A2640895462F90E061E050E00E94B56403
:10C98000009729F460E070E080E090E00DC0BC0109
:10C9900080E090E00E944EA49B01AC0160E070EA50
:10C9A0008CE09AE40E94B5A308956DE00E94BA64F9
:10C9B00008956CE00E94BA6408958F929F92AF929E
:10C9C000BF92CF92DF92EF92FF920F931F9361E09D
:10C9D00046E050E00E94B564BC017F7180E090E0C9
:10C9E0000E944EA40E948BA54B015C01C090C9041B
:10C9F000D090CA04E090CB04F090CC048AED92E091
:10CA000040E050E068E472EC00E010E028E432E43A
:10CA10000E9416299B01AC01C501B4010E9404A526
:10CA20001F910F91FF90EF90DF90CF90BF90AF904C
:10CA30009F908F9008958F929F92AF92BF92CF92C6
:10CA4000DF92EF92FF920F931F9361E043E050E07B
:10CA50000E94B564BC0180E090E00E944EA40E9458
:10CA60008BA54B015C01C090C104D090C204E09042
:10CA7000C304F090C40482ED92E040E050E068E42A
:10CA800072EC00E010E028E432E40E9416299B01D9
:10CA9000AC01C501B4010E9404A51F910F91FF9044
:10CAA000EF90DF90CF90BF90AF909F908F900895C0
:10CAB0008F929F92AF92BF92CF92DF92EF92FF92AE
:10CAC0000F931F9361E044E050E00E94B564BC0105
:10CAD00080E090E00E944EA40E948BA54B015C0177
:10CAE000C090BD04D090BE04E090BF04F090C0049C
:10CAF0008EEC92E040E050E068E472EC00E010E080
:10CB000028E432E40E9416299B01AC01C501B4015E
:10CB10000E9404A51F910F91FF90EF90DF90CF909E
:10CB2000BF90AF909F908F900895CF92DF92EF9239
:10CB3000FF920F931F93CF93DF9361E042E050E0A9
:10CB40000E94B564EC01DF7796FDD068C090B10417
:10CB5000D090B204E090B304F090B40482EC92E080
:10CB600040E050E068E472EC00E010E028E432E4D9
:10CB70000E9416296B017C01BE01882777FD8095F4
:10CB8000982F0E9450A49B01AC01C701B6010E94DE
:10CB900004A5DF91CF911F910F91FF90EF90DF904F
:10CBA000CF900895CF92DF92EF92FF920F931F9351
:10CBB000CF93DF9361E041E050E00E94B564EC0167
:10CBC000DF7796FDD068C090AD04D090AE04E090C1
:10CBD000AF04F090B0048EEB92E040E050E068E4E7
:10CBE00072EC00E010E028E432E40E9416296B01A8
:10CBF0007C01BE01882777FD8095982F0E9450A464
:10CC00009B01AC01C701B6010E9404A5DF91CF9141
:10CC10001F910F91FF90EF90DF90CF9008958F922A
:10CC20009F92AF92BF92CF92DF92EF92FF920F93BB
:10CC30001F9361E045E050E00E94B564BC0180E0D4
:10CC400090E00E944EA40E948BA54B015C01C09015
:10CC5000B904D090BA04E090BB04F090BC048AEC14
:10CC600092E040E050E068E472EC00E010E028E47C
:10CC700032E40E9416299B01AC01C501B4010E9457
:10CC800004A51F910F91FF90EF90DF90CF90BF9080
:10CC9000AF909F908F9008958F929F92AF92BF9286
:10CCA000CF92DF92EF92FF920F931F9361E040E0EB
:10CCB00050E00E94B564BC0180E090E00E944EA468
:10CCC0000E948BA54B015C01C090B504D090B604C6
:10CCD000E090B704F090B80486EC92E040E050E0B9
:10CCE00068E472EC00E010E028E432E40E941629C7
:10CCF0009B01AC01C501B4010E9404A51F910F91D5
:10CD0000FF90EF90DF90CF90BF90AF909F908F906B
:10CD10000895462F90E061E050E00E94B5640895C8
:10CD20006BE00E9489669C012F773070295030405B
:10CD3000C9010895462F90E060E050E00E94B5647C
:10CD4000089569E00E949A669C0194E036952795C3
:10CD50009A95E1F780E0922F9F700E9415620895E6
:10CD600069E00E949A669C012F70307080E0922FDB
:10CD70000E941562089569E00E949A6680E092958B
:10CD80009F700E941562089569E00E949A6680E093
:10CD90009F700E9415620895662319F46FE070E099
:10CDA00002C06FE870E00E949A66292F30E045E0EB
:10CDB000220F331F4A95E1F7C9019F7034FD906F30
:10CDC0000E9447620895662319F46FE070E002C084
:10CDD0006FE870E00E949A66282F30E055E0220F3D
:10CDE000331F5A95E1F7C9019F7034FD906F0E947F
:10CDF00047620895662319F46DE070E002C06DE8A3
:10CE000070E00E949A66292F30E065E0220F331F00
:10CE10006A95E1F7C9019F7034FD906F0E947C62B2
:10CE20000895662319F46DE070E002C06DE870E0CB
:10CE30000E949A66282F30E075E0220F331F7A9502
:10CE4000E1F7C9019F7034FD906F0E947C620895E4
:10CE5000662319F46BE070E002C06BE870E00E949A
:10CE60009A660E94B1620895662319F46CE070E03E
:10CE700002C06CE870E00E949A660E94B162089558
:10CE8000662319F46EE070E002C06EE870E00E9464
:10CE90009A660E94E3620895662319F468E070E0E0
:10CEA00002C068E870E00E949A660E94E3620895FA
:10CEB00066E00E949A66BC0160707F70672F7727DA
:10CEC00080E090E00E944EA420E030E048EC52E484
:10CED0000E9404A520E030E040E751E40E94B5A3A1
:10CEE000089566E00E949A669C012F773070295061
:10CEF0003040C901089561E00E949A660E9415625F
:10CF0000089564E00E949A660E94B162089560E00C
:10CF10000E949A660E94E36208950E949A669C01AC
:10CF20003F7094FD306FC9010895CF92DF92EF9268
:10CF3000FF920F931F93CF93DF9363E00E948D675F
:10CF4000EC01C090A104D090A204E090A304F09062
:10CF5000A40482EB92E040E050E068E472EC00E070
:10CF600010E028E432E40E9416296B017C01BE0126
:10CF7000882777FD8095982F0E9450A49B01AC01D3
:10CF8000C701B6010E9404A5DF91CF911F910F91B7
:10CF9000FF90EF90DF90CF90089562E00E948D6740
:10CFA0000E944762089565E00E948D670E947C623E
:10CFB000089590E060E044E850E00E94B564089570
:10CFC00094600E94A2640895EF92FF921F93CF9302
:10CFD000DF93EB017A011FB7F89428E52CBD2DB53E
:10CFE00021602DBD289A90680E943405CE01B701BA
:10CFF0000E944F05289817FF01C07894DF91CF91C8
:10D000001F91FF90EF900895DF93CF9300D0CDB79D
:10D01000DEB77A836983BE016F5F7F4F41E050E0E6
:10D020000E94E4670F900F90CF91DF9108951F93B6
:10D03000182F84E094E00E94A264BC017F73912FBA
:10D040009295907F80E0682B792B84E094E00E9499
:10D0500004681F91089594600E9404680895CF9217
:10D06000DF92EF92FF921F93CF93DF93EC017B014E
:10D070006A011FB7F8940E94A264B601609570958A
:10D08000682379236E297F29CE010E94046817FF47
:10D0900001C07894DF91CF911F91FF90EF90DF90C6
:10D0A000CF9008950F931F93CF93DF93762FEA01CC
:10D0B000890190E060E0472F50E00E94E361BE01EB
:10D0C000A8010E942F68DF91CF911F910F910895C1
:10D0D0001F93182FCB01BA010E94156380E0492FDE
:10D0E000582F4031510510F04FE050E0F4E0440F6C
:10D0F000551FFA95E1F7812F69E020EF30E00E949B
:10D1000052681F9108951F93182FCB01BA010E94F6
:10D11000156380E0492F582F4031510510F04FE042
:10D1200050E0812F69E02FE030E00E9452681F91AB
:10D1300008951F93182FCB01BA010E94156380E058
:10D14000492F582FCA018031910510F08FE090E0EF
:10D15000582F5295507F812F69E040E020E030EF5A
:10D160000E9452681F9108951F93182FCB01BA0196
:10D170000E94156380E0492F582F9A012031310514
:10D1800010F02FE030E0812F69E040E0522F20E0E6
:10D190003FE00E9452681F9108951F93CF93DF9341
:10D1A000182FCB01BA01222319F4CFE0D0E002C03E
:10D1B000CFE8D0E00E9462639C01A5E035952795F9
:10D1C000AA95E1F74FEF203834071CF420E830E04F
:10D1D00007C0203831051CF02FE730E001C0307067
:10D1E000812F6C2F40E0522F20E03FEF0E945268C9
:10D1F000DF91CF911F9108951F93CF93DF93182F45
:10D20000CB01BA01222319F4CFE0D0E002C0CFE86D
:10D21000D0E00E946263AC01B5E055954795BA95A0
:10D22000E1F72FEF403852071CF440E850E007C008
:10D23000403851051CF04FE750E001C05070812F7D
:10D240006C2F2FEF30E00E945268DF91CF911F9139
:10D2500008951F93CF93DF93182FCB01BA01222398
:10D2600019F4CDE0D0E002C0C8E8D0E00E94986395
:10D270009C0185E0359527958A95E1F74FEF203899
:10D2800034071CF420E830E007C0203831051CF0DA
:10D290002FE730E001C03070812F6C2F40E0522F1B
:10D2A00020E03FEF0E945268DF91CF911F910895D7
:10D2B0001F93CF93DF93182FCB01BA01222319F4C8
:10D2C000CDE0D0E002C0C8E8D0E00E949863AC0195
:10D2D00095E0559547959A95E1F72FEF403852071D
:10D2E0001CF440E850E007C0403851051CF04FE7FF
:10D2F00050E001C05070812F6C2F2FEF30E00E9462
:10D300005268DF91CF911F9108951F93CF93DF93C0
:10D31000182FCB01BA01222319F4CBE0D0E002C0D0
:10D32000CBE8D0E00E94CE63AC01812F6C2F2FEFB1
:10D330003FE00E945268DF91CF911F9108951F93A3
:10D34000CF93DF93182FCB01BA01222319F4CCE03D
:10D35000D0E002C0CCE8D0E00E94CE63AC01812FC7
:10D360006C2F2FEF3FE00E945268DF91CF911F9109
:10D3700008951F93CF93DF93182FCB01BA01222377
:10D3800019F4CEE0D0E002C0CEE8D0E00E941B64E9
:10D39000AC01812F6C2F2FEF3FE00E945268DF918C
:10D3A000CF911F9108951F93CF93DF93182FCB0137
:10D3B000BA01222319F4C8E0D0E002C0C8E8D0E0E6
:10D3C0000E941B64AC01812F6C2F2FEF3FE00E9465
:10D3D0005268DF91CF911F910895CF93DF93C0E002
:10D3E000D0E00E94D9180E94F41880E00E947319BE
:10D3F000009729F0219681E0C43FD80791F7DF918B
:10D40000CF91089580919411882319F086E20E94AB
:10D41000E305089580911713882319F087E20E948D
:10D42000E30508950F931F93DF93CF93CDB7DEB736
:10D4300028970FB6F894DEBF0FBECDBF8FE891E1FD
:10D440000E9494468DB79EB708970FB6F8949EBF7A
:10D450000FBE8DBFEDB7FEB731968E010F5F1F4F28
:10D46000ADB7BEB712961C930E93119788E090E06B
:10D47000938382838091D0119091D111958384837D
:10D480008091171290E00196978386830E94CEA721
:10D49000F80101900020E9F78DB79EB708960FB606
:10D4A000F8949EBF0FBE8DBFC8018E1B9F0B459683
:10D4B0009695879561E00E949F04C8010E944B06E3
:10D4C0000AE711E1C80160E270E044E150E00E9427
:10D4D00071A780911713882381F06091D411709106
:10D4E000D511DB01FD0101900020E9F73197EA1B1E
:10D4F000FB0BC801AF010E9468A76091D211709127
:10D50000D311DB01FD0101900020E9F73197EA1BFF
:10D51000FB0B24E130E02E1B3F0B36952795265858
:10D520003E4EC901AF010E9468A782E090E00E94D0
:10D530003906809117126EE00E949A66192F809129
:10D5400017126CE00E949A66929591701295117074
:10D55000910F092F909394118AE791E160E270E0B6
:10D5600044E150E00E9471A7002391F06091D8112E
:10D570007091D911DB01FD0101900020E9F731978D
:10D58000EA1BFB0B2CE731E1C901AF010E9468A740
:10D5900083E090E00E94390628960FB6F894DEBF2B
:10D5A0000FBECDBFCF91DF911F910F910895CF9303
:10D5B000DF9388EC90E00E948905CAE7D1E1CE01B3
:10D5C00060E270E044E150E00E9471A781E00E94B7
:10D5D0005E12BC01FC0101900020E9F73197E81BC5
:10D5E000F90B24E130E02E1B3F0B369527952C0FCD
:10D5F0003D1FC901AF010E9468A780E090E00E9432
:10D600003906CE0160E270E044E150E00E9471A76B
:10D6100081E090E00E94390682E090E00E943906A5
:10D6200083E090E00E9439060E941A128BE00E946B
:10D630005E129093D1118093D0118FE00E945E1200
:10D640009093D3118093D21183E70E945E1290933E
:10D65000D5118093D41187E60E945E129093D91160
:10D660008093D8118FE891E10E94D6460E94126AF9
:10D67000DF91CF91089588E00E94E305089586E048
:10D680000E94E30508958AE00E94E305089587E07B
:10D690000E94E305089585E00E94E3050895EF9256
:10D6A000FF920F931F93DF93CF93CDB7DEB72897E9
:10D6B0000FB6F894DEBF0FBECDBF8FE891E10E9498
:10D6C00094468DB79EB708970FB6F8949EBF0FBECD
:10D6D0008DBFEDB7FEB731968E010F5F1F4FADB70F
:10D6E000BEB712961C930E93119788E0E82EF12C8A
:10D6F000F382E2828091D0119091D111958384833D
:10D7000080911D1290E00D96978386830E94CEA78C
:10D710008DB79EB708960FB6F8949EBF0FBE8DBF0B
:10D7200085E061E00E949F04C8010E944B06ADB7EE
:10D73000BEB718970FB6F894BEBF0FBEADBFEDB71A
:10D74000FEB7319612961C930E931197F382E282E4
:10D750008091D2119091D311958384838091181276
:10D7600090E00196978386830E94CEA78DB79EB7DF
:10D7700008960FB6F8949EBF0FBE8DBF8AE061E099
:10D780000E949F04C8010E944B0690911E1286EAD7
:10D79000989FC00111243091181221E1329F90010D
:10D7A0001124820F931F8E569E4F60E04BE022E0C3
:10D7B0000E94F92781FD03C002EF17E002C002E0DA
:10D7C00018E082E063E00E949F04C8010E944B06BB
:10D7D00028960FB6F894DEBF0FBECDBFCF91DF9174
:10D7E0001F910F91FF90EF900895EF92FF920F938A
:10D7F0001F93DF93CF93CDB7DEB728970FB6F8947A
:10D80000DEBF0FBECDBF8FE891E10E9494468DB779
:10D810009EB708970FB6F8949EBF0FBE8DBFEDB7A9
:10D82000FEB731968E010F5F1F4FADB7BEB7129690
:10D830001C930E93119798E0E92EF12CF382E2826B
:10D840008091D0119091D1119583848380911D1284
:10D8500090E00D96978386830E94CEA78DB79EB7E2
:10D8600008960FB6F8949EBF0FBE8DBF85E061E0AD
:10D870000E949F04C8010E944B06ADB7BEB718971F
:10D880000FB6F894BEBF0FBEADBFEDB7FEB7319671
:10D8900012961C930E931197F382E2828091D2111B
:10D8A0009091D311958384838091191290E0019611
:10D8B000978386830E94CEA78DB79EB708960FB632
:10D8C000F8949EBF0FBE8DBF8AE061E00E949F0466
:10D8D000C8010E944B0628960FB6F894DEBF0FBE13
:10D8E000CDBFCF91DF911F910F91FF90EF900895E1
:10D8F0000F931F93DF93CF93CDB7DEB728970FB663
:10D90000F894DEBF0FBECDBF8FE891E10E94944630
:10D910008DB79EB708970FB6F8949EBF0FBE8DBF08
:10D92000EDB7FEB731968E010F5F1F4FADB7BEB793
:10D9300012961C930E93119788E090E09383828354
:10D940008091D0119091D1119583848380911D1283
:10D9500090E00D96978386830E94CEA7F8010190F0
:10D960000020E9F78DB79EB708960FB6F8949EBFD2
:10D970000FBE8DBFC8018E1B9F0B45969695879550
:10D9800061E00E949F04C8010E944B0628960FB6D2
:10D99000F894DEBF0FBECDBFCF91DF911F910F91E5
:10D9A00008950F931F93CF93DF9388EC90E00E942C
:10D9B0008905CAE7D1E1CE0160E270E044E150E0C0
:10D9C0000E9471A781E00E945E12BC01FC010190DF
:10D9D0000020E9F73197E81BF90B04E110E098010A
:10D9E0002E1B3F0B369527952C0F3D1FC901AF010C
:10D9F0000E9468A780E090E00E943906CE0160E2B4
:10DA000070E044E150E00E9471A781E090E00E9444
:10DA1000390681E10E945E12BC01FC0101900020E8
:10DA2000E9F73197E81BF90B0E1B1F0B16950795AD
:10DA30000C0F1D1FC801AF010E9468A782E090E093
:10DA40000E943906CE0160E270E044E150E00E949D
:10DA500071A783E090E00E9439068FE891E10E946F
:10DA6000D646DF91CF911F910F910895CF93DF9309
:10DA70000E94D16C8FE50E945E12EC0180E062E0B2
:10DA80000E949F04CE010E944B0680E60E945E1217
:10DA9000EC0182E063E00E949F04CE010E944B06ED
:10DAA0000E941A128CE00E945E129093D111809312
:10DAB000D0118EE00E945E129093D3118093D21108
:10DAC000DF91CF91089590911E1286EA989FC00130
:10DAD00011243091181221E1329F90011124820FFC
:10DAE000931F8E569E4F60E04BE022E00E94F92784
:10DAF00081FF02C08D7001C0826060911E1296EAA3
:10DB0000699FB00111242091181291E1299F900181
:10DB10001124620F731F6E567E4F0E94EC270E94E5
:10DB2000366D0895CF93DF930E94D16C8FE50E94EC
:10DB30005E12EC0180E062E00E949F04CE010E9430
:10DB40004B060E941A128CE00E945E129093D11133
:10DB50008093D0118DE00E945E129093D311809338
:10DB6000D211DF91CF910895CF93DF930E94D16CB2
:10DB700087E70E945E12EC0180E062E00E949F0451
:10DB8000CE010E944B0688E70E945E12EC0182E003
:10DB900063E00E949F04CE010E944B060E941A126D
:10DBA0008CE00E945E129093D1118093D011DF918E
:10DBB000CF9108958FE10E94E305089580911F128F
:10DBC000882319F088E20E94E30508958EE10E94FF
:10DBD000E30508958DE10E94E30508958CE10E941C
:10DBE000E30508950F931F93DF93CF93CDB7DEB76F
:10DBF00028970FB6F894DEBF0FBECDBF8FE891E136
:10DC00000E9494468DB79EB708970FB6F8949EBFB2
:10DC10000FBE8DBFEDB7FEB731968E010F5F1F4F60
:10DC2000ADB7BEB712961C930E93119788E090E0A3
:10DC3000938382838091D0119091D11195838483B5
:10DC400080911E1290E00D96978386830E94CEA746
:10DC5000F80101900020E9F78DB79EB708960FB63E
:10DC6000F8949EBF0FBE8DBFC8018E1B9F0B4596BB
:10DC70009695879561E00E949F04C8010E944B061B
:10DC800028960FB6F894DEBF0FBECDBFCF91DF91BF
:10DC90001F910F910895EF92FF920F931F93CF93CF
:10DCA000DF9388EC90E00E948905CAE7D1E1CE01BC
:10DCB00060E270E044E150E00E9471A781E00E94C0
:10DCC0005E12BC01FC0101900020E9F73197E81BCE
:10DCD000F90B04E110E098012E1B3F0B36952795B8
:10DCE0002C0F3D1FC901AF010E9468A780E090E0A2
:10DCF0000E943906CE0160E270E044E150E00E94EB
:10DD000071A781E090E00E94390687E70E945E12C9
:10DD1000BC01FC0101900020E9F73197E81BF90BE9
:10DD2000CE01AF010E9468A78FE00E945E12BC0185
:10DD3000FC0101900020E9F73197E81BF90B9801ED
:10DD40002E1B3F0B369527952C0F3D1FC901AF01A8
:10DD50000E9468A789E70E945E12BC01FC01019045
:10DD60000020E9F73197E81BF90B0E1B1F0B0C0F76
:10DD70001D1FC801AF010E9468A782E090E00E94C9
:10DD80003906CE0160E270E044E150E00E9471A7E4
:10DD900082E798E00E942912BC01FC01019000205A
:10DDA000E9F73197E81BF90B9E012E1B3F0B2E5E06
:10DDB0003F4FC901AF010E9468A788E70E945E1229
:10DDC000BC01FC0101900020E9F73197E81BF90B39
:10DDD0002296CE01AF010E9468A783E090E00E94E6
:10DDE00039068FE891E10E94D6460E941A128CE013
:10DDF0000E945E129093D1118093D011DF91CF9148
:10DE00001F910F91FF90EF900895382F262F862FA6
:10DE100063E00E9436A690E0880F991F86599A4FBA
:10DE2000FC01A591B4912150253010F020E005C0EF
:10DE3000E22FF0E0E057F74F2081832F90E08C57DE
:10DE40009F4F34E0880F991F3A95E1F7642F70E0F7
:10DE50006F707070022E02C0660F771F0A94E2F78F
:10DE60004FE050E002C0440F551F2A95E2F78A0F99
:10DE70009B1F0E942F6808951F93382F262F862FEF
:10DE800063E00E9436A690E0880F991F86599A4F4A
:10DE9000FC01459154912150253010F010E005C04F
:10DEA000E22FF0E0E057F74F1081832F90E08C577E
:10DEB0009F4F64E0880F991F6A95E1F7840F951FC3
:10DEC0000E94A26402C0969587951A95E2F78F701A
:10DED0001F91089570E0660F771F62597A4FFB011A
:10DEE0002591349190E08C579F4FE4E0880F991F63
:10DEF000EA95E1F7820F931F0E94A26408956630AD
:10DF000018F020E030E015C070E0660F771F640F56
:10DF1000751FFB012591349190E08C579F4FA4E031
:10DF2000880F991FAA95E1F7820F931F0E94A264A0
:10DF30009C01C9010895643018F020E030E015C05C
:10DF400070E0660F771F640F751FFB0125913491F8
:10DF500090E08C579F4F44E0880F991F4A95E1F756
:10DF6000820F931F0E94A2649C01C901089560E082
:10DF70004AEC55E00E949B6FBC01009729F460E0D9
:10DF800070E080E090E00CC080E090E00E944EA441
:10DF90009B01AC0160E070EA8CE09AE40E94B5A3BA
:10DFA000089542ED55E00E949B6F0895DF93CF9353
:10DFB0000F92CDB7DEB7E62FF0E0EE0FFF1FEE5168
:10DFC000FA4F8591949169830E94A264282F6981F8
:10DFD000862F63E00E9436A641E050E002C0440F65
:10DFE000551F9A95E2F7822F84230F90CF91DF91EE
:10DFF0000895CF92DF92EF92FF920F931F93CF93EA
:10E00000DF93182FC62E0E949B6FEC01DF7796FDE1
:10E01000D06826EA129F90011124225A3E4F8C2D7F
:10E0200090E0B4E0880F991FBA95E1F7C090D5044D
:10E03000D090D604E090D704F090D804820F931FBC
:10E0400040E050E068E472EC00E010E028E432E4E4
:10E050000E9416296B017C01BE01882777FD8095FF
:10E06000982F0E9450A49B01AC01C701B6010E94E9
:10E0700004A5DF91CF911F910F91FF90EF90DF905A
:10E08000CF90089542E955E00E94F96F089542ED5E
:10E0900055E00E94F96F0895CF92DF92EF92FF92C0
:10E0A0000F931F93CF93DF93082F162F42EB55E06A
:10E0B0000E947F6FEC01DF7796FDD06826EA029F11
:10E0C0009001112429563E4F81E1189FC00111246F
:10E0D000C090DD04D090DE04E090DF04F090E00416
:10E0E000820F931F40E050E068E472EC00E010E023
:10E0F00028E432E40E9416296B017C01BE018827C6
:10E1000077FD8095982F0E9450A4A70196010E9448
:10E1100004A5DF91CF911F910F91FF90EF90DF90B9
:10E12000CF9008956F927F928F929F92AF92BF92FD
:10E13000CF92DF92EF92FF920F931F93CF93DF93D3
:10E14000A82EB62EEA013801490126EA829F9001E5
:10E1500011242D563E4F81E1689FC0011124C090CB
:10E16000D904D090DA04E090DB04F090DC04820F54
:10E17000931F40E050E068E472EC00E010E028E417
:10E1800032E40E9416299B01AC0185E08B15A0F1B9
:10E190008B2D90E0880F991F8C0F9D1FFC01C5915E
:10E1A000D491C401B3010E94B5A30E941DA4669F2F
:10E1B0009001679F300D769F300D1124B90180E0EA
:10E1C00090E00E944EA40E9467A59B01AC018A2D9D
:10E1D00090E08C579F4F14E0880F991F1A95E1F734
:10E1E000C80FD91FCA01B9010E9422A49B01AC012A
:10E1F000CE01B9010E940468DF91CF911F910F9168
:10E20000FF90EF90DF90CF90BF90AF909F908F9056
:10E210007F906F9008950F931F9389019A014AE7A9
:10E2200055E00E9492701F910F9108950F931F93D4
:10E2300089019A0146E855E00E9492701F910F9162
:10E240000895FF920F931F93CF93DF93F82E6430BE
:10E2500020F5862F90E0880F991F840F951FFC01F1
:10E26000C591D491C901B8010E9467A59B01AC0179
:10E270008F2D90E08C579F4F64E0880F991F6A950F
:10E28000E1F7C80FD91FCA01B9010E9422A49B015E
:10E29000AC01CE01B9010E940468DF91CF911F91BA
:10E2A0000F91FF9008956F927F928F929F92AF92FD
:10E2B000BF92CF92DF92EF92FF920F931F93B82EEF
:10E2C000A62E39014A0186EA2B2D289FC001112470
:10E2D000825A9E4F262F30E0E4E0220F331FEA954A
:10E2E000E1F7C090D504D090D604E090D704F09028
:10E2F000D804820F931F40E050E068E472EC00E025
:10E3000010E028E432E40E9416299B01AC01C4010C
:10E31000B3010E94B5A30E9422A480E090E00E9475
:10E320004EA48B019C018B2D6A2D42E955E00E9481
:10E3300021711F910F91FF90EF90DF90CF90BF90D0
:10E34000AF909F908F907F906F9008956F927F9283
:10E350008F929F92AF92BF92CF92DF92EF92FF92F5
:10E360000F931F93B82EA62E39014A0186EA2B2D52
:10E37000289FC0011124865A9E4F262F30E0F4E0DA
:10E38000220F331FFA95E1F7C090D104D090D20448
:10E39000E090D304F090D404820F931F40E050E04B
:10E3A00068E472EC00E010E028E432E40E941629F0
:10E3B0009B01AC01C401B3010E94B5A3562F472FA6
:10E3C000382F292FDA01F9016B2F7A2F8F2F9E2FEB
:10E3D0002B2F3A2F4F2F5E2F0E9404A50E9422A4BC
:10E3E00080E090E00E944EA48B019C018B2D6A2D51
:10E3F0004AE955E00E9421711F910F91FF90EF9023
:10E40000DF90CF90BF90AF909F908F907F906F9054
:10E4100008956F927F928F929F92AF92BF92CF9208
:10E42000DF92EF92FF920F931F93CF93DF93B82E5B
:10E43000A62EEA013801490186EA2B2D289FC0014A
:10E4400011248A5A9E4F262F30E0A4E0220F331F5A
:10E45000AA95E1F7C090CD04D090CE04E090CF040F
:10E46000F090D004820F931F40E050E068E472EC1B
:10E4700000E010E028E432E40E9416299B01AC0180
:10E48000C401B3010E94B5A3562F472F382F292F5F
:10E49000DA01F9016B2F7A2F8F2F9E2F2B2F3A2F16
:10E4A0004F2F5E2F0E9404A50E9422A480E090E0DE
:10E4B0000E944EA48B019C018B2D6A2DAE010E94FF
:10E4C0002171DF91CF911F910F91FF90EF90DF901D
:10E4D000CF90BF90AF909F908F907F906F90089556
:10E4E0000F931F9389019A0142EA55E00E94097235
:10E4F0001F910F9108950F931F9389019A014AEA82
:10E5000055E00E9409721F910F910895EF92FF92BA
:10E510001F93DF93CF930F92CDB7DEB7162F862FC1
:10E5200090E0880F991F8E519A4FFC01E590F4906E
:10E53000C70149830E94A2649C01812F63E00E946D
:10E5400036A661E070E002C0660F771F9A95E2F789
:10E55000CB0180959095282339234981442311F0DC
:10E56000262B372BC701B9010E9404680F90CF9169
:10E57000DF911F91FF90EF9008952F923F924F925D
:10E580005F926F927F928F929F92AF92BF92CF9243
:10E59000DF92EF92FF920F931F93DF93CF930F922F
:10E5A000CDB7DEB7182F062F29830E947F6F4C014D
:10E5B000AA24BB242981222359F5C501B4010E9454
:10E5C0004EA40E948BA54B015C0126EA129F90018C
:10E5D00011242D563E4F81E1089FC0011124C090A7
:10E5E000D904D090DA04E090DB04F090DC04820FD0
:10E5F000931F40E050E068E472EC00E010E028E493
:10E6000032E40E9416299B01AC01C501B4014EC041
:10E6100081E1089F1001112486EA189FC00111248E
:10E62000280E391EC090E504D090E604E090E7047F
:10E63000F090E804C10181569E4F40E050E068E44C
:10E6400072EC00E010E028E432E40E9416292B016D
:10E650003C01C090E104D090E204E090E304F0902B
:10E66000E404C10185569E4F40E050E068E472EC3E
:10E6700000E010E028E432E40E9416297B018C01BE
:10E68000C501B4010E944EA44B015C01C301B2015B
:10E6900020E030E44CE156EC0E9404A59B01AC0163
:10E6A000C501B4010E944DA3A80197010E9404A5D1
:10E6B0000F90CF91DF911F910F91FF90EF90DF901E
:10E6C000CF90BF90AF909F908F907F906F905F9012
:10E6D0004F903F902F9008954AE755E020E00E9428
:10E6E000BD72089546E855E020E00E94BD7208958D
:10E6F000242F4EEB55E00E94BD7208958F929F9299
:10E70000AF92BF92CF92DF92EF92FF920F931F933F
:10E71000082F162F0E949B6FBC0180E090E00E94A2
:10E720004EA40E948BA54B015C0126EA029F90013A
:10E730001124265A3E4F812F90E014E0880F991F34
:10E740001A95E1F7C090D104D090D204E090D304A0
:10E75000F090D404820F931F40E050E068E472EC24
:10E7600000E010E028E432E40E9416299B01AC018D
:10E77000C501B4010E9404A51F910F91FF90EF9075
:10E78000DF90CF90BF90AF909F908F9008954AE90F
:10E7900055E00E947E7308954AED55E00E947E7315
:10E7A00008958F929F92AF92BF92CF92DF92EF9295
:10E7B000FF920F931F93082F162F0E949B6FBC018F
:10E7C00080E090E00E944EA40E948BA54B015C016A
:10E7D00026EA029F900111242A5A3E4F812F90E091
:10E7E00004E0880F991F0A95E1F7C090CD04D090FE
:10E7F000CE04E090CF04F090D004820F931F40E04D
:10E8000050E068E472EC00E010E028E432E40E949A
:10E8100016299B01AC01C501B4010E9404A51F91FA
:10E820000F91FF90EF90DF90CF90BF90AF909F90AF
:10E830008F90089542EA55E00E94D17308954AEA04
:10E8400055E00E94D17308954EEE55E00E94D173B9
:10E8500008958EE10E94D90508958F929F92AF92FC
:10E86000BF92CF92DF92EF92FF920F931F93DF93AD
:10E87000CF93CDB7DEB764970FB6F894DEBF0FBE67
:10E88000CDBF80911B12882309F479C08091C112F9
:10E890008F3F09F474C08091C3128F3708F06FC0A6
:10E8A00090918F1180911712992351F50E940F6654
:10E8B0006093941170939511809396119093971192
:10E8C0008091171290E00E941B65609398117093DD
:10E8D000991180939A1190939B118091171290E057
:10E8E0000E94956560939C1170939D1180939E1179
:10E8F00090939F118091171290E00E94D9642AC0D2
:10E9000090E00E944C6660939411709395118093EF
:10E910009611909397118091171290E00E9458657C
:10E92000609398117093991180939A1190939B1111
:10E930008091171290E00E94D26560939C117093B1
:10E940009D1180939E1190939F118091171290E0DA
:10E950000E94D5646093A8117093A9118093AA11A5
:10E960009093AB118091171290E00E94DD64609348
:10E97000AC117093AD118093AE119093AF11809153
:10E980001B12882309F431C180911E1290911F122D
:10E99000891708F02AC1609119120E9424746093AB
:10E9A0008F11709390118093911190939211809197
:10E9B0001E12609119120E94CC7360939311709390
:10E9C0009411809395119093961180911E126091ED
:10E9D00019120E94477060939B1170939C11809351
:10E9E0009D1190939E1180911E12609119120E94A8
:10E9F000B76F6093971170939811809399119093CA
:10EA00009A1160918F117091901180919111909154
:10EA10009211209193113091941140919511509140
:10EA200096110E9404A5D62EC72EB82EA92EA60197
:10EA30009501652F742F832F922F20E030E040EA5C
:10EA400050E40E9400A518165CF00F2EF0E0EF2EA7
:10EA5000F0E0FF2EF0E00F2FF0E01F2FF02D33C07D
:10EA600060919B1170919C1180919D1190919E11CC
:10EA7000D601F5012B2F3A2F4F2F5E2F0E94B5A301
:10EA8000E62EF72E082F192F20E030E0A9010E9472
:10EA9000B1A3882324F417FB109517F91095C8012A
:10EAA000B70120E030E040E85FE30E9400A51816BF
:10EAB00054F40F2EF0E0EF2EF0E0FF2EF0E80F2FD1
:10EAC000FFE31F2FF02D80E060E00E949F048DB7D0
:10EAD0009EB70E970FB6F8949EBF0FBE8DBFEDB7D1
:10EAE000FEB731964E010894811C911CADB7BEB79C
:10EAF00012969C928E92119784E190E09383828388
:10EB000085E998E0958384838091191290E00196BD
:10EB100097838683E086F1860287138780911E1291
:10EB200090E00D96958784870E94CEA78DB79EB7FB
:10EB30000E960FB6F8949EBF0FBE8DBFC4010E9403
:10EB40004B0680E061E00E949F0460918F117091FC
:10EB5000901180919111909192114DEA58E025E029
:10EB60000E94930687E061E00E949F0460919711E4
:10EB7000709198118091991190919A1143EB58E0FE
:10EB800025E00E9493068EE061E00E949F04609160
:10EB900093117091941180919511909196114DEA75
:10EBA00058E025E00E94930683E062E00E949F0403
:10EBB00060919B1170919C1180919D1190919E117B
:10EBC00049EB58E027E00E9493068BE062E00E9448
:10EBD0009F04A6019501652F7C2D832F9A2D49EB6B
:10EBE00058E027E00E94930630C087E060E00E9472
:10EBF0009F0486E392E00E944B0680E061E00E9461
:10EC00009F0488E392E00E944B068EE061E00E9440
:10EC10009F0488E392E00E944B0683E062E00E943A
:10EC20009F0486E392E00E944B068BE062E00E9424
:10EC30009F0486E392E00E944B068BE060E00E9416
:10EC40009F0486E392E00E944B0664960FB6F89408
:10EC5000DEBF0FBECDBFCF91DF911F910F91FF900F
:10EC6000EF90DF90CF90BF90AF909F908F900895DE
:10EC7000EF92FF92CF93DF9381E080938F1184EF27
:10EC800091E00E948905CAE7D1E1CE0160E270E01F
:10EC900044E150E00E9471A780E090E00E943906B4
:10ECA000CE0160E270E044E150E00E9471A781E48F
:10ECB0000E945E12BC01FC0101900020E9F731972F
:10ECC000E81BF90B9E01245F3F4FC901AF010E9471
:10ECD00068A786E580937F1181E480938D1181E0A0
:10ECE00090E00E943906CE0160E270E044E150E01D
:10ECF0000E9471A783E40E945E12BC01FC01019096
:10ED00000020E9F73197E81BF90BCE01AF010E9413
:10ED100068A787E58093841182E40E945E12BC019B
:10ED2000FC0101900020E9F73197E81BF90B9E01E7
:10ED30002E5E3F4FC901AF010E9468A782E090E0BC
:10ED40000E943906CE0160E270E044E150E00E948A
:10ED500071A783E090E00E9439060E942D74DF9134
:10ED6000CF91FF90EF90089580910513882371F45F
:10ED700080E090E0DC018093971190939811A0932C
:10ED80009911B0939A110E947526089580910613E7
:10ED9000882311F080E001C083E080930613109275
:10EDA000D81080E090E0DC018093D9109093DA10C5
:10EDB000A093DB10B093DC10089580910513882395
:10EDC00071F480E090E0DC018093971190939811AA
:10EDD000A0939911B0939A110E946B260895809187
:10EDE0000613882311F080E001C083E080930613AE
:10EDF0001092D81080E090E0DC018093D9109093BD
:10EE0000DA10A093DB10B093DC10089580911B12F0
:10EE1000882349F1109202131092011380911E125F
:10EE2000609118120E943C6F80FF05C0482F4E7FF2
:10EE30001092B31107C0482F416081E08093B31155
:10EE40001092DE1085E08093DD1080911E1260919B
:10EE500018120E94056F8EEC98E00E94A2649093B5
:10EE600008138093071308958091B411882331F417
:10EE700080911E126091181241E005C080911E120F
:10EE80006091181240E00E9486720895CF93DF933C
:10EE900080910513882389F58CE060E00E949F042F
:10EEA00086E392E00E944B0687E060E00E949F04A8
:10EEB00086E392E00E944B0680E061E00E949F049E
:10EEC00088E392E00E944B068EE061E00E949F047E
:10EED00088E392E00E944B0683E062E00E949F0478
:10EEE00086E392E00E944B068BE062E00E949F0462
:10EEF00086E392E00E944B0616C0C0E0D0E08CE0B2
:10EF00006C2F0E949F0486E392E00E944B0682E0F1
:10EF10006C2F0E949F0486E392E00E944B0621968C
:10EF2000C430D10561F7DF91CF910895CF93DF937E
:10EF3000109205131092061384EF91E00E94890548
:10EF4000CAE7D1E1CE0160E270E044E150E00E9406
:10EF500071A780E090E00E943906CE0160E270E087
:10EF600044E150E00E9471A781E090E00E943906E0
:10EF7000CE0160E270E044E150E00E9471A782E0BF
:10EF800090E00E943906CE0160E270E044E150E07A
:10EF90000E9471A783E090E00E9439060E941A1235
:10EFA0008CE00E945E129093D1118093D0118EE07C
:10EFB0000E945E129093D3118093D21187ED98E056
:10EFC0000E9429129093D5118093D41186E90E9452
:10EFD0005E129093D7118093D6118EED98E00E9427
:10EFE00029129093D9118093D81185EE98E00E9450
:10EFF00029129093DB118093DA1187E90E945E1247
:10F000009093DD118093DC118CEE98E00E94291220
:10F010009093E1118093E0118FEE98E00E94291205
:10F020009093DF118093DE11DF91CF910895CF92FD
:10F03000DF92EF92FF920F931F93CF93DF93EC0138
:10F04000162F042F862F642F0E94D66F482F8DA372
:10F05000812F602F0E947873688379838A839B83D2
:10F0600080910513882349F0812F602F0E944C70F6
:10F07000688779878A879B873DC0C090D910D090D8
:10F08000DA10E090DB10F090DC10812F602F0E94EE
:10F090004C709B01AC01C701B6010E944DA3262F05
:10F0A000372F482F592F2093D9103093DA104093DF
:10F0B000DB105093DC102091D810322F3F5F30933B
:10F0C000D8102430B8F020E030E040EA50E40E944C
:10F0D000B5A3688779878A879B871092D81080E0CC
:10F0E00090E0DC018093D9109093DA10A093DB10AC
:10F0F000B093DC10812F602F0E946A6F292F30E0BF
:10F1000039A328A3013031F0013090F0802F8450D2
:10F11000823070F4C90144E0969587954A95E1F7ED
:10F1200083708BA396E0369527959A95E1F707C0F3
:10F13000822F83708BA3369527953695279523705C
:10F140002AA30330D8F4812F60E00E9424746B015D
:10F150007C016C837D838E839F83812F60E00E947E
:10F16000CC739B01AC01C701B6010E9404A56C8B56
:10F170007D8B8E8B9F8B812F60E01AC0812F61E089
:10F180000E9424746B017C016C837D838E839F833A
:10F19000812F61E00E94CC739B01AC01C701B601D5
:10F1A0000E9404A56C8B7D8B8E8B9F8B812F61E0E1
:10F1B0000E944770688F798F8A8F9B8F812F602F75
:10F1C0000E943C6F81708CA3EC88FD880E891F899A
:10F1D000C801B7012AE037ED43E25CE30E9400A5D5
:10F1E00018160CF03CC0688D798D8A8D9B8DA80116
:10F1F00097010E94B5A3562F472F382F292FE62EAF
:10F20000F72E082F192F862F942FA32FB22F8C8F14
:10F210009D8FAE8FBF8F652F742F832F922F20E08D
:10F2200030E0A9010E94B1A3882344F417FB109594
:10F2300017F91095EC8EFD8E0E8F1F8F6C8D7D8DC6
:10F240008E8D9F8D20E030E040E85FE30E9400A5B6
:10F25000181664F480E090E0A0E8BFE303C080E00B
:10F2600090E0DC018C8F9D8FAE8FBF8F6C817D8194
:10F270008E819F81288139814A815B810E9404A50A
:10F280007B018C01862F9F2DA02FB12F888B998B0E
:10F29000AA8BBB8B6E2D7F2D802F912F20E030E02D
:10F2A00040EA50E40E9400A518160CF03EC06885A4
:10F2B00079858A859B852E2D3F2D402F512F0E94C9
:10F2C000B5A3562F472F382F292FE62EF72E082FBC
:10F2D000192F862F942FA32FB22F8C879D87AE874F
:10F2E000BF87652F742F832F922F20E030E0A90174
:10F2F0000E94B1A3882344F417FB109517F91095C9
:10F30000EC86FD860E871F876C857D858E859F85A3
:10F3100020E030E040E85FE30E9400A5181664F4A6
:10F3200080E090E0A0E8BFE303C080E090E0DC0173
:10F330008C879D87AE87BF87DF91CF911F910F91FB
:10F34000FF90EF90DF90CF9008951F93DF93CF93BE
:10F35000CDB7DEB72A970FB6F894DEBF0FBECDBF8C
:10F36000182F8FE891E160911E12412F0E941778AB
:10F370008091B311882321F08091B11180FD38C0B4
:10F380004091B4119E012F5F3F4F812F90E04423A5
:10F39000C9F44DB75EB74C5050400FB6F8945EBFFD
:10F3A0000FBE4DBFEDB7FEB73196ADB7BEB71296E3
:10F3B0003C932E9311972AE030E03383228322EF8F
:10F3C00038E04AC0ADB7BEB71C970FB6F894BEBFC1
:10F3D0000FBEADBFEDB7FEB7319612963C932E939C
:10F3E00011972AE030E0338322832EEF38E034C0D7
:10F3F0004091B4119E012F5F3F4F812F90E0442335
:10F40000B1F4ADB7BEB71C970FB6F894BEBF0FBE30
:10F41000ADBFEDB7FEB7319612963C932E93119780
:10F420002AE030E03383228329E039E015C0ADB70C
:10F43000BEB71C970FB6F894BEBF0FBEADBFEDB7F9
:10F44000FEB7319612963C932E9311972AE030E046
:10F450003383228325E139E0358324830196978322
:10F46000868380918F1190919011A0919111B0910C
:10F47000921180879187A287B3870E94CEA74DB74C
:10F480005EB7445F5F4F0FB6F8945EBF0FBE4DBFCF
:10F49000CE0101960E944B062A960FB6F894DEBF65
:10F4A0000FBECDBFCF91DF911F9108951F93DF93C2
:10F4B000CF93CDB7DEB72A970FB6F894DEBF0FBE55
:10F4C000CDBF182F8FE891E160911E12412F0E944D
:10F4D00017788091B311882321F08091B11180FDBC
:10F4E00038C04091B4119E012F5F3F4F812F90E0B3
:10F4F0004423C9F44DB75EB74C5050400FB6F89452
:10F500005EBF0FBE4DBFEDB7FEB73196ADB7BEB70C
:10F5100012963C932E9311972AE030E03383228396
:10F5200020E239E04AC0ADB7BEB71C970FB6F894D9
:10F53000BEBF0FBEADBFEDB7FEB7319612963C937E
:10F540002E9311972AE030E0338322832CE239E0B6
:10F5500034C04091B4119E012F5F3F4F812F90E046
:10F560004423B1F4ADB7BEB71C970FB6F894BEBF35
:10F570000FBEADBFEDB7FEB7319612963C932E93FA
:10F5800011972AE030E03383228327E339E015C066
:10F59000ADB7BEB71C970FB6F894BEBF0FBEADBFD8
:10F5A000EDB7FEB7319612963C932E9311972AE051
:10F5B00030E03383228323E439E0358324830196CA
:10F5C000978386838091971190919811A0919911BA
:10F5D000B0919A1180879187A287B3870E94CEA7A6
:10F5E0004DB75EB7445F5F4F0FB6F8945EBF0FBE76
:10F5F0004DBFCE0101960E944B062A960FB6F89495
:10F60000DEBF0FBECDBFCF91DF911F910895CF9286
:10F61000DF92EF92FF921F93DF93CF93CDB7DEB7C8
:10F620002B970FB6F894DEBF0FBECDBF182F8FE813
:10F6300091E160911E12412F0E9417788091B311C1
:10F64000882321F08091B11180FD37C08091B411E1
:10F650007E010894E11CF11C8823C9F48DB79EB784
:10F660000C970FB6F8949EBF0FBE8DBFEDB7FEB7D7
:10F670003196ADB7BEB71296FC92EE9211976BE041
:10F68000C62ED12CD382C2828EE499E035C0ADB7AC
:10F69000BEB71C970FB6F894BEBF0FBEADBFEDB797
:10F6A000FEB731961296FC92EE9211978AE090E0A6
:10F6B0009383828384E699E07CC08091B4117E01BB
:10F6C0000894E11CF11C882309F05EC0ADB7BEB7F9
:10F6D0001C970FB6F894BEBF0FBEADBFEDB7FEB717
:10F6E00031961296FC92EE9211975BE0C52ED12CCA
:10F6F000D382C28281E799E095838483168317823F
:10F700008091971190919811A0919911B0919A11AF
:10F7100080879187A287B3870E94CEA78DB79EB7B7
:10F720000C960FB6F8949EBF0FBE8DBFC7010E9406
:10F730004B068BE062E00E949F04ADB7BEB71A97FC
:10F740000FB6F894BEBF0FBEADBFEDB7FEB7319692
:10F750001296FC92EE921197D382C2828BE599E0C9
:10F760009583848380919B1190919C11A0919D1110
:10F77000B0919E1186839783A087B1870E94CEA700
:10F780008DB79EB70A962AC0ADB7BEB71C970FB605
:10F79000F894BEBF0FBEADBFEDB7FEB7319612965F
:10F7A000FC92EE9211978AE090E0938382838EE739
:10F7B00099E09583848316831782809197119091A5
:10F7C0009811A0919911B0919A1180879187A28781
:10F7D000B3870E94CEA78DB79EB70C960FB6F8944C
:10F7E0009EBF0FBE8DBFCE0101960E944B062B9689
:10F7F0000FB6F894DEBF0FBECDBFCF91DF911F9142
:10F80000FF90EF90DF90CF900895EF92FF920F93CB
:10F810001F93DF93CF93CDB7DEB7A8970FB6F894B9
:10F82000DEBF0FBECDBF80910513823009F486C0C4
:10F83000833009F419C1813009F0BCC180E060E077
:10F840000E949F0480E00E94A5798AE060E00E9407
:10F850009F0481E00E94A57980E061E00E949F04FE
:10F8600082E00E94A5798AE061E00E949F0483E023
:10F870000E94A57980E062E00E949F0484E00E94DB
:10F88000A5798AE062E00E949F0485E00E94A57944
:10F8900080E063E00E949F0480911E1260E00E945D
:10F8A000CC732DB73EB72A5030400FB6F8943EBF08
:10F8B0000FBE2DBFEDB7FEB731968E010B5E1F4F09
:10F8C000ADB7BEB712961C930E931197BAE0EB2E0C
:10F8D000F12CF382E2822BE839E0358324836683BE
:10F8E0007783808791870E94CEA72DB73EB7265F8A
:10F8F0003F4F0FB6F8943EBF0FBE2DBFC8010E9408
:10F900004B068AE063E00E949F0480911E1261E032
:10F910000E94CC73ADB7BEB71A970FB6F894BEBFAE
:10F920000FBEADBFEDB7FEB7319612961C930E9386
:10F930001197F382E28225E939E07CC080E060E043
:10F940000E949F0480E00E94567A8AE060E00E9454
:10F950009F0481E00E94567A80E061E00E949F044B
:10F9600082E00E94567A8AE061E00E949F0483E070
:10F970000E94567A80E062E00E949F0484E00E9428
:10F98000567A8AE062E00E949F0485E00E94567ADF
:10F9900080E063E00E949F0480911E1260E00E945C
:10F9A0004770ADB7BEB71A970FB6F894BEBF0FBE7B
:10F9B000ADBFEDB7FEB731968E010B5E1F4F1296AD
:10F9C0001C930E931197AAE0EA2EF12CF382E282A7
:10F9D0002FE939E035832483668377838087918795
:10F9E0000E94CEA72DB73EB7265F3F4F0FB6F894C3
:10F9F0003EBF0FBE2DBFC8010E944B068AE063E0E8
:10FA00000E949F0480911E1261E00E944770ADB772
:10FA1000BEB71A970FB6F894BEBF0FBEADBFEDB715
:10FA2000FEB7319612961C930E931197F382E282E1
:10FA300029EA39E035832483668377838087918739
:10FA40000E94CEA72DB73EB7265F3F4F0FB6F89462
:10FA50003EBF0FBE2DBFC8010E944B0680911B12F6
:10FA6000882309F09FC083C2109106131111125010
:10FA70008FE891E160911E12412F0E94177880E07B
:10FA800060E00E949F04812F8F5F0E94077B412FBF
:10FA90004E5F8FE891E160911E120E94177880E01E
:10FAA00061E00E949F04812F8D5F0E94077B412FA0
:10FAB0004C5F8FE891E160911E120E94177880E000
:10FAC00062E00E949F04812F8B5F0E94077B80E091
:10FAD00063E00E949F048DB79EB70C970FB6F89411
:10FAE0009EBF0FBE8DBFEDB7FEB731968E010B5E88
:10FAF0001F4FADB7BEB712961C930E9311977BE0C4
:10FB0000E72EF12CF382E28283EB99E095838483E4
:10FB10008091061390E081709070019697838683A0
:10FB20008091A7119091A811A091A911B091AA114B
:10FB300080879187A287B3870E94CEA72DB73EB753
:10FB4000245F3F4F0FB6F8943EBF0FBE2DBFC801D4
:10FB50000E944B068BE063E00E949F048DB79EB726
:10FB60000A970FB6F8949EBF0FBE8DBFEDB7FEB7D4
:10FB70003196ADB7BEB712961C930E931197F382D0
:10FB8000E2828BE599E0958384838091AB1190911B
:10FB9000AC11A091AD11B091AE1186839783A0876F
:10FBA000B1874ECF90911E1280911F12981708F0C6
:10FBB000DEC1DFC18FE891E160911E124091181201
:10FBC0000E9417788AE791E160E270E044E150E03A
:10FBD0000E9471A781E480938D118091B4118823D4
:10FBE00019F486E580937F1181E090E00E94390648
:10FBF00080E061E00E949F0400D000D000D0EDB70B
:10FC0000FEB731968E010F5F1F4FADB7BEB712968C
:10FC10001C930E93119784E190E09383828380EC90
:10FC200099E0958384830E94CEA72DB73EB72A5FC3
:10FC30003F4F0FB6F8943EBF0FBE2DBFC8010E94C4
:10FC40004B068AE791E160E270E044E150E00E94F7
:10FC500071A78091B411882379F480E580937A119B
:10FC60008AE380937B1187E58093841186E58093F6
:10FC70008C1181E480938D1182E090E00E9439061E
:10FC800080911B12882309F472C190911E128091F9
:10FC90001F12981708F06BC180E060E00E949F047B
:10FCA0008091B311882321F08091B11180FD32C081
:10FCB0002091B411CE0145962223B1F4ADB7BEB761
:10FCC0001E970FB6F894BEBF0FBEADBFEDB7FEB71F
:10FCD000319612969C938E93119784E190E09383D2
:10FCE000828383ED99E031C0ADB7BEB71A970FB6E6
:10FCF000F894BEBF0FBEADBFEDB7FEB731961296FA
:10FD00009C938E93119784E190E0938382838BEE92
:10FD100099E051C02091B411CE0145962223B1F54E
:10FD2000ADB7BEB71E970FB6F894BEBF0FBEADBF3E
:10FD3000EDB7FEB7319612969C938E93119784E19E
:10FD400090E09383828382E09AE09583848380911C
:10FD5000181290E001969783868380919B11909171
:10FD60009C11A0919D11B0919E1180879187A287CF
:10FD7000B38780911E1290E00D96958784870E942C
:10FD8000CEA72DB73EB7225F3F4F29C0ADB7BEB754
:10FD90001A970FB6F894BEBF0FBEADBFEDB7FEB752
:10FDA000319612969C938E93119784E190E0938301
:10FDB00082838AE19AE0958384838091181290E08F
:10FDC00001969783868380911E1290E00D9691870D
:10FDD00080870E94CEA72DB73EB7265F3F4F0FB654
:10FDE000F8943EBF0FBE2DBFCE0145960E944B0634
:10FDF0000091D4111091D5118091B311882391F401
:10FE00008091DE10882329F48091D6119091D7112A
:10FE100004C08091DA119091DB11909304138093C8
:10FE2000031331C08091B11180FF05C08091DC11B6
:10FE30009091DD11F2CF8091DD109091DE1088233A
:10FE400089F4992301F58091D8119091D91190935B
:10FE500004138093031384E08093DD1081E080938A
:10FE6000DE1011C081508093DD10992361F0813044
:10FE700051F48091DA119091DB11909304138093E7
:10FE800003130E9406778091B4118823A9F4E090AF
:10FE9000DE11F090DF1161E00E949F0460919311E8
:10FEA00070919411809195119091961141E35AE0CF
:10FEB00025E00E94930604C0E090E011F090E1116B
:10FEC0008EE061E00E949F0460918F11709190110B
:10FED000809191119091921141E35AE025E00E94A6
:10FEE00093068091B411882311F583E062E00E94AB
:10FEF0009F04609197117091981180919911909140
:10FF00009A1147E35AE027E00E9493068BE062E0F3
:10FF10000E949F0460919F117091A0118091A11186
:10FF20009091A21147E35AE027E00E94930687E0F0
:10FF300063E00E949F0480910313909104130E9438
:10FF40004B0682E063E00E949F04C7010E944B06BB
:10FF5000F801D8010D900020E9F7EA1B8E2F8B5E87
:10FF600063E00E949F04C8010E944B0602C00E94E9
:10FF70004677A8960FB6F894DEBF0FBECDBFCF91DF
:10FF8000DF911F910F91FF90EF9008950F931F93B2
:10FF9000109105131F5F10930513143021F48DE1A8
:10FFA0000E94D9050AC0009106130E94967710930B
:10FFB0000513009306130E94057C1F910F9108956D
:10FFC0008091A811813019F40E94441F089581E0A6
:10FFD0008093A71108958091A911882309F45FC027
:10FFE0008091A811833081F18430E9F18230E9F009
:10FFF0002091941130919511409196115091971143
:020000021000EC
:1000000080911D12609119120E94707220919811B6
:100010003091991140919A1150919B1180911D122C
:10002000609119120E947B723AC020919811309110
:10003000991140919A1150919B1180911D126091DC
:1000400019120E94A6712BC020919811309199111C
:1000500040919A1150919B1180911D12609119123B
:100060000E9453711CC020919411309195114091C0
:1000700096115091971180911D12609118120E9453
:100080000B71209198113091991140919A115091D2
:100090009B1180911D12609118120E94167110928E
:1000A000A91108950E94EB7F0E94BC050895EF926C
:1000B000FF920F931F938091A811833009F45AC0C7
:1000C000843009F484C0823061F180911D12609106
:1000D00019120E941A746093941170939511809371
:1000E00096119093971180911D12609119120E94A0
:1000F0001F74609398117093991180939A11909343
:100100009B1180E090E0DC0180939C1190939D1105
:10011000A0939E11B0939F1180E090E0A0E7B3E41C
:1001200082C00F2EF0E0EF2EF0E0FF2EF6E90F2F49
:10013000F3EC1F2FF02DE0929411F09295110093A3
:1001400096111093971180911D12609119120E94BF
:10015000C773609398117093991180939A1190933B
:100160009B11E0929C11F0929D1100939E111093AF
:100170009F1155C00F2EF0E0EF2EF0E0FF2EFAE7B2
:100180000F2FF4EC1F2FF02DE0929411F0929511A7
:10019000009396111093971180911D12609119127E
:1001A0000E944270609398117093991180939A11F4
:1001B00090939B11E0929C11F0929D1100939E11DF
:1001C00010939F1180E090E0AAE7B4E42CC08091E6
:1001D0001D12609118120E946C73609394117093B9
:1001E0009511809396119093971180911D126091B3
:1001F00018120E94727360939811709399118093F2
:100200009A1190939B1180E090E0A6E9B3EC809363
:100210009C1190939D11A0939E11B0939F1180E02B
:1002200090E0A6E9B3E48093A0119093A111A0936C
:10023000A211B093A3111F910F91FF90EF90089519
:10024000EF92FF92CF93DF938093A8111092A711A2
:100250001092A6111092AA111092A91188EC90E0A8
:100260000E9489050E945780CAE7D1E1CE0160E271
:1002700070E044E150E00E9471A78EE50E945E129A
:10028000BC01FC0101900020E9F73197E81BF90B54
:100290002AE030E02E1B3F0B36952795265F3F4F17
:1002A0002C0F3D1FC901AF010E9468A780E090E0BC
:1002B0000E943906CE0160E270E044E150E00E9405
:1002C00071A781E090E00E9439068EE20E945E12E2
:1002D000BC01FC0101900020E9F73197E81BF90B04
:1002E000CE01AF010E9468A780E30E945E12BC01AC
:1002F000FC0101900020E9F73197E81BF90B9E0102
:100300002E1B3F0B2C5E3F4FC901AF010E9468A717
:1003100082E090E00E943906CE0160E270E044E1A4
:1003200050E00E9471A78FE20E945E12BC01FC01A6
:1003300001900020E9F73197E81BF90B9E012E5F31
:100340003F4FC901AF010E9468A781E30E945E127E
:10035000BC01FC0101900020E9F73197E81BF90B83
:10036000CE1BDF0B6296CE01AF010E9468A783E02F
:1003700090E00E9439060E941A120E944822DF91E2
:10038000CF91FF90EF90089584E00E9420818EE04D
:100390000E945E129093D1118093D0118EE30E943F
:1003A0005E129093D3118093D211089581E00E9440
:1003B00020818DE00E945E129093D1118093D01124
:1003C0008BE30E945E129093D3118093D2118CE341
:1003D0000E945E129093D5118093D4118DE30E94F8
:1003E0005E129093D7118093D61108950E94EB7FEF
:1003F0008091A811823029F0833049F00E94BC0519
:10040000089581E08093A8111092A71106C082E0A0
:100410008093A81181E08093A7110E9457800895CE
:100420000E94EB7F8091A811813019F0823071F425
:1004300004C092E09093A81104C083E08093A811B7
:1004400081E08093A7110E94578008950E94BC0507
:100450000895EF92FF920F931F93DF93CF93CDB741
:10046000DEB728970FB6F894DEBF0FBECDBF0E944F
:10047000152580E060E00E949F04E091A711F0E064
:10048000EE0FFF1FE155FE4E808191810E944B06C9
:100490008091A8118E010F5F1F4F843009F042C078
:1004A00080E061E00E949F048DB79EB708970FB669
:1004B000F8949EBF0FBE8DBFEDB7FEB73196ADB7B6
:1004C000BEB712961C930E93119788E090E0938329
:1004D00082838091D0119091D111958384838091F2
:1004E000181290E00196978386830E94CEA78DB75D
:1004F0009EB708960FB6F8949EBF0FBE8DBFC80179
:100500000E944B0686E061E00E949F048091D21118
:100510009091D3110E944B0682E161E00E949F04FA
:1005200081E453C080E061E00E949F04ADB7BEB794
:1005300018970FB6F894BEBF0FBEADBFEDB7FEB7AC
:10054000319612961C930E93119788E090E0938356
:1005500082838091D0119091D11195838483809171
:10056000191290E00196978386830E94CEA78DB7DB
:100570009EB708960FB6F8949EBF0FBE8DBFC801F8
:100580000E944B068091A811823041F0833061F0C7
:10059000E090D211F090D31106E50BC0E090D41199
:1005A000F090D51101E405C0E090D611F090D7117C
:1005B00007E585E061E00E949F04C7010E944B06A9
:1005C00082E161E00E949F04802F0E94B2048BE0D0
:1005D00061E00E949F04E091A711F0E0EE0FFF1F81
:1005E000EE0FFF1FE157FE4E658176818781908572
:1005F00045E55AE027E00E94930628960FB6F89446
:10060000DEBF0FBECDBFCF91DF911F910F91FF9045
:10061000EF900895772767FD7095E82FF0E0EE0FD3
:10062000FF1FEE0FFF1FE60FF71FEE0FFF1FEE0F6E
:10063000FF1FE152FF4E5081418132812381652F9E
:10064000742F832F922F0895EF92FF920F931F9391
:10065000262F332727FD3095482F50E0CA01880FF9
:10066000991F880F991F820F931F880F991F880F5A
:10067000991F81529F4E0F2EF0E0EF2EF0E0FF2EDB
:10068000F0E00F2FF0E01F2FF02DFC01E082F1824F
:1006900002831383E6EAF0E04E9FB0014F9F700D96
:1006A0005E9F700D11246E5A7E4F44E0220F331F5F
:1006B0004A95E1F7620F731F0E944E281F910F9118
:1006C000FF90EF9008952F923F924F925F926F921A
:1006D0007F928F929F92AF92BF92CF92DF92EF92D2
:1006E000FF920F931F93DF93CF9300D00F92CDB75C
:1006F000DEB74983682E7724A62EBB249301220FF0
:10070000331F220F331F2A0D3B1D220F331F220FD1
:10071000331F3B832A831FED812E10E1912E820E21
:10072000931EF401208031804280538096EA899F95
:10073000C0011124825A9E4F9501B4E0220F331F4D
:10074000BA95E1F7C090D504D090D604E090D704D4
:10075000F090D804820F931F40E050E068E472EC00
:1007600000E010E028E432E40E9416296B017C01CD
:100770000A811B8101501F4EF801608171818281C5
:1007800093810E9450A49B01AC01C701B6010E9455
:1007900004A56B017C01F9812F2F30E0B901882776
:1007A00077FD8095982F0E9450A49B01AC01C70152
:1007B000B6010E94B5A320E030E64AE657E40E9465
:1007C000B5A39B01AC01C201B1010E944DA3F4018C
:1007D0006083718382839383F80110821182128275
:1007E0001382F301EE0FFF1FEA0DFB1DED5DFE4EC0
:1007F00010820F900F900F90CF91DF911F910F916A
:10080000FF90EF90DF90CF90BF90AF909F908F9030
:100810007F906F905F904F903F902F9008954F92F0
:100820005F927F928F929F92AF92BF92CF92DF9210
:10083000EF92FF920F931F93DF93CF930F92CDB759
:10084000DEB7823058F44FEDE42E40E1F42E32E56D
:10085000832E31E0932E442455242CC08430B1F5EE
:10086000F2CFF8018081882359F0872D622F4CE365
:1008700029830E946383C601B5010E944E28298105
:100880002F5F0F5F1F4F84E090E0C80ED91EE0E19C
:10089000F0E0AE0EBF1E243021F70894411C511C1D
:1008A000EE0EFF1E86EA90E0880E991E92E0491631
:1008B000510451F0742C8201000F111F0D5D1E4E6A
:1008C0005401670120E0CDCF10923D110F90CF91E0
:1008D000DF911F910F91FF90EF90DF90CF90BF902D
:1008E000AF909F908F907F905F904F9008958F92E0
:1008F0009F92AF92BF92CF92DF92FF920F931F937E
:10090000DF93CF930F92CDB7DEB7F82E662319F49D
:1009100021E030E034C0882E9924840164E0000F87
:10092000111F6A95E1F701501F4E880C991C83E254
:1009300091E1880E991E20E0F801A080B180C2806C
:10094000D3808F2D622F29830E94D16FAA2797FD14
:10095000A095BA2F8A0D9B1DAC1DBD1DF80181937A
:100960009193A193B1938F01F40180818F5F819363
:100970004F0129812F5F2430F9F620E030E0C901D2
:100980000F90CF91DF911F910F91FF90DF90CF904B
:10099000BF90AF909F908F9008956F927F928F92AB
:1009A0009F92AF92BF92CF92DF92EF92FF920F93FE
:1009B0001F93CF93DF9380913D11882309F060C08E
:1009C00080911B12833009F05BC002E511E0C0E0AA
:1009D000D0E01FC0C7010E94D628F4016193719333
:1009E000819391934F01F5011192119211921192FD
:1009F0005F01F60111926F0180E190E0E80EF91EAF
:100A0000E614F70439F721960A551F4FC230D10575
:100A100001F1CE01B4E0880F991FBA95E1F7AFED6F
:100A20008A2EA0E19A2E880E991EFFEFAF2EF0E1DC
:100A3000BF2EA80EB91E6E01CC0CDD1CE3E2F1E165
:100A4000CE0EDF1E70E4672E712C600E711E7801D1
:100A5000C1CF8091FB0D9091FC0DA091FD0DB09147
:100A6000FE0D80931F1190932011A0932111B0933C
:100A7000221110923B1110923C1181E080933D11A4
:100A8000DF91CF911F910F91FF90EF90DF90CF906A
:100A9000BF90AF909F908F907F906F9008955F92DE
:100AA0006F927F928F929F92AF92BF92CF92DF927E
:100AB000EF92FF920F931F93CF93DF938091FB0DE3
:100AC0009091FC0DA091FD0DB091FE0D20911F1194
:100AD0003091201140912111509122117C018D0102
:100AE000E21AF30A040B150BA8019701243631050D
:100AF0004105510508F469C080931F11909320119E
:100B0000A0932111B09322110E94CD8480913D11B8
:100B1000882309F45AC087E794E860E070E00E94F7
:100B20009F5B80913B118F5F80933B118C3308F466
:100B30004CC010923B1180913C118F5F80933C110F
:100B4000893610F4EE2404C010923C11EE24E39494
:100B50002FEDC22E20E1D22E92E5692E91E0792E62
:100B6000C0E0D0E028C0F8014081442351F0852D39
:100B70006F2D0E946383EE2021F0C501B4010E9415
:100B80004E28F3940F5F1F4F84E090E0A80EB91E2B
:100B9000E0E1F0E08E0E9F1EF4E0FF1621F72196B3
:100BA00000E110E0C00ED11E86EA90E0680E791ECA
:100BB000C230D10551F05C2E8E01000F111F0D5D6A
:100BC0001E4E43015601FF24CECFDF91CF911F91DE
:100BD0000F91FF90EF90DF90CF90BF90AF909F90DC
:100BE0008F907F906F905F90089580911E1260911A
:100BF00019120E9424830895CF92DF92EF92FF9200
:100C00000F931F93DF93CF93CDB7DEB728970FB61F
:100C1000F894DEBF0FBECDBF8FE891E10E949446ED
:100C200080911E12609119120E940A836B017C014F
:100C30008DB79EB708970FB6F8949EBF0FBE8DBFB5
:100C4000EDB7FEB731968E010F5F1F4FADB7BEB740
:100C500012961C930E93119788E090E09383828301
:100C60008091D0119091D111958384838091191234
:100C700090E00196978386830E94CEA78DB79EB79A
:100C800008960FB6F8949EBF0FBE8DBF8AE061E054
:100C90000E949F04C8010E944B0680911B1288236A
:100CA00079F180919411843130F462E00E949F04C4
:100CB00080E20E94B204809194118F5F809394111E
:100CC000883210F01092941100919411102F1E5F31
:100CD000183210F0185206C0043120F4143128F0F4
:100CE00013E103C0143160F400E0802F62E00E9441
:100CF0009F0404C08BED0E94B2040F5F1017D0F761
:100D000083E063E00E949F04C701B6014BE85AE00C
:100D100027E00E94930628960FB6F894DEBF0FBE18
:100D2000CDBFCF91DF911F910F91FF90EF90DF909A
:100D3000CF900895EF92FF920F931F93DF93CF937D
:100D4000CDB7DEB728970FB6F894DEBF0FBECDBF84
:100D500084E690E00E94890585E2809394110AE779
:100D600011E1C80160E270E044E150E00E9471A727
:100D700081E00E945E12BC01FC0101900020E9F7B5
:100D80003197E81BF90B24E130E02E1B3F0B369521
:100D90002795200F311FC901AF010E9468A780E08D
:100DA00090E00E943906C80160E270E044E150E042
:100DB0000E9471A78CE00E945E122DB73EB72850AA
:100DC00030400FB6F8943EBF0FBE2DBFEDB7FEB753
:100DD00031967E010894E11CF11CADB7BEB71296A6
:100DE000FC92EE92119728E030E0338322839583C2
:100DF000848380911E1290E00D96978386830E94D3
:100E0000CEA7F70101900020E9F73197EE19FF090D
:100E100098012B5F3F4F8DB79EB708960FB6F89499
:100E20009EBF0FBE8DBFC901B701AF010E9468A769
:100E300081E090E00E943906C80160E270E044E180
:100E400050E00E9471A782E090E00E94390689E795
:100E50000E945E12BC01FC0101900020E9F731976D
:100E6000E81BF90BC801AF010E9468A784E20E9449
:100E70005E12BC01FC0101900020E9F73197E81BEC
:100E8000F90B0E1B1F0B0E5E1F4FC801AF010E9416
:100E900068A783E090E00E9439068FE891E10E9404
:100EA000D6460E941A128DE00E945E129093D111D4
:100EB0008093D0110E94FC8528960FB6F894DEBF6F
:100EC0000FBECDBFCF91DF911F910F91FF90EF909B
:100ED0000895CF93DF9384E060E00E949F04C8E30D
:100EE000D2E0CE010E944B0680E160E00E949F04A8
:100EF000CE0102960E944B0684E061E00E949F04AE
:100F0000CE010E944B06DF91CF910895EF92FF92A0
:100F10000F931F93DF93CF93CDB7DEB728970FB60C
:100F2000F894DEBF0FBECDBF8DB79EB708970FB642
:100F3000F8949EBF0FBE8DBFEDB7FEB731968E0100
:100F40000F5F1F4FADB7BEB712961C930E9311974C
:100F500088E090E0938382838091D0119091D111A9
:100F6000958384838091171290E0019697838683FE
:100F70000E94CEA78DB79EB708960FB6F8949EBF75
:100F80000FBE8DBF8BE060E00E949F04C8010E94ED
:100F90004B0680911B12882309F439C18091C1123C
:100FA0008F3F09F434C18091171290E00E9471675D
:100FB00090939A11809399118091171290E00E945A
:100FC000876760939B1170939C1180939D11909300
:100FD0009E118091171290E00E94816760939F118B
:100FE0007093A0118093A1119093A2118091171278
:100FF00090E00E94D3676093A3117093A411809333
:10100000A5119093A6118091171290E00E94CD67D0
:101010006093A7117093A8118093A9119093AA11BE
:101020008091171290E00E947B676093AB117093E0
:10103000AC118093AD119093AE118091171290E096
:101040000E9458676093AF117093B0118093B111F3
:101050009093B21180E161E00E949F046091AF1112
:101060007091B0118091B1119091B21149EA5AE09A
:1010700023E00E94930660919B1170919C118091D6
:101080009D1190919E112091A3113091A411409136
:10109000A5115091A6110E9404A50E9467A57B018D
:1010A0008C0184E062E00E949F04C801B7010E94A5
:1010B0001DA4DC01CB016FEA7AE045E00E944E06F8
:1010C00080E162E00E949F048091991190919A11B1
:1010D00063EB7AE043E00E944E0660919F117091AD
:1010E000A0118091A1119091A2112091A71130918E
:1010F000A8114091A9115091AA110E9404A50E9423
:1011000067A57B018C0184E063E00E949F04C80115
:10111000B7010E941DA4DC01CB016FEA7AE045E033
:101120000E944E068FE063E00E949F046091AB1125
:101130007091AC118091AD119091AE1147EB5AE0D6
:1011400024E00E9493068091C3128F3708F087C075
:101150008091171290E00E94956560938F117093B3
:10116000901180939111909392118091171290E0B9
:101170000E94D2656093931170939411809395119E
:10118000909396118091171290E00E949066909330
:1011900098118093971184E060E00E949F04609111
:1011A00093117091941180919511909196110E94D4
:1011B00067A50E941DA4DC01CB016FEA7AE045E03F
:1011C0000E944E0680E160E00E949F04809197118A
:1011D0009091981163EB7AE043E00E944E0684E020
:1011E00061E00E949F0460918F1170919011809135
:1011F0009111909192110E9467A50E941DA4DC019B
:10120000CB016FEA7AE045E00E944E062AC080E1F9
:1012100061E00E949F048AE392E00E944B0684E012
:1012200062E00E949F0488E392E00E944B0680E106
:1012300062E00E949F048AE392E00E944B0684E0F1
:1012400063E00E949F0488E392E00E944B068FE0D7
:1012500063E00E949F048AE392E00E944B060E9492
:10126000698728960FB6F894DEBF0FBECDBFCF9129
:10127000DF911F910F91FF90EF900895CF92DF9231
:10128000EF92FF920F931F93CF93DF9384EF91E040
:101290000E948905CAE7D1E1CE0160E270E044E135
:1012A00050E00E9471A781E60E945E12BC01FC0121
:1012B00001900020E9F73197E81BF90BCE01AF014F
:1012C0000E9468A717E51093831103E400938D1122
:1012D00080E090E00E943906CE0160E270E044E1D7
:1012E00050E00E9471A78AE50E945E12BC01FC01D9
:1012F00001900020E9F73197E81BF90BCE01AF010F
:101300000E9468A782E60E945E12BC01FC01019067
:101310000020E9F73197E81BF90B8BE0E82EF12C60
:10132000EC0EFD1EC701AF010E9468A71093831148
:1013300085E280938D1181E090E00E943906CE0114
:1013400060E270E044E150E00E9471A783E60E94F1
:101350005E12BC01FC0101900020E9F73197E81B07
:10136000F90BCE01AF010E9468A71093831100937F
:101370008D1182E090E00E943906CE0160E270E0BB
:1013800044E150E00E9471A784E60E945E12BC0115
:10139000FC0101900020E9F73197E81BF90BCE0121
:1013A000AF010E9468A785E60E945E12BC01FC01A5
:1013B00001900020E9F73197E81BF90BC701AF0155
:1013C0000E9468A71093831186E580938D1183E0B6
:1013D00090E00E9439060E941A128BE00E945E1271
:1013E0009093D1118093D0110E948687DF91CF9185
:1013F0001F910F91FF90EF90DF90CF900895809113
:101400008F11882321F080919011813019F00E9472
:101410007711089510928F11089580918F11813066
:1014200021F080919111813019F00E946711089587
:1014300080938F1108958091171260E00E943B33D2
:10144000809390118091171261E00E943B3380934A
:10145000911180E090919011913009F481E090E039
:1014600020919111213009F491E0890F809392111C
:1014700008956F927F928F929F92AF92BF92CF9278
:10148000DF92EF92FF920F931F93CF93DF930E940F
:101490001B8A81E060E00E949F04E0919011F0E0DF
:1014A000EE0FFF1FE053FE4E808191810E944B069C
:1014B00081E061E00E949F04E0919111F0E0EE0F65
:1014C000FF1FE053FE4E808191810E944B0680E019
:1014D00060918F110E949F0480919211882311F4D2
:1014E00080E201C08AE20E94B20460E080918F1124
:1014F000882309F461E080E00E949F0480E20E945A
:10150000B20482E162E00E949F048091171290E091
:10151000019665ED7AE042E00E944E0680911B1232
:10152000882309F44AC08091C1128F3F09F445C055
:1015300085E060E00E949F046091291270912A1258
:1015400080912B1290912C124AED5AE027E00E94D4
:1015500093068DE060E00E949F04609121127091DB
:101560002212809123129091241240EE5AE026E03C
:101570000E94930685E061E00E949F0460912D1215
:1015800070912E1280912F12909130124AED5AE0F4
:1015900027E00E9493068DE061E00E949F04609125
:1015A000251270912612809127129091281240EEF8
:1015B0005AE026E00E94930620C085E060E00E9489
:1015C0009F0486E392E00E944B068DE060E00E945B
:1015D0009F0487E392E00E944B0685E061E00E9451
:1015E0009F0486E392E00E944B068DE061E00E943A
:1015F0009F0487E392E00E944B0680911B12882390
:1016000009F4D5C08091C1128F3F09F4D0C08091F8
:101610008F11E82FF0E0E157FE4E9181913009F0F3
:10162000C6C0882321F48091171262E003C0809124
:10163000171265E00E949A66929596959170E9F06E
:1016400080E062E00E949F048091DA119091DB11AA
:101650000E944B06E091DE11F091DF11DF010D9049
:101660000020E9F7EA1B8E2F8D5E63E00E949F0445
:101670008091DE119091DF111CC080E062E00E9439
:101680009F048091DC119091DD110E944B06E09146
:10169000E011F091E111DF010D900020E9F7EA1B64
:1016A0008E2F8D5E63E00E949F048091E0119091E7
:1016B000E1110E944B06E0918F11F0E0EE0FFF1F49
:1016C000EE0FFF1FE75BFD4E608171818281938188
:1016D0000E9467A57B018C018AE062E00E949F0462
:1016E000C801B7010E9422A4DC01CB0166EE7AE0BA
:1016F00043E00E944E06E0918F11F0E0EE0FFF1FD5
:10170000EE0FFF1FEF5BFD4E608071808280938043
:10171000C401B3010E94C9A57B018C0120E030E027
:10172000A9010E94B1A3882334F4C0E0D0E0AA2428
:10173000BB24650127C0C801B70120E03CE34CE1B0
:1017400056E40E9400A518164CF4CBE3D0E08FE0DD
:10175000A82E87E2B82EC12CD12C14C0C801B70125
:101760000E9422A45B01C401B301A80197010E9459
:101770004CA320E030E040E752E40E9404A50E9420
:1017800022A4EB0180E063E00E949F04C5016AEEA1
:101790007AE044E00E944E0685E063E00E949F04E8
:1017A000CE016EEE7AE042E00E944E0618C08AE05A
:1017B00062E00E949F048AE392E00E944B0680E070
:1017C00063E00E949F0489E392E00E944B0685E05B
:1017D00063E00E949F048BE392E00E944B06DF913E
:1017E000CF911F910F91FF90EF90DF90CF90BF901E
:1017F000AF909F908F907F906F900895EF92FF929F
:101800000F931F93CF93DF9384EF91E00E9489059C
:101810000E941B8A80919111813021F49091901146
:10182000913019F410928F1102C080938F118AE7C2
:1018300091E160E270E044E150E00E9471A707E5A9
:101840000093861111E410938D1180E090E00E94C6
:1018500039068AE791E160E270E044E150E00E94DD
:1018600071A70093861110938D1181E090E00E9482
:1018700039068AE791E160E270E044E150E00E94BD
:1018800071A785E2809387118FE30E945E12BC01ED
:10189000FC0101900020E9F73197E81BF90BC9E83A
:1018A000D1E1CE01AF010E9468A782E090E00E94E2
:1018B0003906CE010F9760E270E044E150E00E94EB
:1018C00071A78AE380937E1189E40E945E12BC01B5
:1018D000FC0101900020E9F73197E81BF90B24E1A6
:1018E00030E02E1B3F0B3695279526583E4EC901FA
:1018F000AF010E9468A783E090E00E9439060E9431
:101900001A128AE392E09093D1118093D0118EE461
:101910000E945E129093D3118093D21180E50E94B1
:101920005E129093D5118093D41184E50E945E12CB
:101930009093D7118093D61182E50E945E12909306
:10194000D9118093D81183E80E945E129093DB1125
:101950008093DA1184E80E945E129093DD118093E7
:10196000DC1185E80E945E129093DF118093DE11F6
:1019700086E80E945E129093E1118093E0110E942C
:10198000398ADF91CF911F910F91FF90EF900895C9
:101990009C01FB011AC081912827822F8295822702
:1019A000082E869586958025082E86958025877039
:1019B000022E232F869507948795302D282706948D
:1019C000879530252827415050404115510519F77A
:1019D000C901089581FF02C082E0089581700895D1
:1019E0001092171310921513109216138CE0E9E061
:1019F000F3E1DF011D928A95E9F708951F930E9494
:101A00007B64182F882321F480913E11882381F074
:101A10001092171310921513109216138CE19DE873
:101A200060E070E00E948B5C10933E11112311F472
:101A30000E94F08C1F9108951F93182F662311F4B4
:101A400090E022C00E94D967982F977092FF05C03E
:101A500091E090931513982F9370E12FF0E0E75FDA
:101A6000FC4E8081981781F0292F91FF02C022E05F
:101A700001C0217081FF02C082E001C0817028177F
:101A800019F081E080931613E12FF0E0E75FFC4E40
:101A9000908380E090E01F91089508950895DF936A
:101AA000CF9300D0CDB7DEB7BE016F5F7F4F42E06E
:101AB0000E94C84D998180E02A8130E0282B392B83
:101AC000C9010F900F90CF91DF910895CF92DF92CF
:101AD000EF92FF920F931F93CF93DF937C01EB0163
:101AE000FC01008111818AE0FB0111928A95E9F7DE
:101AF000C80142E00E94C84D99819F3F09F44AC045
:101B00008881829586958770282F30E026303105B0
:101B10000CF043C00E5F1F4F9072D9F0C8010E94B5
:101B20004F8D6C010E5F1F4FC8010E944F8D0E5FDD
:101B30001F4F960140E050E0A90133272227A0E083
:101B4000B0E0282B392B4A2B5B2B2A833B834C8319
:101B50005D83898187FF0CC0C8010E944F8D8E83F1
:101B60009F838F7390E08C339105BCF40E5F1F4F01
:101B70008981807461F0BE01685F7F4FC80142E0D7
:101B80000E94C84D88858F3140F40E5F1F4FF701CA
:101B90001183008320E030E002C02FEF3FEFC90146
:101BA000DF91CF911F910F91FF90EF90DF90CF9039
:101BB0000895CF92DF92EF92FF920F931F9381E0EF
:101BC00080933F1187EE92E061E070E048E552E0DB
:101BD00021E030E00E94A9289093BC148093BB14AC
:101BE00089EE92E061E070E048E552E023E030E009
:101BF0000E94A92890932913809328138BEE92E0DA
:101C000061E070E048E552E023E030E00E94A9285E
